:020000040000FA
:10000000787A00200D57000045900000B55500009B
:10001000B5550000B5550000B5550000B5550000B8
:10002000B5550000B5550000B5550000FD51000064
:10003000B5550000B5550000A5510000858F0000A2
:10004000E5560000E5560000E5560000E5560000C4
:10005000E5560000E5560000E5560000E5560000B4
:10006000E5560000E5560000E5560000E5560000A4
:10007000E5560000E5560000E5560000E556000094
:10008000E5560000E5560000E5560000E556000084
:10009000E5560000E5560000E5560000E556000074
:1000A000E5560000E5560000E5560000E556000064
:1000B000E5560000E5560000E5560000E556000054
:1000C000E5560000E5560000E5560000E556000044
:1000D000E5560000E5560000E5560000E556000034
:1000E000E5560000E5560000E5560000E556000024
:1000F000E5560000E5560000E5560000E556000014
:100100007BB972B90029BEBF00204FF0004106E064
:1001100008BF00281CBF6FF000414FF0FF3000F017
:10012000BDB9ADF1080C6DE904CE002909DB002B47
:100130001ADB00F04DF8DDF804E0DDE9022304B03D
:100140007047404261EB4101002B1BDB00F040F89F
:10015000DDF804E0DDE9022304B0404261EB410137
:10016000524263EB43037047524263EB430300F098
:100170002FF8DDF804E0DDE9022304B0404261EB32
:1001800041017047524263EB430300F021F8DDF870
:1001900004E0DDE9022304B0524263EB43037047FD
:1001A00053B94AB9002908BF00281CBF4FF0FF31DE
:1001B0004FF0FF3000F072B9ADF1080C6DE904CEDC
:1001C00000F006F8DDF804E0DDE9022304B0704732
:1001D0002DE9F047089E04468846002B4BD18A4201
:1001E000154667D9B2FA82F24AB1C2F1200701FA84
:1001F00002F320FA07F7954047EA030894404FEAD4
:10020000154E230CB8FBFEF71FFA85FC0EFB178872
:1002100043EA084307FB0CF1994209D9EB1807F1AF
:10022000FF3080F01B81994240F21881023F2B443D
:100230005B1AA4B2B3FBFEF00EFB103344EA034496
:1002400000FB0CFCA44509D92C1900F1FF3380F008
:100250000781A44540F2048102382C4440EA07405B
:10026000A4EB0C0400271EB1D4400023C6E90043D0
:100270003946BDE8F0878B4209D9002E00F0EB80AB
:100280000027C6E9000138463946BDE8F087B3FAD1
:1002900083F7002F47D18B4202D3824200F2FA80CB
:1002A000841A61EB030301209846002EE0D0C6E9D2
:1002B0000048DDE702B9FFDEB2FA82F2002A40F020
:1002C0008F80491B4FEA154E1FFA85F80127B1FBB5
:1002D000FEFC230C0EFB1C1143EA014308FB0CF14E
:1002E000994207D9EB180CF1FF3002D2994200F283
:1002F000CD808446591AA3B2B1FBFEF00EFB101458
:1003000043EA044408FB00F8A04507D92C1900F182
:10031000FF3302D2A04500F2B6801846A4EB0804D1
:1003200040EA0C409FE7C7F1200CBB4022FA0CFECC
:100330004EEA030E01FA07F420FA0CF521FA0CF349
:100340004FEA1E482543B3FBF8F92C0C08FB193380
:100350001FFA8EFA44EA034309FB0AF49C4202FAAC
:1003600007F200FA07F10BD91EEB030309F1FF3086
:1003700080F087809C4240F28480A9F10209734496
:100380001B1BADB2B3FBF8F008FB103345EA034486
:1003900000FB0AFAA24508D91EEB040400F1FF3362
:1003A0006BD2A24569D90238744440EA0940A0FBE7
:1003B0000289A4EB0A044C45C2464B4654D351D0A3
:1003C000002E69D0B1EB0A0564EB030404FA0CFCBF
:1003D000FD40FC404CEA0505C6E90054002747E70C
:1003E000C2F1200320FA03F7954001FA02F021FA46
:1003F00003F34FEA154E3843010CB3FBFEF71FFA27
:1004000085F80EFB173341EA034107FB08F38B42E3
:1004100004FA02F407D9691807F1FF3C2FD28B4286
:100420002DD9023F2944CB1A81B2B3FBFEF00EFB5B
:10043000103341EA034100FB08F38B4207D96918E6
:1004400000F1FF3C17D28B4215D902382944C91A52
:1004500040EA07473BE73746304609E70746E7E605
:100460001846FBE64145ABD2B8EB020A69EB0E0237
:1004700001381346A4E76046E9E7184695E7674662
:10048000D1E781467CE702382C4447E7ACF1020C07
:100490002B442FE7384608E73746E9E6704700BFA8
:1004A00070B586B000F06EF81F4800F043F800B950
:1004B000FEE71E4806F080FC436804461D680D22D6
:1004C0004FF480730021A84763680D229D680021C6
:1004D00001AB2046A847019B23B904F077FA1448E2
:1004E00004F0ECFD03A800F00BFB00B1FEE702A94D
:1004F0009DF8100007F056FC029B059C1C44039BD2
:100500001D8966194FF02002EFF3118382F31188E1
:10051000BFF36F8F08F037FD02F0CEFC635983F311
:10052000088873689847FEE7ACC00000BFC00000B1
:1005300018BD000010B5044C236813B906F03CFC4C
:100540002060206810BD00BF0800002002289ABF6C
:10055000024B53F820006FF01500704720BD0000DB
:100560001FB5074B0C4601AA014618680AF0DBFBD1
:1005700018B9019B2360029B636004B010BD00BFEB
:10058000080000204FF4C051014805F015BB00BF22
:10059000D62800202DE9F84F0A9EDFF84CB0074618
:1005A000884691469A460024B44201D300200EE0CA
:1005B000351BB5F5806F28BF4FF480652B460A4A7E
:1005C00004EB0901384608F02AFC10B10120BDE80F
:1005D000F88F2B465A4604EB0A01404608F03CFCD3
:1005E0000028F3D12C44DFE7D64000202DE9F34169
:1005F000DFF84C80064600252C272846FFF7A6FF8B
:1006000001A9C0B203F0B4F8014698B9202307FB52
:100610000582019808F003FC041C18BF012401980E
:1006200008F0FCFB44B1002D18BF3446204602B050
:10063000BDE8F0810124F2E7002DF7D10125DCE7C8
:100640000C000020F0B587B00546FFF77FFF04A936
:10065000C0B203F08DF8002843D12846FFF776FF9B
:10066000214E2C2405A9C0B204FB056403F080F8D8
:1006700088B12C226A43B3181B6913F0100315D1FB
:10068000B1581A4A914219D085B104980021826864
:1006900008F00BFC0AE0059807F08AFB074605986E
:1006A00008F0BCFB631EE21C9A4202D14FF0FF34FB
:1006B00011E013F8011FB942F6D0DAE7CDE90133B2
:1006C000009320464FF48073094A049900F082FC9D
:1006D00004460028D8D1049808F0A0FB204607B0B3
:1006E000F0BD0124FAE700BF0C0000203DB8F396EE
:1006F000D64400202DE9F8430378022B074623D087
:10070000052B23D10125124B2C2202FB053593F832
:100710006400AC6A07F0C9FB04F10054013C804658
:10072000E40000266B6A1A191959D2F804901B6864
:100730004A46C91A38464E4408F0B7FBB045A4F102
:100740000804EFD8BDE8F8830025DCE70120F9E7CD
:100750000C00002073B502AD802645F8046D174CDF
:100760002946626A022003F017F840B9019B226D06
:10077000A36229460520019603F00EF808B1012571
:1007800018E0019BE26D636529460620019603F09F
:1007900003F805460028F2D1019B206A236608F081
:1007A000AAFB0646A06D08F0A6FBB04238BF304653
:1007B00084F86400284602B070BD00BF0C00002021
:1007C0002DE9F041224B82B01D68EB1D23F0070399
:1007D00000AFADEB030D4379002B064607F1040192
:1007E00014BF0620022002F0C3FF78BB786807F030
:1007F0006FFB184B347993F864203368013C013B5C
:1008000002EB4201544301FB03440444786808F0BE
:1008100072FB8046786807F0CBFA2A4601466846A4
:1008200008F071FC33798DF80030214643466A4662
:10083000786808F011FB041C18BF0124786808F0E0
:10084000EDFA20460837BD46BDE8F0810124F5E702
:1008500038BD00000C0000202DE9F04F04468BB09D
:100860002368A34E0020012BCDE905003CD123795C
:10087000012B39D19F4D3268AA4203D106AA3146D5
:1008800007F0ADFAF36AAB4204D105AA9A490120F8
:1008900007F0A5FADDE90532934288BF0693069B6F
:1008A000A36000230699376DD6F824C01A461D466A
:1008B000914202D89A4280F01181E8000CEB000EC0
:1008C0009942DEF804E0724402D8934280F0048139
:1008D000384491424068034404D8994202D89A426D
:1008E00000F0F5800135E3E704F1080000F0DCFAE0
:1008F000A3680693D5E7B36D726A99684FF0000854
:1009000002EBC5035B684344994203D3013D98461B
:100910006B1CF5D12368013B5B4500F2C6806B1C64
:1009200096F8640052F833701368FF1A07F0BDFAA6
:10093000B36A726A013B07EB080152F83330126860
:100940009B1A994223688CBFA8EB000AC246012B70
:1009500040F0B480BAEB080318BF0123637107A904
:10096000022002F005FF08A9052002F001FF09A9F5
:10097000062002F0FDFE2379012B23D142460021FF
:10098000099808F092FA0023CDF800A03A46DDE974
:100990000801FFF7FFFD2368012B08D1637904F1FB
:1009A0000801002B00F08C80099807F045FA02231B
:1009B00023712046FFF704FF20B1D9F8003001333E
:1009C000C9F800302379022B1FD1424639460898D6
:1009D00008F06BFA3B46CDF800A03A46DDE9070186
:1009E000FFF7D8FD2368012B04D1637913B9089868
:1009F000FFF780FE032323712046FFF7E1FE20B1BD
:100A0000D9F800300133C9F800302379032B43D1E2
:100A100042463946079808F048FA3B46CDF800A010
:100A2000002207990998FFF7B5FD637933B3099858
:100A300007F04EFA96F86430079903EB43030093EE
:100A400002460AEB07030998FFF7A4FD20B1D9F885
:100A500000300133C9F8003004A9062007F060FA1D
:100A60009DF81230012B02D1079807F068FAA168AF
:100A7000079807F068FA079800F05AFA23680133DC
:100A800023600123A3802046FFF79AFE20B1D9F806
:100A900000300133C9F80030079808F0BFF9089812
:100AA00008F0BCF9099808F0B9F90BF1010B002D19
:100AB000BFF621AF00200BB0BDE8F08F00234DE75B
:100AC00007980391FFF716FE039907986DE74FF01B
:100AD000000BDFF82890EAE79142FFE6994202D83E
:100AE0009A427FF6FCAE07EBC50040680344F4E68B
:100AF0000C0000203DB8F396380000207400002060
:100B00002DE9F04FAA4CAB4B6362AB4B236589B028
:100B1000AA4BE36506460020FFF718FD04F120010B
:100B2000C0B202F025FE0120FFF710FD04F14C01D8
:100B3000C0B202F01DFE04F15801062002F018FEBA
:100B4000FFF708FE054600285ED1FFF74FFD05467A
:100B5000002859D1D4F82880B8F1800F00F24881DC
:100B6000D4F854E0BEF1800F00F24281A36DD4F8B6
:100B700050A09B68D4F82490019302460146074692
:100B80008446034688454CD896454AD8884540F067
:100B90002F81964540F02C81BC4540F029810C22E4
:100BA000002105A808F0AFFA012304A9022005934B
:100BB0008DF8183007F0B4F903A9062007F0B0F952
:100BC0007F499DF810C09DF80CE09DF8118000232E
:100BD0000A4611F82350042D4FEA830001D0AC459A
:100BE0004FD115186F78042F01D0BE4549D1AD788B
:100BF000042D01D0454544D10244D078012863D06A
:100C000042D3022861D00725A06D08F007F9E06CF7
:100C100008F004F9206A08F001F9284609B0BDE897
:100C2000F08FAB4216D109EBC10B0131DBF804B0F8
:100C30005B440AEBC20B0132DBF804B05D44AB420B
:100C4000A0D1019898429C441F44C0F0D18000205C
:100C5000054696E70AD209EBC10B0228DBF804B07F
:100C60005B4400F0C58001310120E8E70AEBC20BCC
:100C70000128DBF804B05D4400F0BA8001320220A4
:100C8000DDE70133042BA4D1059B012B03D19DF893
:100C90001870012F61D005A8FFF7DEFD00F056F9AE
:100CA0000428054666D0FF2803D001280CBF032581
:100CB00005252B1F012B5FD9013D042D74D8DFE8DA
:100CC00005F0978181819000062004A902F050FD73
:100CD000054608B1012597E7DDF81090484607F072
:100CE000F7F88346484607F0E5F8A84682462F46BF
:100CF000C24504DC3DB3002F08BF474616E094F818
:100D00006410012303AA08FB01B1484607F052F81A
:100D1000002820DB012806D115B1002F08BF474667
:100D200008F10108E4E7A5B1002FF9D0013F032342
:100D300097FBF3F35A1C03EB4303FF1A01370592A9
:100D40008DF818700025049808F068F8002D9BD0E5
:100D50005AE70125E4E70125F5E700F0F7F8831EDF
:100D6000022B0546A5D83846FFF76CFC00284DD06D
:100D700005259EE702259CE705A9022002F0F8FC64
:100D800090B904A9059800F045F8074668B99DF8A0
:100D900012300598032B02D107F0D1F807460598C9
:100DA00008F03CF8002F87D0FEE70127F7E700BFE7
:100DB0000C00002078000020780800207804002033
:100DC000C6C0000005A9022002F0D2FC0028EBD129
:100DD000059807F0B0F80546059808F01FF8002DB3
:100DE000E2D10020FFF702FC054600287FF40CAF9B
:100DF0000020FFF727FC054630B9236A5A78327184
:100E00005B68B3603460FFE60325FDE605A8FFF7E5
:100E100023FD4EE730B50C46816885B010236A4645
:100E20001039054606F0C6FF002802DA012005B099
:100E300030BD012820D1032323702B78062B0CD042
:100E4000A9680123E2182039284606F0B3FF0028DC
:100E5000ECDB01281AD103236370A9680123A21CCB
:100E60001839284606F0A6FF0028DFDB012813D139
:100E70000323A3700020DAE710220A49684608F02D
:100E800005F9002814BF02230123D5E76378012B5D
:100E90000CBF01230223DFE7A378012B0CBF012342
:100EA0000223E6E73CBD000010B586B0044601A968
:100EB000022002F05DFC18B10124204606B010BDEE
:100EC00001988168102302AA103907F0A8FF20B109
:100ED0000124019807F0A2FFEFE71022134902A8AE
:100EE00008F0D4F868B9019803788168062B1BD103
:100EF00020392246042307F092FF041C18BF012466
:100F0000E7E7019807F08AFF01A9062002F030FC0C
:100F10000028D1D101988168102302AA103907F066
:100F20007EFF0028D4D1DEE72839E2E73CBD00008F
:100F30008168054A08B51039102307F08DFF00308D
:100F400018BF012008BD00BF3CBD00002DE9F341E2
:100F50000220694606F0D0FFB8BB01A9052006F0C3
:100F6000CBFF90BB1A4A9DF800409DF804509DF8B5
:100F700002609DF806709DF801C09646835C042BC4
:100F800002EB000801D0A3421AD10EEB00035978FE
:100F9000042901D0A94213D19978042901D0B14282
:100FA0000ED1D978042901D0B94209D11B79042B7B
:100FB00004D198F8050002B0BDE8F0816345F8D08F
:100FC00006301228DAD10120F5E7FF20F3E700BF51
:100FD000D6C000002DE9F04FF3B007467C9C7D9D04
:100FE00032A8884692461E4609F053FC002132A8DA
:100FF00009F053FC34B1002D04DD2A46214632A805
:1010000009F08AFCB7F80890FB6800249944A145D0
:1010100021D807A932A809F016FD7E9B23B1202212
:1010200007A9184608F042F8FB683C891C4405AA49
:1010300004232146404607F0F2FE834638B9BDF846
:10104000141046F6071291421AD04FF0FF3B584653
:1010500073B0BDE8F08FA9EB0405B54228BF354653
:101060002B4652462146404607F0D9FE83460028CB
:10107000EDD12A46514632A809F04EFC2C44C6E771
:10108000BDF81620DFF83891DFF838A10290131967
:101090000393043406464FF0FF35039B9C4208D36C
:1010A000029B002BD1D0B6FA86F67609C6F1000B6A
:1010B000CDE7042306AA2146404607F0B0FE83464A
:1010C0000028C4D19DF818B0BDF81A70BBF1100FFC
:1010D00018D1202FB9D13B4632AA211D404607F036
:1010E0009EFE83460028B2D13A4632A907A807F0EF
:1010F000CDFF0028A9D101230293BDF81A30043393
:101100001C44CAE7BBF1010F32D1202F9DD83B46CA
:1011100032AA211D404607F082FE8346002896D160
:101120009DF81A70D9F80050AB4503DB4FF0FF3B38
:101130005D46E2E717A809F0ACFB002117A809F00B
:10114000ACFB0AEBCB025AF83B10526817A81268A6
:1011500009F0E2FB0FA917A809F075FC3A4632A97D
:101160000FA807F093FF0028E2D00BF1010BDBE79B
:10117000BBF1200FC1D1002D1FDBD9F80030AB42ED
:101180001BDDB7F5807F7FF460AF3B4632AA211D9F
:10119000404607F044FE00287FF457AFEDB20095BB
:1011A000BDF81A3032AA594607A800F00DF80028F9
:1011B0004FF0FF3508BF01269FE74FF0FF359CE752
:1011C0002CBD000030BD00002DE9F04F1746ADF5F5
:1011D0004B7D00228046894627A811469DF8506322
:1011E0001D4609F012FB714B53F83640029403EB95
:1011F000C6038AAE5B681B681C4432463023214616
:1012000002A807F0EAFF10B14FF0FF34BAE0029BEA
:10121000326813449C4240F0C68029AA214602A8A5
:1012200007F0EFFF002840F0BB800DF1B00B5A46ED
:10123000214602A807F0E5FF8246002840F0B08072
:1012400029A808F042FB029B28909C4240F0A58010
:10125000CDE900AB5346524629A927A809F091FAD7
:10126000002840F0978027A804F052FD044600288B
:1012700040F0868029A808F028FB8542289040F09D
:101280008180B5F5807FBFD1B9F1200FBCD1324646
:10129000394627A804F060FD05460028B4D196F829
:1012A000FF30BC2BB0D10DF5A4790390DF274C465D
:1012B0000CA809F0EEFA00210CA809F0EEFA2022A1
:1012C0000DF207310CA809F027FB042203A90CA892
:1012D00009F022FB04A90CA809F0B5FB1F2F9DF80B
:1012E0000F30D4BFBA464FF0200A01334846524669
:1012F00004A9A7EB0A078DF80F3007F0D7FE002FDF
:10130000D144D5DC0023E25CF15C4A40E254013375
:10131000DF2BF8D1237803F07F032370665D002E66
:101320007FF472AF0135BE2DF8D194F8BE30012B99
:101330007FF46AAF0CA809F0ACFA31460CA809F0AA
:10134000ACFA08221A490CA809F0E6FA2022414614
:101350000CA809F0E1FA20220DF207210CA809F0EF
:10136000DBFA04A90CA809F06EFB20220DF207316C
:1013700004A807F08BFE003018BF0120444201E0B2
:101380006FF0050427A809F04BFA20460DF54B7DB8
:10139000BDE8F08F6FF00404F4E76FF00304F1E7A9
:1013A0006FF00204EEE76FF00104EBE730BD0000E0
:1013B000E8C000002DE9F043079C1CB914602046EA
:1013C000BDE8F0830325B4FBF5F505EB4507BC420A
:1013D00018BF0135B5F1804F05D34FF0FF331360CF
:1013E0006FF00B00ECE7AD0001358D4200D808B975
:1013F0001560F5E7DFF8BCE006460025BD42314642
:101400009C4606F1040603F103032CD3A54225D222
:101410009CF80060274F0135A54238BF9CF8013089
:101420004FEAA60C28BF002317F80CC081F800C0B3
:10143000A54207EB131C3CBF9B0003F03C034FEAA3
:10144000061606F0300638BFFB5C1CF806604E70CE
:1014500028BF3D238B703D23CB700431081A1060E8
:1014600000200870ACE713F803CC13F8021C13F843
:10147000018C4FEAAC094FEA0C1C1EF8099006F8E3
:10148000049C0CF0300C0EEB1119890019F80CC0FB
:1014900006F803CC01F03C010EEB981C08F03F0865
:1014A0001CF8011006F8021C1EF8081006F8011CB2
:1014B0000335A3E77EC200002DE9F043DDF81CE010
:1014C000DFF8148100273C46BC46F445654629D226
:1014D0005E5D202E23D0AEEB0509B9F1010F25D0BA
:1014E0000D2E23D103EB050999F80190B9F10A0FEC
:1014F00012D065456CD13D2E02D10137022F67D83D
:1015000016F0800F64D118F806607F2E60D03F2E51
:1015100001D8002F5CD1013405F1010CD5E701356C
:10152000AE45D5D124B91460002021E00A2EDFE7B2
:1015300004F0070C0626E40806FB0CFC74430CF1CF
:10154000070CE41B04EBDC0478B18C420DD80027B7
:10155000DFF884E0DFF884801D44014603263C4622
:101560009D4207D1091A1160DEE714606FF00B008D
:10157000BDE8F08313F8019BA9F10A0C5FFA8CFC1B
:10158000BCF1160F04D828FA0CFC1CF0010FE7D1AF
:101590001EF809C00134BCF1400F08BF013E0CF039
:1015A0003F0C042C4CEA8717DAD17EB13C0C012E9B
:1015B0000C7002D101310024D2E7022E4FEA172429
:1015C0004C7016BF8F7002310331F4E73446C7E721
:1015D0006FF01500CCE700BFFEC10000090040001D
:1015E0000B6801330B60014B1B681847B88700205C
:1015F0002DE9F04F85B09B460E9CDFF890A0012CA2
:10160000B8BF0124012B0CBF302320231546804690
:1016100089460194029301260A2700220AF1010457
:101620000AB9AA451FD2B5FBF4F049463030C0478D
:1016300001360122013F012FB5FBF4F14FF00A03FF
:1016400004FB1155BAFBF3FAE8D1494605F1300025
:10165000C047BBF1030F03D1019B9C1B002C0FDC87
:1016600005B0BDE8F08F019BBB42E3DBBBF1020F8D
:10167000E0D84946029803920136C047039AD9E759
:1016800049462020C047013CE8E700BFFFC99A3B1C
:1016900013B502AC002344F8043D02460B46034850
:1016A000214606F0D7FE02B010BD00BFE1150000D4
:1016B0004FF02003EFF3118283F31188BFF36F8F94
:1016C00006490123C1F840354FF08041C1F8783513
:1016D00082F31188BFF36F8F0020704700E0014054
:1016E000074BC0B21860BFF34F8F0649064BCA685C
:1016F00002F4E0621343CB60BFF34F8F00BFFDE7FE
:101700001C05004000ED00E00400FA0520B1034B89
:10171000800143F001031847704700BF10BD00006F
:10172000054B1B68082B01BF044B1868B0FA80F00A
:10173000400918BF0020704730010010340100102C
:1017400008B54FF080430022C3F80C21C3F81021E4
:10175000C3F838254FF0805203F54043D2F8041403
:10176000C3F82015D2F80814C3F82415D2F80C14C5
:10177000C3F82815D2F81014C3F82C15D2F8141495
:10178000C3F83015D2F81814C3F83415D2F81C1465
:10179000C3F84015D2F82014C3F84415D2F8241425
:1017A000C3F84815D2F82814C3F84C15D2F82C14F5
:1017B000C3F85015D2F83014C3F85415D2F83414C5
:1017C000C3F86015D2F83814C3F86415D2F83C1485
:1017D000C3F86815D2F84014C3F86C15D2F8442445
:1017E000C3F87025FFF79CFF10B1164B164A1A601C
:1017F000FFF796FF18B1154BFB22C3F81825FFF72A
:101800008FFF48B11249134B0A681B6822F00F0280
:1018100003F00F0313430B60FFF782FF18B10E4B69
:101820004FF400721A604FF08043D3F80024D207BF
:1018300044BF6FF00102C3F80024084B084A1A6045
:1018400008BD00BF8C5600404881030000F00040F6
:10185000E40E00405802001040960240BC87002071
:101860000090D003044AD2F80034DB07FBD50160B6
:10187000BFF35F8F704700BF00E001404FF080531F
:101880001A69B0FBF2F302FB130373B9084B02228F
:10189000C3F80425C3F80805D3F80024D207FBD504
:1018A0000022C3F80425034870470348704700BF6F
:1018B00000E001400000AD0B0A00AD0B10B5054C77
:1018C0000123C4F80435FFF7CDFF0023C4F8043525
:1018D00010BD00BF00E001402DE9F8431E4B154646
:1018E0000122C3F8042510F0030304460E4610D06D
:1018F000C3F10407AF4228BF2F463A46A0EB0308C6
:1019000006F0C2FF01464046FFF7ACFFED1B3C442A
:101910003E4425F00308B0443746A4EB0609B84519
:1019200013D115F003020AD025F003010C44204620
:10193000314406F0A9FF01462046FFF793FF064B0E
:101940000022C3F80425BDE8F88309EB070057F827
:10195000041BFFF787FFE2E700E00140044A9168BB
:101960009368CB1A23F07F438342F9D3704700BFBB
:1019700010E000E0034B044A1B68B3FBF2F358434A
:10198000FFF7ECBFBC87002040420F00064A10F072
:10199000800F00F00F0314BFD2F81005D2F8140521
:1019A000D84000F00100704700700240054B1B68F2
:1019B000082B05D1044B1868003018BF0120704770
:1019C000002070473001001034010010054B10F06A
:1019D000800FA3F1900208BF134600F00F0003EB45
:1019E00000107047E80D0020024A00231360024AED
:1019F000137070471C7C0240D745002007B5084A89
:101A000000231370074A019302A81370012300F802
:101A1000043D054B1B68984703B05DF804FB00BF0D
:101A2000D6450020D9450020780E0020F8B54D6835
:101A30000B4F954228BF15460C4606462A460968B4
:101A4000384607F033FB60682368401BC6E9007521
:101A500060601D440030256018BF0120F8BD00BF44
:101A6000800E0020F8B54C68944228BF1446064604
:101A70000D468CB1094F09682246384607F016FB1F
:101A800037606B6874601B1B6B602B68201C2344E1
:101A90002B6018BF0120F8BD0460F2E7800E002023
:101AA00007B500238DF804300B4BD3F82025ADF893
:101AB0000620D3F8C034094A002B13680CBF4FF43A
:101AC00080714FF001210B431360054B01A81B6887
:101AD000984703B05DF804FB00700240540D0020ED
:101AE000780E0020074BBFF35B8F024653E8000FD0
:101AF00000EA020143E8001CBCF1000FF6D1BFF37D
:101B00005B8F7047E40C002013B5FFF76DFF0D4BA2
:101B100093F88E20032A12D0D3F880407CB96FF05E
:101B20008070FFF7DFFF06238DF8043008238DF85F
:101B30000630054B8DF807401B6801A8984702B096
:101B400010BD00BF580D0020780E002008B5FFF72B
:101B50004BFF084B93F89E20032A05D16FF001003C
:101B6000BDE80840FFF7BEBFD3F89030002BF5D09A
:101B700008BD00BF580D0020012273B502FA01F51F
:101B80001E491F4E0B6810F0800F43EA0503044600
:101B90000B6027D000F00F021A4B33F8123003F11C
:101BA000804303F51C331A684AB100221A60BFF360
:101BB0006F8FBFF34F8F802811D006F0D8FE3168A9
:101BC00029400AD106238DF804308DF806408DF89F
:101BD00007100D4B01A81B68984702B070BDFFF7B6
:101BE000B5FFECE733681D42F7D106238DF80430CA
:101BF0008DF806008DF80720EBE700BF540D00209C
:101C0000E40C002088C00000780E002008B5054BC9
:101C10001A78104606F0A1FEBDE8084001461046BD
:101C2000FFF7AABFD945002013B5FFF7DDFE104B23
:101C300093F81E21032A05D16FF48070FFF752FF3D
:101C400002B010BDD3F81041002CF9D16FF48070B0
:101C5000FFF748FF06238DF8043088238DF80630FF
:101C6000044B8DF807401B6801A89847E8E700BFC0
:101C7000580D0020780E0020204B13B5D3F80044F7
:101C8000C3F80044BFF36F8FBFF34F8FBFF36F8F65
:101C9000BFF34F8FE1050BD5194B01221A7002A833
:101CA00000230193022300F8043D164B1B6898475C
:101CB000A2050AD5124A002302A801931370032338
:101CC00000F8043D0F4B1B689847630513D50C4B78
:101CD0001A7882B100221A70084B0121C3F8081546
:101CE000582006F0F2FD02A80423019200F8043DFA
:101CF000044B1B68984702B010BD00BF0070024043
:101D0000D6450020780E00202DE9F04F724B87B0A9
:101D10001A780193002A40F08280DFF8C4B16F4B3B
:101D200018686F4B1C68204079D010F0012479D0DE
:101D300094FAA4F4B4FA84F40F2C86BFA4F110082A
:101D40005FFA88F844F080084046FFF73FFE4FFAFC
:101D500088FABAF1000F064608F00F05828966DAA4
:101D6000D0E9003104A8984700B930605D4B822269
:101D70001A60019B059A01201870A040B368DBF837
:101D80000040134424EA0000BAF1000FCBF8000031
:101D9000B3600498544B77DA072D9BBF142101FBE5
:101DA0000533C3F8A006C3F800068CBFC3F8A42609
:101DB000C3F80426FFF7FAFDAB002DB26E004B4AC4
:101DC0004B49002871D1BAF1000FB5BF92468A463F
:101DD00004242824B244474F474E1C44054635602E
:101DE000BFF36F8FBFF34F8F204606F06EFD0220CA
:101DF000FFF7C0FD3368002BF1D01E20FFF7BAFDBE
:101E00003B689B064FD50120FFF7B4FDBAF80030C0
:101E100003F1804303F51C331B68002BDFD007B0B0
:101E2000BDE8F08F90FAA0F0B0FA80F484E7072DB7
:101E30002D4B24D9D3F8C09419F4803F18BF4FF02C
:101E400000094B467168376804A8B847049B002B0B
:101E50008AD0059B4B4587D201200225A040B5734F
:101E6000C043FFF73FFE06238DF80C30234B8DF85F
:101E70000E808DF80F501B6803A898474FE705F5B3
:101E8000947153F82190DCE7072D9BBF142101FBCF
:101E90000533C3F8A007C3F800078CBFC3F8A42715
:101EA000C3F8042786E70220A8E7BAF1000FACBF09
:101EB00028200420184406F008FD12EA2A0A38BF38
:101EC0008A463AF8153003F1804303F51C331A684B
:101ED000002AFCD0A3E700BFD7450020E40C002077
:101EE000540D00201C7C02400070024088C000009D
:101EF0009AC000007474024004710240780E002001
:101F000038B5174BD3F86C44C3F86C44BFF36F8FEC
:101F1000BFF34F8FFFF74AFD38B9124A136823F019
:101F2000011103F001130C43136001251CB9BDE836
:101F30003840FFF7E9BE94FAA4F3B3FA83F30F2B0A
:101F4000D9B2C8BFA1F1100005FA03F3CCBFC0B2EB
:101F500041F0800024EA0304FFF70EFEE6E700BF2D
:101F6000007002407C0E002037B50446FFF73CFDB0
:101F7000FFF72CFD837B032B0CD1204606F0EDFCF4
:101F8000012303FA00F0C043FFF7ACFDFFF7BCFEEE
:101F900003B030BD0568002DF8D1204606F0DDFC09
:101FA000012303FA00F0C043FFF79CFD06238DF8E0
:101FB0000430044B8DF806408DF807501B6801A8CB
:101FC0009847E3E7780E0020024A00231360024A94
:101FD00013707047780E0020D845002038B5514B5B
:101FE0004FF40062C3F80024BFF36F8FBFF34F8F2D
:101FF000FFF7DCFC4C49A8B14FF02003EFF311844C
:1020000083F31188BFF36F8F0868484B03220028C1
:102010007ED149F2753008601A60086084F3118837
:10202000BFF36F8F4FF02003EFF3118483F3118818
:10203000BFF36F8F08683E4AC02300286AD149F277
:10204000753008601360086084F31188BFF36F8FE8
:10205000344B0120C3F80005BFF36F8FBFF34F8FE0
:10206000D3F800040005FBD54FF40060C3F800046A
:10207000BFF36F8FBFF34F8F4FF02003EFF3118447
:1020800083F31188BFF36F8F0868002844D149F2A9
:1020900075330B6010600B6084F31188BFF36F8F92
:1020A000244B40F2E3721A60043340221A60BFF3FB
:1020B0006F8FBFF34F8FA3F6040300248022C3F871
:1020C0001C25C3F830451C4B40F2FF121A601B4B15
:1020D0001C60FFF789FC1A4B1C701A4B02221A7005
:1020E000FFF764FC98B14FF02003EFF3118583F301
:1020F0001188BFF36F8F08680C4B80B949F27532B5
:102100000A6018600A6085F31188BFF36F8F38BDCD
:102110001A6083E7136097E700231360BCE71C6035
:10212000F1E700BF0070024000EC064014ED0640ED
:1021300014EC064000780240540D0020E40C00200E
:10214000D9450020D84500200E4B002210B51A704A
:10215000A8B9FFF72BFC0C4B0C4A00280CBF184603
:1021600010460B4CC4F80403272003F0A3F9012305
:10217000C4F80435BFF36F8FBFF34F8F10BD024813
:10218000EFE700BFD64500200714E0010714C001A7
:1021900000700240034B1878012894BF00200120F2
:1021A000704700BFD84500201B4B70B51C7884BB1E
:1021B0001A4A106001221A70264664F07F05082C26
:1021C000EDB20CBF4FF400714021284606F013FC1D
:1021D0002846FFF7FBFB0134092C867306608660F6
:1021E000EBD1002440212546204606F004FC204681
:1021F000FFF7ECFB0134E4B2092C857305608560C0
:1022000001D1074870BD082C0CBF4FF4007140216C
:10221000EAE70448F6E700BFD8450020780E002022
:102220000000AD0B0500AD0B2DE9F843074606F0A5
:1022300094FB4FF02003EFF3118583F31188BFF374
:102240006F8F17F00F0903D1274B1B78BB4246D184
:10225000264A274B12681C68D243012692B2864058
:102260002243324298463CD13846FFF7AFFB0C235D
:102270003A06844603FB09F32DD51E4A0868134429
:1022800000F060408A68B0F1005F02F001021DD1E9
:10229000D2B9194ACCF8002007C983E80700CCF866
:1022A00004300023CCF808308CF80E30134B14485F
:1022B00034438022C8F80040C3F8042185F3118814
:1022C000BFF36F8FBDE8F8830E4AE3E70AB90E4A01
:1022D000E0E70E4ADEE70E4A13440E4ADAE70E48FC
:1022E000ECE70E48EAE700BFD9450020540D002076
:1022F000E40C0020E80C00200F89000000E100E061
:102300000000AD0B318900002D1A0000651A000095
:10231000780C0020E18800000A00AD0B0B00AD0B2B
:10232000044B40F48070C3F81805BFF36F8FBFF300
:102330004F8F70470070024000F00F03072B11D839
:1023400010F0800F084A0BBF03F5887303F5847300
:1023500002EB830352F8230008BF5868431E58421B
:1023600058417047002070470070024010B50822A5
:102370000021044606F0C7FE0E4BD3F880242270DD
:10238000D3F884246270D3F88824D3F88C1442EAFA
:1023900001226280D3F89024D3F8941442EA0122F7
:1023A000A280D3F89824D3F89C3442EA0323E38034
:1023B00010BD00BF0070024013B5FFF715FB0F4BB7
:1023C0009A7B032A05D16FF48030FFF78BFB02B0B4
:1023D00010BD1C687CB96FF48030FFF783FB0623C7
:1023E0008DF80430064B8DF806408DF807401B68C9
:1023F00001A89847EBE706F01AFBE8E7580D002024
:10240000780E0020014B1878704700BFD945002096
:1024100038B50246FFF7CAFA0446104606F09DFAA0
:1024200001238340DB4302F00F001B4ABCB94FF08D
:102430002001EFF3118581F31188BFF36F8F1168CD
:102440000B4013604000154B00F2C57018605C60D3
:1024500004331B6885F31188BFF36F8F38BD4FF0CD
:102460002001EFF3118481F31188BFF36F8F11689E
:10247000072803EA0103136009D800F59470084B9C
:10248000002243F82020BFF36F8FBFF34F8F84F3F8
:102490001188BFF36F8FE1E7540D002000780240F0
:1024A00000700240F7B501464FF02003EFF31184AE
:1024B00083F31188BFF36F8FFFF788FA054608464C
:1024C00006F04BFA012311F0800F03FA00F02A4EB8
:1024D00017D1336830EA03020AD00846FFF798FFA5
:1024E0000323AB7384F31188BFF36F8F03B0F0BD88
:1024F0002A60C043214A03403360136803401360DD
:10250000EEE701F00F02072A0FD880291C4F1D4B60
:1025100028D002F2DA3252003A601A681F68D2B24A
:1025200042F002023A431A601B68144F32683B685B
:1025300062EA030C1CEA000FD4D022EA000218431E
:10254000002332602B600323AB738DF807300E4BF2
:10255000386006228DF804208DF806101B6801A84B
:102560009847BFE740F2B4723A601A681F68D2B267
:1025700042F00402D6E700BFE40C0020540D002016
:102580000078024004780240780E0020F7B5164B20
:10259000164CD3F880542368154EDA43154B377820
:1025A0001B6892B238461A4306F0D7F9012303FAA2
:1025B00000F0104202D03846FFF774FF05F08005A6
:1025C0006FF001103570FFF78DFA236843F00103B7
:1025D000236002A800230193052300F8043D064B65
:1025E0001B68984703B0F0BD00700240540D0020F6
:1025F000D9450020E40C0020780E0020554B2DE931
:10260000F041D3F80453002229461646012400293C
:102610007CD1FFF7CBF9002869D14F4B1B78002BF9
:1026200065D1960263D54D494C4E40F2A9730B60BB
:102630004B4B1C6814F0FF041CBF1868044040F2A8
:10264000AA700860186810F0FF001CBF19680840E5
:1026500040F2AB713160196811F0FF01B4461CBF44
:102660001E68314040F2AC76CCF800601E68344001
:102670003C4E08D037682743376040F2A977CCF842
:1026800000701C601C68354F40F2AD743C601C68E3
:10269000204008D0346844EA0044346040F2AA7410
:1026A0003C60186018682D4840F2AE7404601868E9
:1026B00001400DD0CC0748BF42F40002C8062748AD
:1026C00040F2AB74046019601B6848BF42F001021D
:1026D000336833F001111CBF05F08070024313F022
:1026E000011F04D06B0544BF316042F480621E4F6D
:1026F00002F4000622F400044FF00108E4B9FFF7E9
:1027000003FB2EB3BDE8F041FFF740BF91FAA1F300
:102710001648B3FA83F39F00384407683FB1066058
:10272000BFF36F8FBFF34F8F04FA03F0024304FA35
:1027300003F321EA03016AE794FAA4F5B5FA85F5F3
:1027400057F8253008FA05F5984724EA0504D5E737
:10275000BDE8F08100700240D745002000780240BB
:10276000047802407C0E002070BD00000071024021
:10277000F8B5114E114A34681268240C240414432D
:1027800001271CB940F2FF133360F8BD94FAA4F599
:10279000B5FA85F5E8B20F2DC6BF1038C0B240F0CB
:1027A000800000F00F03072B01D8FFF77BFE07FA2C
:1027B00005F524EA0504E4E7540D0020E40C0020AC
:1027C0000D4B802210B52720C3F8842102F096FE1D
:1027D00080B10A4CFFF7CCFF0023C4F80435BFF3E7
:1027E0006F8FBFF34F8F272002F074FE4FF0FF333F
:1027F000C4F8083310BD00BF00E100E000700240E3
:1028000008B5FFF7DDFF094BD3F80423C3F808230D
:102810000022C3F80025BFF36F8FBFF34F8FFFF780
:10282000E3F8034B01221A7008BD00BF007002409C
:10283000D845002038B54FF02003EFF3118583F31E
:102840001188BFF36F8F0F4B1B7803F0FF0433B970
:10285000002485F31188BFF36F8F204638BDFFF742
:1028600087FF094AD2F8003413F40073F0D1012134
:10287000C2F82C15D2F80014890544BFC2F82C35D3
:102880001C46E6E7D64500200070024010B504461D
:10289000FFF708FE134A04F00F0064B2002C4FF05B
:1028A0000103B4BFD2F81015D2F8141503FA00F3DF
:1028B0006FEA0303B5BF0B400B40C2F81035C2F8F6
:1028C0001435BFF36F8FBFF34F8F074B074A33EABF
:1028D000240428BF14460123225C9340014AC2F815
:1028E000083310BD00700240D6C20000CDC2000007
:1028F000F8B5234A234B244D47B233EA270328BFB8
:10290000134600F00F0401211B5D01FA03F3C5F823
:1029100004330646FFF73AF888BB002FB4BFD5F85A
:102920001035D5F8143501FA04F1B5BF1943194330
:10293000C5F81015C5F81415BFF36F8FBFF34F8F8F
:10294000013C062C1BD8002F19DB4FF02003EFF3BE
:10295000118483F31188BFF36F8F3046FFF758FD62
:10296000304605F0FAFF094A012303FA00F0136824
:1029700023EA0003136084F31188BFF36F8FF8BD5F
:10298000CDC20000D6C2000000700240E40C00205E
:10299000030610B504460AD400F00F03072B06D82F
:1029A0009B00074AD358012B01D1FFF731FD054B9E
:1029B000C3F81845BFF36F8FBFF34F8F10BD00BF33
:1029C00044740240007002402DE9F041114B124D59
:1029D000124C5B1B9B106343114C4FF0240ED4F838
:1029E0001CC000249C4203D16FF02200BDE8F0819E
:1029F0000EFB0456776867450AD3366946B197F8E7
:102A000002808788B84503D13346BDE8F0411847B6
:102A10000134E7E7108B0020EC8A0020398EE33880
:102A2000C00E00202DE9F041114B124D124C5B1BE2
:102A30009B106343114C4FF0240ED4F81CC00024AB
:102A40009C4203D16FF02200BDE8F0810EFB0456DA
:102A5000776867450AD3B66946B197F802808788D8
:102A6000B84503D13346BDE8F04118470134E7E7E4
:102A7000108B0020EC8A0020398EE338C00E002035
:102A80002DE9F84F9046104B104A0F469B1A1049FB
:102A90009B10064601FB03FA002491464FF0240BDD
:102AA000A24502D16FF022000BE00BFB04935D699D
:102AB0000DB90134F4E7424639463046A8470028AC
:102AC000F7D1BDE8F88F00BF108B0020EC8A002002
:102AD000398EE33807B583788DF800300379427971
:102AE00043EA0223ADF80230C378032B0FD86846BF
:102AF0008DF8043001F044FC9DF8000001F0B8FCB2
:102B0000044B012083F8710003B05DF804FB002042
:102B1000FAE700BFC00E002037B5104C02ABE268E8
:102B200043F8042D0546A168802001F0DDFC019AE0
:102B3000A3681344A360E3689B1AE3605BB9402A6F
:102B400009D1402D07D900231A461946802001F0EB
:102B5000CBFC0B30F7D003B030BD00BFC00E00205F
:102B600008B509480378C3F34113083350F82330FC
:102B70003BB100F1080200F110019847C043C00FBB
:102B800008BD1846FCE700BFC00E002037B5002284
:102B90000B4601920546002849D1294C01BB082269
:102BA000214606F0E0F9002803DA802001F008FC55
:102BB00020E0E588256104F13003C4E9023515B150
:102BC0002378DB0916D0FFF7CBFF0028EDD023696F
:102BD000AB42D4BFE360E5602846FFF79DFF09E004
:102BE000D4E90212002A01AB06DC024606F0BBF96A
:102BF0000028DADB03B030BD06F0B5F9002804DAAE
:102C0000802001F0DDFB2846D0E70199A268E36847
:102C10000A445B1AA260E360002BEBD104F130039D
:102C2000A360FFF79DFF0028BFD0E088D5E780288C
:102C3000E0D1034BDA68002ADCD0D888CDE700BFAA
:102C4000C00E0020014600F10803BFF35B8F53E87C
:102C5000002F42F0010043E8000CBCF1000FF6D158
:102C6000BFF35B8FD30702D4014808F0A3BD7047C0
:102C7000542800202DE9F74F8E4D6B6906460C460F
:102C8000904663B9377807F01F07012F00F09C804A
:102C90000BD3022F00F0D5806FF0150002E09847AB
:102CA0000028EFD103B0BDE8F08F72787088D8F8B3
:102CB0000030092AF0D801A151F822F0E52C0000DB
:102CC000AF2D0000992C0000BD2D0000992C0000B4
:102CD000FF2C0000092D0000992C0000372D00006A
:102CE000412D000000201870587095F87320824222
:102CF00014BF022202461A7002232360D2E7C0B238
:102D000001F02EFB0020CDE7020A131F012BC3D9CF
:102D1000072AC1D8EB690021C0B21D78002DBBD0B5
:102D20005E78964203D1884200F0BB8001312B448B
:102D3000F3E71B78BBE095F872201A700123B6E028
:102D4000C4B28DF8074014B985F87240DAE74FF045
:102D5000FF08EE690027C146337843B9AB691BB160
:102D60000DF1070103209847002F95D0ECE7737809
:102D7000042B0DD0052B0ED0022B06D196F8058022
:102D80009DF80730434508BF012733781E44E3E729
:102D900096F80390F9E79DF807304345F5D1B9F16E
:102DA000000FF2D13046FFF795FE0746EDE7012808
:102DB0007FF472AF002085F8730073E701287FF479
:102DC0006BAF85F873009DE77078D8F800300A285B
:102DD00007D00B2809D000287FF45EAF1870587018
:102DE0008AE70020187027605CE796F804A096F840
:102DF00002B0EE69FF27B9464FF0000833783BB9BF
:102E0000AB6913B14146072098470020206049E78D
:102E10007378042B04D0052B0BD033781E44EDE7D8
:102E2000B77896F80390BA45F7D1CB4508BFB046BE
:102E3000F3E7BA45F1D1CB45EFD13046FFF74AFE73
:102E4000EBE773783079D8F800808DF80700012B14
:102E500018D010D3032B7FF41FAF7488002C7FF49D
:102E60001BAF01F0ADFAAB69002B3FF44BAF0DF196
:102E70000701082013E0414601F0E0FA002088F83D
:102E80000100B0E77488002C7FF406AF01F0BEFAB1
:102E9000AB69002B3FF436AF0DF1070109209847CD
:102EA00030E7022AC8F800307FF443AF5B88236024
:102EB00028E700BFC00E002010B5064C94F8700043
:102EC00030B101F0F7F90028A4BF002084F87000A9
:102ED00010BD00BFC00E00200A4930B500233C24BD
:102EE00004FB031292F87450854206D1906F10F1E2
:102EF000100F14BF0020012030BD0133042BEFD18F
:102F00000020F9E7C00E002073B5194C0D460646A7
:102F100000233C2101FB03F2A01890F87400B0429A
:102F200013D1743214446B1E012B0CD894B9012DAB
:102F300009D101AB01220DF10301304601F03CFB48
:102F4000019B002BF5D102B070BD0133042BE1D100
:102F50000024E8E704F01EFD2C3408B1012D03D154
:102F6000204605F091FDEEE72046FFF76BFEEAE70D
:102F7000C00E00202DE9F04F85B005460191904626
:102F800099464FF02003EFF3118B83F31188BFF3C1
:102F90006F8F2E4F00263C2307F1900203FB06F4AF
:102FA00002EB040A002150460393029204F0B6FC9F
:102FB000DDE9022350B93E19B36F13F1100F12D19E
:102FC0005046019304F084FC019B04E00136042E7A
:102FD000E4D16FF00B038BF31188BFF36F8F1846AA
:102FE00005B0BDE8F08F019BC6F88400C6E91F3824
:102FF0000E9BC6F888300F9BC6F88C306FF00F031D
:1030000086F87450C6F8AC90B367284601F06AFBA6
:1030100068B1284601F066FBB8FBF0F303FB1080B3
:1030200028B1D6F8AC3043F00403C6F8AC3019F040
:10303000020F06D004F1A0003844FFF703FE00237E
:10304000C9E7284601F0FCFA0346C4E7C00E002099
:103050002DE9F0410F4D00246FF0470705F1A0085E
:103060004FF02003EFF3118683F31188BFF36F8FC6
:103070002B199A6F103204D19F6708EB0400FFF7F9
:10308000E1FD86F31188BFF36F8F3C34F02CE7D15C
:10309000BDE8F081C00E00202DE9F74F1F4C204EF7
:1030A000204A361BB31002FB03FA031F012B804694
:1030B000894624D81C4D95F8713003B3FFF7C8FF3B
:1030C00027464FF0000BDA4516D0396A0022387FC8
:1030D000D3B2984203D80BF1010B2437F3E701EB8D
:1030E000C30301921879009101F0E0F9019A009967
:1030F000002802F10102EADA002385F87130002588
:10310000AE4202D103B0BDE8F08F2819C36813B1F5
:103110004A46414698472435F2E700BFEC8A002032
:10312000108B0020398EE338C00E0020054B064A74
:103130001A62064A5A62064A9A62064AD8615A6177
:1031400000207047C00E0020752C0000C929000027
:10315000812A0000252A00002DE9F743384E96F811
:103160007040002C4ED13748B06101F0B5FA01F043
:1031700061F8002847DB02AD402305F8084D2846DA
:10318000ADF802308DF8044001F0FAF800283ADB7F
:10319000802728468DF8007001F0F2F8002832DB15
:1031A0002949204601F086FA00282CDB26493846BA
:1031B00001F080FA002826DB244D254B254F5B1BB0
:1031C0009B105F43A74221D1234CDFF8908004F18C
:1031D000F00700250122A561C4E9045820461146E4
:1031E0003C3408F0CDFBA742F4D1002001F040F9B7
:1031F000002808DB802001F03BF9002803DB0123D5
:1032000086F87030002003B0BDE8F083D5F8209038
:103210004FF000082A7F5FFA88F39A4202D80134FF
:103220002435CFE709EBC30259F83310107901F0C8
:1032300041FA08F101080028ECD04FF0FF30E2E736
:10324000C00E0020993000008D2B0000EC8A002079
:10325000108B0020398EE338500F0020898A00003F
:10326000084B10B593F8704034B900F0F1F828B16C
:10327000FFF75CFFFFF770FF002010BD4FF0FF303D
:10328000FBE700BFC00E00202DE9F04F6B4A6C4BEE
:103290006C499B1A87B09B1000264B430446009351
:1032A0004FF001193746B246B046934623783BB9F2
:1032B000654AA01C904200F0BF80FFF7E5FF24E0C4
:1032C0006378052B0AD8DFE803F07B09B57B037828
:1032D000E3781BB9A378DBB10137FFB223781C4434
:1032E000E4E702FB03BADAF804108C4207D1DAF8FB
:1032F0000830002BF0D0394620469847ECE70133E0
:1033000000999942EDD14FF0FF3007B0BDE8F08F42
:103310002422F5E701FA05FC1CEA090F2DD001353E
:10332000102D0DD101339AF81C209342EBDADAF814
:103330002020A57802EBC30210798542F2D1012545
:1033400094F803C08DF814C094F805E094F804C014
:103350004CEA0E2CADF812C094F802C08DF810C0E3
:103360001CF0800FE8B2D5D005F1100C01FA0CFC6E
:103370001CEA090FD3D160F07F008DF8100004A87B
:10338000CDE90221019305F0D5FDDDE90132039974
:103390000028C4D19DF81030A37013F0800F137172
:1033A00018BF10354FF0010315BFAB4003FA05F508
:1033B00049EA030949EA050990E700230121B2E738
:1033C000032E1DD105F0E4FB019060B105F049FE2C
:1033D00005461E4805F045FE8542019903D12A465F
:1033E000A01C05F063FE2146002011F8023BDA1E06
:1033F0005B08013B0B44002A13DA0136F6B26DE795
:10340000002EF0D1B8F1000F3FF47DAFA4EB08031C
:1034100088F80230C3F3072388F8033088F8047073
:10342000EBE78854013B8D1893F800C005F801CCF8
:10343000023AE0E7A04651E7184666E7EC8A00202A
:10344000108B0020398EE338EB8A0020DFC20000A9
:1034500008B50448FFF718FF0028024818BF0020ED
:1034600008BD00BF4C8A002070B504460E460179A5
:103470001048154605F09AFBB0B16378212B0ED0A9
:10348000222B08D0202B12D1072229680C3805F0F6
:103490000DFE002070BD638800F8053CF9E70C388C
:1034A000072328603360F4E76FF01200F2E76FF053
:1034B0001500EFE72410002008B50146034805F089
:1034C00083FB10B1012300F8033C08BD2410002049
:1034D00010B50446104804F0FBF9104B1868C4F806
:1034E000B000002198889B79A4F8B40084F82510D6
:1034F00084F8241084F8261084F8271084F8B63055
:1035000084F8B81084F8B71004F128004022BDE810
:10351000104005F0F8BD00BF2C10002000BD0000D9
:10352000D0F8A4301B68F7B59B681B6A1D7D044664
:103530002846FFF7D1FC90B904F1500640223146ED
:10354000D4F8940005F07DF9A4F11807054B009319
:1035500002460197022331462846FFF70BFD03B0D0
:10356000F0BD00BF0537000030B5036885689A6874
:10357000104C85B042F2A1004FF40033CDE90103B5
:10358000002385F8B930106AADF80C100A2201A9A1
:10359000007905F067FA95F8B93013B1002005B04D
:1035A00030BD012008F0FAF9013CF4D16FF00400BD
:1035B000F5E700BFA186010010B584680023C4F8B8
:1035C000C0300E4BC4F8BC00596804F1C00289B980
:1035D000C3E900224FF0FF320021094808F0D0F97A
:1035E000084B0020C4E90430074BE060A061C4E947
:1035F000073010BD0A605A60ECE700BF24100020BD
:103600002C1000200B8C000021350000014600F139
:103610000803BFF35B8F53E8002F42F0010043E83B
:10362000000CBCF1000FF6D1BFF35B8FD30702D4BF
:10363000014808F0BFB870475428002073B51446FD
:1036400002F128050A1E064604DD2946D4F8A80022
:1036500005F0A4F8012384F82530636833B194F8A9
:1036600027301BB104F10C00FFF7D0FF054B00938E
:1036700001940123402229463046FFF77BFC02B02B
:1036800070BD00BF3D36000038B50D4601461348F9
:1036900005F080FA0446F8B10A2D1DD023681B6896
:1036A000032D9B6804F8BC5CA0F1BC0007D0042D7E
:1036B00001D0012D10D1BDE83840FFF709BF1B6ACA
:1036C00002460021187BFFF7B9FF012304F8983C5C
:1036D00004F8963C04F8953C38BD00BF2410002047
:1036E00007B502AB012203F8011D194605F061FB85
:1036F0006421034804F012F903B05DF804FB00BF35
:103700002C10002010B50123144682F824300C48F8
:1037100004F0DEF8636833B194F826301BB104F18D
:103720000C00FFF773FFD4F8AC30D3E900329A42B3
:1037300005D004F11800BDE81040FFF767BF10BDC9
:103740002C100020084B30B51C68084B196800226B
:10375000944202DC0023184630BD0B4610311D7820
:103760008542F8D00132F3E7A8BE0000D4880020DB
:10377000084B1B6810B50C462BB1FFF7E3FF28B1CF
:103780002060002010BD6FF00C00FBE76FF001001F
:10379000F8E700BFD488002030B589B00C46154644
:1037A0000190FFF7CFFFB0B14368029383682268AE
:1037B000C068CDE903350023CDE90623059303F066
:1037C000FBFA01AA054907F0B2FA079808B9059B68
:1037D000236009B030BD6FF01500FAE7E18D0000FD
:1037E00008B504464FF02002EFF3118382F31188ED
:1037F000BFF36F8F05F0C7FB2046FDF771FF03484D
:1038000004F084FF01F0D0FEFCE700BFEEC2000030
:1038100010B54FF02003EFF3118283F31188BFF34B
:103820006F8F154C237833B982F31188BFF36F8FF4
:103830006FF0440010BD013BDBB2237033B182F363
:103840001188BFF36F8F6FF00F00F3E70B4B187801
:10385000012138B1217082F31188BFF36F8F6FF0AF
:103860000A00E7E7197082F31188BFF36F8F044AEB
:1038700011601870DEE700BFDC4D0020DB4D00203A
:1038800004000040F8B54FF02002EFF3118382F3FB
:103890001188BFF36F8F294A1078441C147080B1CF
:1038A00083F31188BFF36F8F4FF08043D3F80C344C
:1038B00003F00113B3F1011F0CBF00206FF04300B0
:1038C00009E01F4D2F783FB1107083F31188BFF3CB
:1038D0006F8F6FF00A00F8BD01262E7083F31188F8
:1038E000BFF36F8F4FF0804419B3384601F0F2FDFB
:1038F000C4F80071D4F80433C4F804632660D4F823
:10390000002192B10022C4F800210E4A13F0010FE9
:103910004FF0010308BFC4F808330020C2F880311B
:1039200001F0C8FD00232B70BEE720BF40BF20BFC1
:10393000E5E7C4F800112660F4E700BFDC4D002085
:10394000DB4D002000E100E070B54FF02002EFF306
:10395000118382F31188BFF36F8F244D2A789AB1B7
:1039600083F31188BFF36F8F4FF08042D2F81C347D
:10397000D2F8182403F0030343F48033934314BFB5
:103980006FF04300002070BD01242C7083F3118878
:10399000BFF36F8F4FF08043154EC3F8042102250B
:1039A000C3F81815C3F8045311F0030134604FF045
:1039B0001806C3F80863C3F80C21C3F81021D3D14B
:1039C0001022C3F83825C3F80463D3F81824D203AF
:1039D00002D4C3F80453C7E7C3F80443FFF752FF08
:1039E0000028C1D1034BC3F80041BDE7DA4D0020E8
:1039F0000800004000E100E02DE9F0434FF0804373
:103A00004E4DD3F80891D3F80423D3F800E1804653
:103A1000D3F80403D3F804C1D3F80C11D3F8104140
:103A20002F68AE680435003485B002F0010218BF7B
:103A300001242D68B9F1000F03D04FF00009C3F83D
:103A40000891BEF1000F69D04FF080434FF0000E97
:103A5000C3F800E15AB14FF08043DFF8E4E00122FF
:103A60004FF00209C3F80823CEF800901A61BCF1A8
:103A7000000F41D161B1324B4FF0804900211960F4
:103A80004046C9F80C11FFF7C3FE0123C9F81430F2
:103A900074B14FF0804300210124C3F81011404657
:103AA000C3F80443FFF7EEFE10B9264BC3F80041FC
:103AB0004FB1224B00221A601B6801934FF48E70A5
:103AC000019B00F095FB4EB11F4B00221A601B6852
:103AD00002934FF49270029B00F08AFB55B31B4B8C
:103AE00000221A601B680393039B4FF4907005B08B
:103AF000BDE8F04300F07CBB4FF080430022C3F8E8
:103B000004218207B6D50222C3F80823D3F81C3457
:103B10009B07AFD10029BCD00124ACE7002AA6D076
:103B20004FF08043D3F80C3403F00113B3F1011FBD
:103B30009DD190E705B0BDE8F08300BF1C010040B7
:103B4000340C004000E100E024010040200100406E
:103B50000146014807F02EBE3C8A0020020600F014
:103B60000F0303D5072B05D909487047072B07D941
:103B7000084870470848242202FB03002830704799
:103B800003F10900044B242202FB0030F6E700BFDA
:103B9000E4200020282200209C1F002038B5054684
:103BA0000F4803F009F9B0B10E4C217845B181B945
:103BB00043681B68984758B110F1440F08D038BDCE
:103BC00061B1436829465B68984710F1100FF2D144
:103BD00025700020F3E76FF01200F0E70846EEE7EB
:103BE00021C30000DD4D00200949BFF35B8F51E880
:103BF000003F43F0010241E800200028F7D1BFF365
:103C00005B8FDB0703D40839024807F0D3BD704748
:103C1000AC1F00205428002010B5054C0021204680
:103C200003F026FB18B1043007F027FDF6E710BDBE
:103C30003C8A002013B56C46002318222146134805
:103C400003F0C6F9002818DAFFF7E6FF0023182270
:103C500021460E4803F0BCF900280CDB009B94E8D9
:103C600003001A1D82E8030004221A751846FFF7A4
:103C70006FFFFFF7B9FF002305E0009B94E8030006
:103C80001A1D82E80300184602B010BD0C8A0020FD
:103C9000817870B506460846FFF760FF0B060546BB
:103CA000F47813D5002C41D1FFF7C4FF0346002858
:103CB0003CD0012285F82240027503220274DD60A7
:103CC000FFF746FFBDE87040FFF78EBF54B1012CEF
:103CD0002CD1FFF7AFFF034640B385F821400475B0
:103CE0000474ECE7FFF7A6FF00B3B27812F0800F80
:103CF00002F00F030E4A0FD0072B9BBF142101FBCC
:103D00000323D2F8A836D3F80836EB6001230375F5
:103D100002230374C560D3E7072B9BBF142101FB6B
:103D20000323D2F8A837D3F80837EEE770BD00BFF9
:103D300000700240F0B5064689B01822002102A8A2
:103D400005F0E1F93378013B052B20D8DFE803F0DB
:103D50007703141F671603238DF814300024FFF730
:103D600069FF034698B105A9047500F10C0203C967
:103D700082E8030018461DE00423EDE7B178084609
:103D8000FFF7ECFE837A05461BB1032B43D909B03C
:103D9000F0BD0B06F47812D5002CF8D1FFF74AFFDE
:103DA00003460028F3D0012285F822400275032241
:103DB0000274DD60FFF7CCFEFFF716FFE7E75CB1AA
:103DC000012CE4D1FFF736FF03460028DFD085F849
:103DD000214004750474ECE7FFF72CFF0746002828
:103DE000D5D00123037502230374C56005F10C01CE
:103DF000B07804F005FE134AE968B2F8B0328B429D
:103E000006D95B1AA2F8B03204F011FE3846D1E7A9
:103E1000A2F8B042FAE73046FFF73AFFB7E7684644
:103E2000FEF7A4FA9DF80130052B04D19DF800306F
:103E300013F0600FABD0044B059301248FE70224ED
:103E40008DE700BF9C1F002008210020F8B5002549
:103E5000424F2E4665F07F00C0B2FFF77FFE036938
:103E60000446002B5CD02369E660C4E906330123D5
:103E70001D44082D84F82030267284F8216084F8CF
:103E80002260E7D10025354F2E46E8B2FFF766FEE7
:103E900003690446002B4ED02369E660C4E906336B
:103EA00001231D44082D84F82030267284F82160F7
:103EB00084F82260E9D12A4CD4F85831002B43D041
:103EC000D4F85831C4F86031C4F8643101220023B9
:103ED00084F86821C4F8543184F8693184F8503189
:103EE00084F86A31D4F89C323BB94FF480621D49A2
:103EF0001A4803F06DF800281ADBD4F89C32C4F895
:103F0000A4320020C4F8A832012384F8AC32C4F8EB
:103F1000980284F8AD0284F8940284F8AE0209E0B5
:103F200000F110014022384603F052F800289ADAD6
:103F30006FF00B00F8BD00F110014022384603F08D
:103F400047F80028A8DAF3E74FF4806204F5AC7173
:103F5000024803F03DF80028B2DAE9E7F0890020D2
:103F60009C1F0020382200202DE9F043DFF87C92CE
:103F70009A4D85B080460021484603F079F90746FE
:103F800010B905B0BDE8F0836B793A7D5BB9002AC2
:103F9000F1D13A7B042A52D8DFE812F0CD008F002D
:103FA0009900DB00E700042A49D801A151F822F06A
:103FB000933F0000C53F000081410000A94100007F
:103FC000B94100003B7CFC68032B38D8DFE803F0E4
:103FD000023F5E63A66908220021304605F093F88F
:103FE0007F4BD3F880243270D3F884247270D3F8D6
:103FF0008824D3F88C1442EA01227280D3F89024EA
:10400000D3F8941442EA0122B280D3F89824D3F86A
:104010009C3442EA0323F3800823E36000212368F1
:10402000607A984796F90030002B0CDBF28852B189
:10403000B5F8B0329B1AA5F8B03204F0F8FC381D80
:1040400007F01BFB97E70023A5F8B032F7E794F8D9
:104050002130002BF3D094F82030002BEFD0002635
:1040600084F821604FF0FF3184F820605D4803F050
:104070004FF8A36901936368CDE9023601A9607A1C
:10408000FEF7D2F8574803F0B3F8D8E723680121C8
:10409000607A9847D3E7A37A63B994F823304BB991
:1040A0004FF0FF314F4803F033F804F0D5FC4D4892
:1040B00003F09EF823680221EAE7FEF76BF8002878
:1040C000BDD1FDF78BFF0120FFF768FDB7E70024A6
:1040D00064F07F00C0B2FFF741FD037A13B1407A6C
:1040E000FEF706FC0134082CF2D195F850311BB1D3
:1040F00095F85101FEF7FCFB0024E0B2FFF72EFD1E
:10410000037A13B1407AFEF7F3FB0134082CF4D1A3
:1041100095F894321BB195F89502FEF7E9FB012062
:10412000FEF712F801236B712B68002B87D000215A
:104130000220984783E700246C71FEF761FB20465C
:10414000FFF72CFD2B68002B3FF479AF21460420AC
:10415000EFE7002B3FF473AFFEF76CFB2B68002BEF
:104160003FF46DAF00210520E3E72A68002A3FF401
:1041700066AF002B3FF463AF0021062090475EE757
:1041800008F10C044FF0FF31204602F0C1FFFFF7A9
:104190005DFE204603F02CF858F8083C002B3FF455
:1041A0004EAF00210120C4E758F8083C002B3FF433
:1041B00046AF00210A20BCE7002004F0AEFEFEF767
:1041C0001FFBFDF701FFFFF727FDFFF73FFE012073
:1041D00004F0A3FE0448FDF7E7FF30E79C1F002032
:1041E00000700240B01F0020353D00003C8A0020D6
:1041F000B0F5907F10B517D0B0F5927F04D0B0F530
:104200008E7F13D1012400E00224FFF713FD68B173
:10421000002202750473FFF79BFC054B1B792BB141
:10422000BDE81040FFF7E0BC0024EEE710BD00BF82
:104230009C1F002038B51A4C257965BB194BA56029
:1042400004F11400C4E9033507F033FA2A460121CA
:10425000272001F061F91448FDF7A6FF134B98429F
:104260001BD1012004F059FEFFF7F0FD054608B907
:10427000012323710E4B1B680BB1FFF7B5FC4FF008
:104280008043D3F83834DB0703D54FF48E70FFF743
:10429000AFFF284638BD0025FBE76FF00405F8E7BF
:1042A0009C1F0020693F0000353D00000000AD0B61
:1042B0003C8A002038B54FF0FF31274802F028FF34
:1042C000FFF7AAFC002464F07F00C0B2FFF746FCB1
:1042D0000546103007F0D1F9013424220021284688
:1042E00004F011FF082CEED10024E0B2FFF736FCF9
:1042F0000546103007F0C1F9013424220021284678
:1043000004F001FF082CF0D1144C04F5AC7007F058
:10431000B4F92422002104F5A47004F0F4FE04F59D
:10432000277007F0AAF92422002104F5237004F075
:10433000EAFEFEF765FAFDF747FE0020FFF72EFCC8
:10434000002004F0EAFD002504F11400257102F0BC
:104350004FFF284638BD00BFB01F00209C1F002023
:10436000064B1A7932B15B79002B0CBF6FF012004B
:10437000002070476FF01200704700BF9C1F0020A4
:1043800038B50E4B1B790146A3B105782846FFF7D7
:10439000E5FB18B96FF01504204638BD45720B795E
:1043A000498883724C1E0C404160F3D1284604F0CA
:1043B00022FBF1E76FF01204EEE700BF9C1F002024
:1043C000114B1A7910B50146BAB15B79ABB1FFF761
:1043D000C5FB0446A0B1837A032B05D8DFE803F0C0
:1043E0000210090904F03BFB0020A369E060E361CF
:1043F00010BD0846FDF794FFF6E76FF01200F7E7EF
:104400006FF01500F4E700BF9C1F002008B50A4BB1
:104410001A7901464AB15B793BB1FFF79FFB38B18E
:104420000846FEF7B5FA002008BD6FF01200FBE762
:104430006FF01500F8E700BF9C1F002038B50B4B4C
:104440001A7905460C4652B15B7943B1FFF786FBFA
:1044500040B12846FDF770FF2070002038BD6FF096
:104460001200FBE76FF01500F8E700BF9C1F00206B
:104470000D4938B50B7905466BB1FFF76FFB68B195
:10448000047A74B901230372487918B12846FEF7FB
:104490002FFA204638BD6FF01200FBE76FF01500D1
:1044A000F8E76FF04400F5E79C1F00200D4B1A79E8
:1044B00010B501466AB15B795BB1FFF74FFB04466B
:1044C00050B1037A5BB10846FEF7E0F90020207294
:1044D00010BD6FF01200FBE76FF01500F8E76FF00A
:1044E0004400F5E79C1F00202DE9F0432F4C1F46A8
:1044F000237985B0064689469046002B50D06379D3
:10450000002B4DD003064ED5FFF728FB05460028AB
:1045100049D04FF0FF3104F1140002F0F9FD95F895
:10452000223003F0FF024BB104F1140002F060FEF0
:104530006FF00A04204605B0BDE8F0836C68A869F6
:1045400044452BBF4446012385F8232085F82330BA
:104550002246494604F0AAFDEC6007B13C60AC7A03
:104560004CB9FDF74FFFB04205D004F075FA104882
:1045700002F03EFEDEE7012385F82230AB690193AD
:104580000024EB68029301A930460394FDF74CFE2A
:10459000084B98421CBF85F822406FF00404E6E700
:1045A0006FF01204C6E76FF01504C3E79C1F0020EC
:1045B000B01F00200000AD0B2DE9F0411D461E4B41
:1045C00090461A790F46002A30D05B7973B3030600
:1045D0002FD411B9B8F1000F2BD1FFF7BFFA044661
:1045E00038B34FF0FF31154802F092FDE3684345C0
:1045F0001E4628BF464657B9B8F1000F07D105B18E
:104600002B600E4802F0F4FD0020BDE8F081324638
:10461000E169384604F04AFDE3693344E361E36845
:104620009B1BE360002DECD02E60EAE76FF01200D8
:10463000EBE76FF01500E8E79C1F0020B01F00209B
:1046400038B51A4D2A79034632B36A7922B31B066C
:1046500025D4FFF783FA044608B34FF0FF3105F184
:10466000140002F055FDE3688BB90125A36984F8B5
:104670002050E36194F821304BB1FFF7DBFA88B1A9
:104680000575C4600574FFF763FAFFF7ADFA0848D3
:1046900002F0AEFD002038BD6FF01200FBE76FF0B6
:1046A0001500F8E76FF00B00F5E700BF9C1F002036
:1046B000B01F002008B5074B1B792BB1FFF74EFA4E
:1046C00028B10160002008BD6FF01200FBE76FF019
:1046D0001500F8E79C1F0020014B1860704700BFD1
:1046E0009C1F002008B5074B1B7923B1FFF736FA52
:1046F00020B1406808BD6FF01200FBE76FF01500B5
:10470000F8E700BF9C1F0020104B002210B4C3F834
:1047100040214FF02002EFF3118482F31188BFF3A0
:104720006F8F0B4AD3F804051168401A20F07F43BD
:1047300023F0FF030B44136084F31188BFF36F8FE2
:10474000C0F30F2010BC03F0B9BA00BF0010014045
:104750005022002037B51E4802F02EFB002833D02F
:1047600043681C4D1B680121984700244FF4807357
:10477000C5F80845C5F840354FF48033C5F8043313
:1047800003F1804303F58A534FF400321C601B6829
:104790000193019B104B0121C3F880211120224677
:1047A00000F0BAFE112000F085FE0C4A01231360D0
:1047B0002B60D5F8043503F5807323F07F43C5F8EB
:1047C0004035204603B030BD4FF0FF30FAE700BF60
:1047D00017C300000010014000E100E00810014094
:1047E00070B54FF6FE76B0F1FF3F08BF30464FF090
:1047F0002003EFF3118483F31188BFF36F8F124D01
:10480000124BD5F804151B68421EB242A1EB0300FF
:10481000A8BF324620F07F4022EAE272FF3000EB70
:10482000022020F0FF000344591A21F07F411F2984
:1048300098BF03F5807323F07F43C5F8403584F3B8
:104840001188BFF36F8F70BD00100140502200200F
:104850004FF02002EFF3118382F31188BFF36F8FC3
:10486000064AD2F80405064A1268801AC0F30F20DF
:1048700083F31188BFF36F8F704700BF00100140B2
:1048800050220020F7B5244D286843685B6C03B1C3
:104890009847286843685B6B002B3BD098470028FB
:1048A00038D01E4C1E4E286843689B69002B31D0BF
:1048B00001220DF10701984701282BD1236843B944
:1048C00033683BB371681A6832608B4200D1726002
:1048D000236014499DF807700A88B2F5007F0846E6
:1048E00006D22368134402F1010CA1F800C01F7224
:1048F0000A2FD8D1236802885A600B4900221A6017
:104900004E6826B9C1E9003302802260CAE73360ED
:104910004B60F9E703B0F0BD7C2600205C2200204C
:1049200054220020D428002074260020044B10B507
:10493000044618684368E1B25B689847204610BD9A
:104940007C260020F8B5064615464FF02003EFF30D
:10495000118C83F31188BFF36F8F194A13684BB121
:10496000184844689C4205D000241C60446894B9EF
:10497000C0E90033144B186828B15F6804681C60F4
:10498000B84208BF5C608CF31188BFF36F8F106072
:1049900020B92860F8BD23604360EBE74C1E4168F6
:1049A0008C42A8BF0C46224600F10801304604F0B4
:1049B0007DFB0023335501232B60E018EAE700BF9D
:1049C0006022002054220020742600201E4B00226A
:1049D00013B5C3E900221D4B1D49C3F8082203F596
:1049E00002721A604A600B601A481B4C02F0E4F92C
:1049F0000246206020B343681BB19B6C0BB1174982
:104A00009847206843685B6B53B1984740B1206872
:104A100043689B6923B101220DF107019847F5E72F
:104A20000F4A2068002313804268926A1C4602B134
:104A3000904784F31188BFF36F8F002002B010BD40
:104A40004FF0FF30FAE700BF7426002064220020F8
:104A500054220020E4C200007C260020854800008B
:104A6000D428002038B543680446981850281546C5
:104A700008D80648184404F019FB62682A446260AA
:104A8000002038BD4FF00040FBE700BFDE4D0020A6
:104A90002DE9F0433F4BDFF80C911B88D9F800005B
:104AA000DFF8048181883C4EB7B00225ADF80C30A8
:104AB0003A4B5F680378C7F3072242EA0722428035
:104AC00001330A02037042EA1122002343708280FC
:104AD0000821009341F2210203F05EFA012203460D
:104AE000ADF810000092394641F22102404603F031
:104AF00053FA336840BAADF81000BCB203A85B6843
:104B00000221984736A904F10A035BBA21F8C63D91
:104B1000022206A804F0CAFAD9F80010ADF8125023
:104B200008220DF11A0004F0C1FABDF81200083095
:104B300006AB80B2ADF812003A464146184404F084
:104B4000B5FABDF81200204406AB80B2ADF81200F1
:104B50002A4604A9184404F0A9FABDF812302B44DF
:104B60009BB205AAADF8123000936D2106AB1AA8CE
:104B7000FCF720FC05993368ADF812101AA85B68A1
:104B800089B29847336806485B682946984737B02A
:104B9000BDE8F08307BD000080260020D8880020F3
:104BA00049C3000084260020DE4D00202DE9F0439B
:104BB0000023ADF52D7D4FF0FF320024CDE9042315
:104BC000CDE9062305460E464FF4007221462CA877
:104BD000039404F098FA3246294617A802F086F8A2
:104BE0000DAB20AA214617A806F0B1FC9DF846306F
:104BF00003F0DF03802B27D003254FF0FF328449D9
:104C0000844802F093F88449814804F0EAF92A467E
:104C1000EB177F4806F08BFA4DB980497C4804F0C9
:104C2000E0F97F4B7A481A682B4606F071FA78490A
:104C3000784806F09DFAFFF72BFF039804F0EEF892
:104C40000DF52D7DBDE8F08312A90DA806F08BFCB3
:104C50000028D1D1734E714FDFF8D48104469DF8FE
:104C60005A30FF2B28D1DDE90423002B08BFB2F115
:104C7000FF3FC1D00020FBF769FC03A9C0B2FEF7DB
:104C800077FD0028B8D1DDE9048958EA0903644EAC
:104C90000AD1039B3060DDE906019A680023824255
:104CA0008B41A9DB604B186033680021894508BF40
:104CB00098455ED00025A0E702A912A806F0D5FC11
:104CC000002899D19DF85A30602B95D1029B062B74
:104CD00092D809AD12AB02AA2946184602F036F85E
:104CE000002889D1029B3146E854284604F0C1F9D6
:104CF000D8B99DF85A30402B7FF47EAF02A912A894
:104D000006F0B3FC00287FF477AF029BB3F5007F79
:104D1000BFF472AF12AB02AA2CA9184602F016F823
:104D200000287FF469AF029C99E73946284604F0D1
:104D3000A0F988B99DF85A30002B7FF45DAF04A923
:104D400012A804F05BF900287FF456AF12A806F011
:104D500084FC002883D04FE74146284604F089F9B7
:104D60000028F3D19DF85A30002B7FF445AF06A9F7
:104D7000E6E72D4A116823448B42904607D20398F8
:104D800004F0B9F8B4FBF0F303FB1040241A3068C8
:104D90000BA92044FBF7E4FB054600287FF42DAF68
:104DA000224F0B993B68994225D123462CAA3168A2
:104DB000039804F051F800287FF41EAF3068D8F84B
:104DC000003004449C4234607FF474AF039803F0D5
:104DD0007FF80BA9FBF7C4FB054600287FF40DAF55
:104DE0000B993B6899427FF765AF0C9A039804F0E2
:104DF0005CF8054601E7039B0C9A0193184639605D
:104E000004F053F8054600287FF4F7AECDE700BF65
:104E1000AC2600208826002059C3000051C30000A2
:104E2000D02600204CC30000D4260020E0880020BB
:104E300055C3000038B50C4C0C4D4FF0FF322146E5
:104E4000284601F073FF0A49204604F0CAF80023FF
:104E50000022204606F06BF92146284606F088F924
:104E6000BDE83840FFF714BEAC260020882600209D
:104E700059C300002DE9FF410C681B4E1B4B023843
:104E80000F46C4F50071009003AA01313019FCF7F8
:104E900013FB054628BB3B68039A1344022B3B6077
:104EA0001BD93288140244EA1224A4B2023B9C4269
:104EB00013D14FF001080346CDF8008041F22102E2
:104EC0002146B01C03F068F838B9022C05D93B68BC
:104ED000023B1E443B60B5704546284604B0BDE821
:104EE000F0814FF0FF35F8E72E4E002031500020C2
:104EF0002DE9F0470729B0B004465ED9027812F0D8
:104F0000FD025AD14088030243EA1023A1F10805AB
:104F10009BB2AB4251D3A188604B61481C600B022D
:104F200043EA11235F49A3804A6006F0ECF8A388A6
:104F3000012B40F0A180E3792BB1012B00F096808A
:104F4000FFF778FF39E04FF0FF3257495448574D8B
:104F5000DFF86081DFF8609101F0E8FE54495248C3
:104F600004F03FF84FF0FF320EA94F4806F0FDF86D
:104F7000002600273046FBF7E9FA05A9C0B2FEF784
:104F8000F7FB044658B92023014606AA059803F00A
:104F900046FF069BAB4216D0059803F03FFF002F5B
:104FA00008BF012E0CD10EA93F4806F0E1F83E499A
:104FB0003B4806F0DDF8FFF76BFD30B0BDE8F08749
:104FC00001260027D6E7CDE901440094402320AA1A
:104FD000059906A8FBF7FEFF0028DDD1059803F030
:104FE0001DFF4FF0FF3217A90EA801F09FFE4146AA
:104FF00017A803F0F6FF32463B4617A806F097F8CD
:10500000494617A803F0EDFF9DF82C1020A803F0E7
:10501000C9FF30AB441C18444FF02E0A20AB00F8F7
:1050200040AC9DF82D10181903F0BCFF30AB2044A4
:10503000441C184420AB00F840ACBDF82E101819E1
:1050400003F0B0FF30AB20440344013003F840AC20
:1050500020AB0C99184403F0A5FF20A917A803F072
:10506000C0FF17A90EA806F083F898E7294604F1B7
:105070000800FFF79BFDA0E7002B9ED1E379012BF1
:105080003FF45EAF052B98D1FFF7D4FEFA2002F073
:10509000F9FB0120FEF7A4FB8FE700BF8426002068
:1050A00088260020D8880020AC2600203DB8F39642
:1050B00035C300003CC3000041C300002DE9F341AB
:1050C0001B4B1C4FDFF870801860064600243D46DD
:1050D000C4F50071336801AA0131381998470028D6
:1050E000019B01DC002BF3D004442BB940F20123D7
:1050F0009C42EDD10024EBE72B78062B11D16B7885
:10510000092B06D102A9002341F8083DA01EFFF794
:10511000B1FE0128EED1009940460239FFF7E8FEC2
:10512000E8E7042BF5D16B78142BF2D16946EDE753
:10513000802600202F500020304E00200448816837
:10514000006A884203D003494FF080520A607047DA
:105150001C28002004ED00E0044800232021C21890
:105160000133302B82F80013F9D1704700E100E0E1
:10517000094A0A49936809689966094958664B685B
:1051800043F080534B60002383F31188BFF36F8F8C
:105190009368986E704700BF1C28002080C00000F4
:1051A00000ED00E013498A684FF028001044EFF347
:1051B000098C80E8F01F202080F31188BFF36F8FE7
:1051C0000D4F4FF000660A6A8A603E60506E002301
:1051D000536680F3118804B50648806803F039FFF0
:1051E000BDE8044002F1280090E8F01F8CF3098824
:1051F000704700001C28002004ED00E01EF0040FA2
:105200000CBFEFF30880EFF30980816931F8021CCD
:1052100011F0FF010229FFD001B503F00FFF01BD1E
:1052200038B51B4C05461B4803F070FAA36AD90633
:1052300002D5194803F06AFAA36A1A0702D517487B
:1052400003F064FAA36A9B070ED5154803F05EFAD3
:10525000616BA36A180607D5124803F057FA1DB10F
:10526000A36A23F08003A362094CA36ADA0702D57C
:105270000D4803F04BFAA36A9B0602D50B4803F0D6
:1052800045FAA36AA36A43F0FF03A362002038BD76
:1052900000ED00E0EAC3000001C4000035C40000D6
:1052A00049C4000062C4000079C4000099C4000031
:1052B00038B51E4C05461E4803F028FAA36AD904E7
:1052C00002D51C4803F022FAA36A1A0502D51A482F
:1052D00003F01CFAA36A9B050ED5184803F016FAD2
:1052E000A16BA36A180407D5154803F00FFA1DB186
:1052F000A36A23F40043A3620C4CA36A590502D5A8
:10530000104803F003FAA36ADA0509D50E4803F042
:10531000FDF9064A936A43F47F439362002038BD47
:10532000A36A9B04F5D50948F1E700BF00ED00E052
:105330005CC3000073C3000035C4000085C30000D7
:105340009FC30000B5C30000D1C3000099C4000092
:1053500010B5194C194803F0D9F9A36A9A0102D57E
:10536000174803F0D3F9A36ADB0102D5154803F00F
:10537000CDF9A36A180302D5134803F0C7F90E4C00
:10538000A36A590302D5114803F0C0F9A36A9A032E
:1053900002D50F4803F0BAF9A36ADB0302D50D4822
:1053A00003F0B4F9044A936A6FEA03436FEA1343C4
:1053B0009362002010BD00BF00ED00E0C9C40000F2
:1053C000E2C40000F6C4000011C5000030C50000B2
:1053D00056C5000071C5000038B5274C6368C3F39B
:1053E0000803DA1E0546092A3AD8DFE802F0053339
:1053F0003530393939393937204803F087F9E36ACC
:105400009A0703D51E4803F081F902E0E36A5B00C6
:1054100005D400202946BDE8384000F0DFB819481F
:1054200003F074F9184B1B782BB10120FFF7F8FE3D
:105430000628EFD138BD154B1B781BB10120FFF7B3
:1054400037FFF5E7124B1B889BB2002BE1D0FFF72B
:105450007FFFEDE70020E9E70020F0E70D48D2E705
:105460000D480E49A3F110020F2BD8BF01460C487E
:1054700003F04CF9CDE700BF00ED00E0CBC5000024
:10548000E3C5000005C6000028ED00E029ED00E0BE
:105490002AED00E025C600009DC50000B2C5000051
:1054A0005CC60000024A536943F010035361704721
:1054B00000ED00E043B2002B08DB012200F01F00EA
:1054C00002FA00F05B09024A42F82300704700BF6D
:1054D00000E100E043B2002B0DDB01225B0900F08C
:1054E0001F0002FA00F02033034A42F82300BFF302
:1054F0004F8FBFF36F8F704700E100E04209054B0B
:1055000000F01F0053F82220012303FA00F010409E
:10551000704700BF00E100E043B2002BA8BF03F1D9
:10552000604301F101014FEA4111AEBF03F5614350
:1055300000F00F00034BC9B2ACBF83F8001319543D
:10554000704700BF14ED00E02DE9F0418C1888464B
:1055500017461E4604220A9B0999054606F040FAA2
:10556000A4F120030C4923F00703002221F00101DC
:10557000C5E91322C5E9168799610699596007990B
:1055800099600899D9604FF080711E60D961AB6451
:105590006A66BDE8F08100BFE38300000149102284
:1055A0000A60704710ED00E0404080F3118830BF82
:1055B000704700BF404080F31188DFF81CC0DCF862
:1055C00000C01CF4006C0CBFEFF30880EFF30980FF
:1055D00001B5FFF701FF01BD04ED00E038B5044659
:1055E0000D4605281AD8DFE800F00319191315171E
:1055F0000D4803F08BF802F065F9AA6901460B48E3
:1056000003F084F829462046BDE8384000F018B879
:105610000748EEE70748ECE70748EAE7014607488E
:1056200003F074F8E7E700BF70C600000EC7000083
:1056300090C60000B6C60000D0C60000EBC6000051
:10564000052810B50CD002F0A5F960B102F0A2F95E
:105650000C490D4B002808BF19460C4803F056F8BA
:10566000FFF7A2FFFCE702F0A5F90028EED1084CF5
:105670000848A16803F04AF8A068BDE8104000F0AF
:105680000BB800BF4AC700004EC700005FC700004C
:105690001C2800207FC7000038B505464FF02003C6
:1056A000EFF3118483F31188BFF36F8F06F079F95C
:1056B0000A4B9B68AB420BD1094B5A68C2F30802F4
:1056C00012B92046FFF754FD5A6842F080525A60E2
:1056D0002046BDE8384006F0A2B800BF1C280020D4
:1056E00000ED00E001B5EFF30580A0F110004FEAF6
:1056F000C0000449014409C99847BDE80140024877
:1057000000470000ACBA00003D51000003F0B9F8BA
:10571000202080F3118808484FF40061401880F37E
:105720000988EFF314800221084380F31488BFF343
:105730006F8F00F007F80000B87B002030BFFFF744
:10574000FDBF00BF08B5084B084A23F07F039360F4
:10575000BFF34F8FBFF36F8F01F054FB01F05CFB81
:10576000FFF7FAFC01F086FB0000000000ED00E00E
:105770001FB5094B0193094B029304A8084B0393EF
:1057800001AB40F8103D074A074B012100F076F8C5
:1057900005B05DF804FB00BF000000200000000021
:1057A00000000B06000000200000042030B5D1E905
:1057B0000043202B896817D9B3F1004F16D8013B5D
:1057C000B3FA83F3C3F11F035B00072841F0010123
:1057D0000ED824F01F02084D024342F010020B4382
:1057E000A860EA602B6130BD0823EEE73E23ECE7BA
:1057F0006FF01500F7E700BF90ED00E0034B0522C6
:105800005A60BFF34F8FBFF36F8F704790ED00E08A
:10581000BFF35F8F014B00225A60704790ED00E0AC
:1058200013490868082810B51ED8FFF7F1FF114C7E
:1058300049680022904201F10C0105D10E4B18700D
:10584000FFF7DCFF002010BDA26051F80C3C23F0F4
:105850001F0343F010031343E36051F8043C43F08B
:10586000010323610132E5E74FF0FF30EBE700BFB2
:1058700050BD000090ED00E030520020F8B5104C13
:10588000074620780E460025B54208DA57F825105D
:105890004B6893B15A1E134203D06FF0150020706D
:1058A000F8BD1F2BF9D90B681A42F6D1C0B2FFF729
:1058B0007DFF10F1160FF0D001300135E4E700BF95
:1058C0003052002070B5104B064618780D46002463
:1058D000AC4207DB10F1160F03D00C4B0022072857
:1058E0000DDD70BD56F824104B6833B1C0B2FFF720
:1058F0005DFF10F1160FF4D001300134E8E7986035
:105900001A610130EBE700BF3052002090ED00E05B
:1059100002680E4B9A4215D1C269A3F11023A3F17C
:10592000EF139A420ED18368012B0BD8C36813B1D1
:105930000269934206D0436933B18069C31A584261
:1059400058417047012070471846704755AA00FF1C
:1059500038B50D4B9D68A5B12846FFF7D9FF014624
:1059600078B9EB686BB92C690CB9084638BD20468C
:10597000FFF7CEFF28B9E368AB4202D12546246980
:10598000F2E70121F1E700BFD82600202DE9F84316
:10599000414E3468DCB1B468CCB101FB00F700289B
:1059A0004CD000294AD0B7FBF0F48C4246D1381DC8
:1059B00044D8B9070ED027F0030808F10408F468AA
:1059C00003E0636843453BD2A469002CF9D120462B
:1059D000BDE8F883B846F2E7F06045E008F1200C36
:1059E00004EB0C03203959600021C3E90214DFF8ED
:1059F000B0E02169196144F80CE0DFF8A8C0C3F8F1
:105A00001CC001B1CB60C3E90520AAB193619A69BA
:105A100002B1536123610023C4E9053333694FF0B8
:105A20000109DB07C4E901892ED5FFF791FF58B3BF
:105A30001A4B48461B6826E0F360E8E70024C6E7F7
:105A4000A3681BB1154B01201B6898476168A1EB47
:105A500008012329D4E9052004F12005BED801233B
:105A6000A360002AB8D09061A36903B15A610023F2
:105A7000C4E905333369DA0706D5FFF769FF18B1C2
:105A8000064B1B68012098473A46002128462C46C1
:105A900003F039FB9BE700BFD8260020E8880020F0
:105AA00055AA00FF669911EE2DE9F041074600283E
:105AB0007CD03F4D2B68002B78D0AA68002A75D087
:105AC000834203D86A681344984203D3394B0120B8
:105AD0001B689847A7F120042046FFF719FF18B16B
:105AE000344B01201B68984757F8183C012B03D012
:105AF000304B01201B68984757F8146C002347F877
:105B0000183CAEB1B26892B957F81C3C03F12002C0
:105B100073681344736057F8103C336103B1DE605F
:105B200020462022002103F0EEFA234634461E468A
:105B30002069002832D08368002B2FD16368426827
:105B400020331344D4E90521636003692361DAB982
:105B500001BB426981696261A161EAB19461A26994
:105B600002B1546103B1DC602022002103F0CBFAC2
:105B70002B699B071AD5FFF7EBFEB8B10D4B01203F
:105B80001B68BDE8F04118479161A1690029E0D088
:105B90004A61DEE7E960F8E7EC60E0E7002EE7D174
:105BA000EB68A36103B15C61EC60E1E7BDE8F08103
:105BB000D8260020E888002038B514220D46044677
:105BC0000021124803F09FFA1149124800F032F800
:105BD000232D1AD914F003031FBF043DED18C3F1A0
:105BE0000403E4182A460021204603F08CFA074BF0
:105BF000094A9C60C3E900452260A2F11022203DC1
:105C0000A2F1EF126560E261DC6038BDD8260020A9
:105C1000A95A00008D59000055AA00FF014B1B68CE
:105C2000184700BFE4880020014B1B68184700BFDD
:105C3000EC880020024B1860024B0020196070476E
:105C4000E4880020EC880020024B0A461B680021F3
:105C5000184700BFF0880020F8B500F10805476834
:105C6000044628460E4603F030FE874201D02748FE
:105C7000F8BD6368B3F5807FF9D80021284603F0AA
:105C8000F1FF0028F3DD0021284603F0EEFD002897
:105C9000EDD0F6B9002104F1140003F0E3FF002871
:105CA000E5DDA6B1002104F1440003F0DBFF00288C
:105CB000DDDD002104F1500003F0D4FF0028D6DD23
:105CC000002104F15C0003F0CDFF0028CFDD0020AF
:105CD000CEE704F12C050021284603F0C3FF00287D
:105CE000C5DD0021284603F0C0FD0028BFD004F127
:105CF00038050021284603F0B5FF0028B7DD002154
:105D0000284603F0B2FD0028C4D1B0E780BFFFFFF2
:105D100070B500210446FFF79FFF0546B8B904F1AE
:105D20000806304603F0B1FD7F2810D91434294607
:105D3000204603F09AFD50B1204603F0A6FD01284D
:105D400005D93146204603F04DFF002800DB014D08
:105D5000284670BD00BEFFFFF0B50C4687B000219D
:105D600005461646FFF778FF80BB03A803F0F7FC53
:105D700021466A6803A803F0AEFD0446D0B905F1D8
:105D80000804214603A803F02DFF00281BDA05F1C3
:105D9000680303A9009305F11402234608466F68BF
:105DA00004F0BBFA044628B93A46314603A803F08A
:105DB000C8FD044603A803F0D8FC0CB1A4F5854443
:105DC000204607B0F0BD6FF00304F3E7004CF7E79F
:105DD00080BFFFFF0023C0E90033C1B9194A1A4B45
:105DE000DFF88CC0C0E90223184B194AC0E904C38C
:105DF000184BC0E90623184B036203F17453A3F553
:105E00002303A3F692434362816600207047134B3D
:105E1000134ADFF860C0C0E9022303F1794303F5B8
:105E2000740303F5016303610E4BC0E905C303F17D
:105E3000D14303F5C01303F51E63C3610A4B03622C
:105E40000A4BE0E767E6096A85AE67BB3AF54FA5FE
:105E50007F520E518C68059BABD9831F07D57C36CA
:105E6000D89E05C1310BC0FFA78FF964A44FFABEBD
:105E700072F36E3C39590EF72DE9F04FCFB000F1B7
:105E8000080304931A46002306AC52F8040B44F8A6
:105E900023000133082BF7D100224B7808781B042C
:105EA00043EA0063C8780343887843EA00230EA8D6
:105EB000043140F822300132102AEED1A14DDDF834
:105EC00034E0099C0C98089B0B99079ADDF8289000
:105ED000069F00950DF1380BDA46A846D8F8005019
:105EE000DAF800604FEAF92C8CEAB91C35448CEAE8
:105EF000796CAC4480EA010505EA09054540AC44EB
:105F000047EA02064FEA7735E64485EAB70507EA2D
:105F1000020C1E4085EAB75546EA0C062E4474442E
:105F2000D8F80450B644DAF804603544054489EAE8
:105F30000100204080EA010C05EB0C004FEAF4253B
:105F400085EAB41585EA746505444EEA07064FEA0A
:105F50007E300EEA070C80EABE00164046EA0C06C8
:105F600080EABE50304428442B44DAF80860D8F860
:105F7000085035440D4484EA0901194081EA090CAE
:105F800005EB0C014FEAF32585EAB31585EA736545
:105F90000D444EEA00064FEA70310EEA000C81EA29
:105FA000B0013E4046EA0C0681EAB0513144294432
:105FB0002A44DAF80C60D8F80C503544A94484EA35
:105FC0000305154085EA040C09EB0C054FEAF2299C
:105FD00089EAB21989EA7269A94440EA01064FEADE
:105FE000713507EB090C85EAB10500EA010706EAFD
:105FF0000E063E4385EAB155DAF810703544D8F8FC
:1060000010604D443E4483EA0209344409EA0C0915
:106010004FEAFC2689EA030986EABC164C4486EA64
:106020007C66264441EA05074FEA753401EA050912
:1060300084EAB504074047EA090784EAB5543C44BA
:106040003444B644D8F81470DAF814603E4433444B
:1060500082EA0C0606EA0E06564033444FEAFE2654
:1060600086EABE1686EA7E661E4445EA04074FEAC3
:10607000743305EA04090F4083EAB40347EA0907C9
:1060800083EAB4533B4433443044D8F81870DAF808
:1060900018608CEA0E093E44324409EA00094FEACE
:1060A000F02689EA0C0986EAB0164A4486EA706648
:1060B000164444EA03074FEA73322F4004EA030907
:1060C00082EAB30247EA090782EAB3523A44324409
:1060D0003144DAF81C70D8F81C608EEA00093E449E
:1060E00009EA01094FEAF127B44489EA0E0987EA6F
:1060F000B117CC4487EA7167BC4405EB0C094FEA41
:10610000723743EA020587EAB207254003EA02062E
:10611000354387EAB2572F440B4D08F12008454517
:1061200067440AF1200A7FF4D9AECDE90B10CDE91E
:106130000672CDE908343EADCDF834E0CDF82890B4
:10614000059503E0C4BE000004BF0000DBF8385032
:10615000DBF804C0DBF800604FEAF54888EA7548D0
:1061600088EA9528DBF824504FEABC4A35448AEA8D
:10617000FC1A8AEADC0AA8444FEAF92608EB0A0569
:1061800086EAB916039586EA796580EA010606EA89
:10619000090646402E44009D2D6C3544039ECBF8E5
:1061A00040603544AE4404EB0E0847EA02054FEA6E
:1061B000773407EA020684EAB7041D4084EAB7543C
:1061C00035432544DBF83C40DBF808604FEAF44AED
:1061D0008AEA744A8AEA942ADBF828406444A24492
:1061E000009CAE444FEAB64585EAF615646C89EA30
:1061F000010C85EAD60555440CEA080C04444FEA24
:10620000F8202C448CEA010C80EAB81080EA78600F
:10621000A44400EB0C04234401934FEA7E3047EA88
:106220000E0307EA0E0C80EABE00134043EA0C039B
:1062300080EABE501844039BCBF844504FEAF34C1D
:106240008CEA734C20448CEA932CDBF80C40DBF88E
:106250002C301E444FEAB44383EAF41383EAD40398
:1062600066441E44019BCBF8486089EA080C0CEA9E
:10627000030C009B9B6C0B4433448CEA090C9C443C
:10628000019B4FEAF32181EAB31181EA736101EBCB
:106290000C031A4402924FEA70314EEA00020EEAF1
:1062A000000C81EAB0013A4042EA0C0281EAB051A6
:1062B00011441944DBF83030DBF810204FEAF54C7C
:1062C0001C448CEA754C019B8CEA9525254488EA90
:1062D0000304029B1C40009B4FEAB24C8CEAF21C68
:1062E000DB6C8CEAD20CAC444B44634484EA080473
:1062F000CBF84CC01C44029B4FEAF32585EAB3154A
:1063000085EA73652B1940EA010500EA010405EAF4
:106310000E0525434FEAF6444FEA713984EA764484
:1063200089EAB10984EA9626DBF8344007EB030AD0
:1063300089EAB159DBF8147022444D441D441644D7
:10634000DDE901344FEAB74282EAF71282EAD70266
:10635000324483EA040606EA0A065E40009BCBF854
:1063600050201B6D4FEAFA241344434484EABA14C4
:106370001E4484EA7A64A31941EA05064FEA75349B
:1063800001EA050884EAB504064046EA080684EAFC
:10639000B55434441C449E44DBF81880DBF8383094
:1063A0004FEAFC4686EA7C4686EA9C2CDE194FEAD8
:1063B000B84383EAF81383EAD80366441E44029B79
:1063C000019FCBF8546083EA0A0C0CEA0E0C8CEAAD
:1063D000030C009B5B6D33443B449C444FEAFE231B
:1063E00083EABE1383EA7E6303EB0C0745EA040CE1
:1063F0004FEA743305EA04090CEA010C83EAB4039A
:106400004CEA090C83EAB45363443B443844DBF858
:106410001C7001974FEAF24CDBF83C708CEA724C2E
:106420008CEA9222B8449044019A019F4FEAB2420A
:1064300082EAF71282EAD7029044009A029F926D94
:10644000CBF858808AEA0E09424409EA00094FEA6B
:10645000F02C89EA0A093A448CEAB01C4A448CEAD6
:10646000706C944444EA03084FEA733208EA050862
:1064700004EA030982EAB30248EA090882EAB3524D
:106480004244624461444FEAF64C8CEA764CDBF8B5
:106490002080039F8CEA962C019E3E444FEAB84729
:1064A00087EAF81787EAD808009F6644FF6D4644DC
:1064B0008EEA0008374408EA01084FEAF12C5744F5
:1064C00088EA0E088CEAB11CB8448CEA716CC444AA
:1064D00005EB0C094FEA723743EA0205CBF85C6022
:1064E00087EAB207254003EA0206354387EAB25736
:1064F0002F44009D20350095059D0BF1200B5D4537
:1065000067447FF423AECDE90B10CDE90672CDE9E7
:106510000834CDF834E0CDF828900023049A1168AF
:1065200006AA52F823200A440499013341F8042BA7
:10653000082B0491F2D100204FB0BDE8F08F00BFCE
:1065400008B5094B1A786AB901211970062005218E
:10655000FEF7E2FF0620FEF7ADFF044B4FF00042CE
:10656000C3F80423002008BD315200200060004021
:106570001F288ABF094B4FF0A04300F01F0003EB18
:106580008000D0F8003723F44033C0F80037D0F84B
:10659000003743EA0141C0F800177047000300507C
:1065A000F7B5036886689B6801F01F040D464C49E7
:1065B0001B79D1F8042344EA4314D2B2002303F533
:1065C000A27051F82000C0F3052084426CD122FA59
:1065D00003F0C00768D59A0002F1804202F5C0427C
:1065E000D2F8100520F00100C2F81005012202FACD
:1065F00003F3C1F8083320460021FFF7B9FFB06864
:10660000E84010F001004DD0F068E84010F00100C3
:1066100048D07069E84010F0010251D0B369EB40F6
:10662000DB0745D43369F269EB4022FA05F503F044
:10663000010305F00105AB420CBF02250125284FDF
:10664000002101F5A27357F8230010F0030031D1A7
:106650008A0002F1804303F5C0432402D3F8106599
:1066600026F44F3626F44076C3F81065D3F810654B
:1066700004F47C5402F1804202F5C24244EA05452A
:106680003543C3F81055106012680192019AD3F88F
:10669000102542F00102C3F81025012303FA01F18D
:1066A000C7F8041303B0F0BD0133082B87D1A2E76C
:1066B0000325C4E701310829C3D16FF01200F1E7C7
:1066C000F16933694B4023FA05F515F0010F2046B7
:1066D0000CBF03210221FFF74BFF1046E2E700BF8A
:1066E000006000402DE9F84F0746856803F47040CC
:1066F000B0F5804F1E4647D02ADCB0F5805F3BD016
:10670000B0F5405F3CD050BB06F44078B8F5807FD0
:106710003CD0A8F500746342634106F0010C4FEAD7
:106720004C08012948EA0C0818BFD4B248EA0020F6
:10673000DFF8D4A012BFA1464FF01F09002440EAA1
:1067400083084FF0010BA14522D20020BDE8F88F4D
:10675000B0F5E04F16D005DCB0F5A04F0ED06FF0CD
:106760001500F3E7B0F5404F04D0B0F5504FF6D127
:106770000720C9E70620C7E70120C5E70320C3E7D4
:106780000420C1E70520BFE70220BDE70323C4E7DB
:106790003B689B681A7904F01F0343EA42131F2BDE
:1067A000C6BF03F01F0352464FF0A04203F5E0734B
:1067B000B10742F82380AB680BFA04F24CBF1343D5
:1067C0009343AB606B69B0064CBF134393436B615B
:1067D000AB6971064CBF13439343AB612B697007E0
:1067E0004CBF134393432B61EB6931064CBF1A43F3
:1067F00023EA0202EA6121463846FFF7D1FE00286B
:10680000A4D10134E4B29EE700030050F0B50026A5
:1068100085B0CDE902662B4D2C68012C0BD12A489E
:1068200004F086F90290294804F082F903902E6062
:106830002B680093009B264E002301279C46D6F828
:10684000042307FA03F111421ED003F1805202F52E
:10685000C25292001168012916D103F5A2700DF100
:10686000100E56F82050C2F800C0C5F340300EEBB1
:106870008000C5F30425A940126850F8085C019215
:106880002943019A40F8081C0133082BD7D1029AFA
:106890001AB10D49886804F0D8F8039A2AB10A4B56
:1068A00003F10C01586904F0D0F8012C08D1064816
:1068B00004F067F9054805B0BDE8F04004F061B99F
:1068C00005B0F0BD7C610040A8890020B48900209B
:1068D00000600040014B00201970704732520020C8
:1068E000024B0B6001231360704700BF2C27002070
:1068F000012210B511460748074C05F041F801F098
:10690000E0FF206001F0D9FF044B606001221A70A3
:10691000002010BD342700202C27002032520020F8
:10692000F8B516460D4601F0C8FF174BB6FBF0F45C
:106930001B78074603BB3146284604F08BF9F0B1BB
:10694000B5FBF7F307FB1353CBB907FB1467B7B9D4
:10695000C4B14FF0FF310D4800F0E0FF01F0ADFF92
:1069600004462846FAF78AFF361B2544F9D1074822
:1069700000F0AEFF3046F8BD6FF00C00FBE76FF0A3
:106980001500F8E72046F6E73252002034270020B1
:106990002DE9F8431D46284B1B780C461646002B64
:1069A00041D12946204604F055F900283ED0002D5B
:1069B0003FD04FF0FF31214800F0B0FF14F0030743
:1069C0000CD0C7F10407AF4228BF2F4631462046FE
:1069D0003A46FAF781FF3C443E44ED1B25F003089C
:1069E00004EB0807A6EB040905E059F8041020465B
:1069F000FAF764FF0434A742F7D1AA086FF0030343
:106A000003FB025206EB080112B13846FAF764FFA5
:106A10000B4AD2F80034DB07FBD5084800F058FFDA
:106A20000020BDE8F8836FF00C00FAE76FF0150066
:106A3000F7E72846F5E700BF325200203427002050
:106A400000E0014070B54B79012B23D18B79032BEA
:106A500020D1CC792CB1012C1CD103689B681B7907
:106A6000C3B10A7912B1022A14D10E2203689B68BD
:106A70001D680B6847F61226B3426BD027D8B3F5D2
:106A8000965F61D012D8B3F5167F4DD005D8B3F517
:106A9000967F74D06FF0220052E0B3F5966F50D01D
:106AA000B3F5166FF6D14FF41D233FE0B3F5615FE8
:106AB0004CD004D8B3F5165FECD1324B36E0B3F5C9
:106AC000964F45D0B3F5E14FE4D12F4B2EE0B3F50F
:106AD000E13F48D012D84DF6C026B3423DD005D88C
:106AE000B3F5164FD6D14FF41D031FE0B3F5614F38
:106AF00036D0B3F5963FCDD1244B17E0B3F5E12F57
:106B000037D008D8B3F5613F30D0214EB342C1D160
:106B10004FF080630AE0B3F5612F2DD01D4EB342D4
:106B2000B8D14FF0805301E04FF41C33C5F8243541
:106B3000836803C92243C5F86C2583E8030000205D
:106B400070BD4FF49E23F1E7134BEFE7134BEDE7D6
:106B5000134BEBE74FF40003E8E74FF46503E5E779
:106B60004FF46B03E2E74FF0EB73DFE74FF06C732A
:106B7000DCE74FF0E863D9E74FF07063D6E74FF4F6
:106B8000A033D3E70050270000C0750000903A0101
:106B900090D0030040420F0000B0130000F03A0014
:106BA00000A04E00F8B503680A689B6885681C68F9
:106BB0001F2A8BBF344E4FF0A04602F01F0313462E
:106BC00001279F4003F5E073C6F80875032746F8D0
:106BD00023704B681F2B8BBF03F01F061E462A4FE6
:106BE0004FF0A04706F5E0764FF0000C47F826C0BE
:106BF000C4F80C25C4F814358B685E1C25D0CA680F
:106C0000511C22D01F2A8BBF1F4E4FF0A04602F00E
:106C10001F01114601278F4001F5E071C6F8087584
:106C20001F2B4FF0030746F821708BBF03F01F01A5
:106C30001946154E4FF0A04601F5E071002746F8C1
:106C40002170C4F80825C4F810352946FFF7FAFE6C
:106C50000246B8B90823C4F800354FF488712046BD
:106C600004F091F8A96805F10C03C4F8343589687B
:106C70000123C4F838352360C4F84415C4F8482506
:106C8000A360E3601046F8BD0003005030B50A4B26
:106C900005460FCB85B06C4684E80F000022012129
:106CA0002820FEF739FC2820FEF704FC2146284660
:106CB000FFF778FF05B030BDE0BC000030B50A4BEF
:106CC00005460FCB85B06C4684E80F0000220121F9
:106CD0000220FEF721FC0220FEF7ECFB21462846AD
:106CE000FFF760FF05B030BDF0BC0000084B03604B
:106CF000084B4360084B8360084BC360084B03613B
:106D0000084B4361084B0162C0E90632704700BF7F
:106D10008DAF0000F9AF0000DFAF0000C3AF00008F
:106D2000ABAF000099AF000093AF0000064B10B46A
:106D300002F100449C4203D9A02310BC04F0A7B97F
:106D40004FF4806010BC7047FEFFFF7F30B51546E2
:106D500085B00C4699B10268526A5269CDE9003299
:106D600021460DF10F032A4604F098FB28B99DF83F
:106D70000F3033B10CB12B68E05405B030BD024A7E
:106D8000ECE74FF00040F8E7B3B10000094B70B5F5
:106D900053F820400130002653F82050A54200D877
:106DA00070BD236820465B68984700B166600C346C
:106DB000F4E700BF6CC00000104B70B5104C0546E6
:106DC0001E469C4204D10E4CB44209D1002412E06C
:106DD00062681AB122681268AA420CD00C34F0E73B
:106DE00063680BB90C34EFE723682846196802F092
:106DF00040F90028F6D1204670BD00BFF089002080
:106E00003C8900200248034A0021121A02F07BB993
:106E1000000000207452002008B50648064A0749C1
:106E2000121A02F043F9064A06490748BDE808402D
:106E300002F03CB9B8870020108B0020D8C70000B2
:106E400000000000D8C700000000002008B50220A4
:106E5000FFF79CFF0320FFF799FF00F023FEF9F7EF
:106E60001FFB034A137B23F00103137308BD00BF0C
:106E7000B027002080B53F4BA2B083F308883E4C7A
:106E80003E4E636943F4007363610025E02384F898
:106E90002230E57725766576A576636A43F4E023AC
:106EA0006362FEF7FFFAFEF779FB4FF0FF33A36250
:106EB000E36207AB29466C22184602F024F9012749
:106EC000B06028468DF82970FFF760FF3846FFF75D
:106ED0005DFF2B4C00F080FC2A4B34624FF42052B3
:106EE000CDE90473CDE90255CDE90055264B27497C
:106EF000204600F08BFD637B23F0040213F01B0F90
:106F00006273354604D1A36913B9204600F09AFA9A
:106F10001F4B204E059301220F23CDE9033200239E
:106F20004FF4A0721C4900933046CDE901331B4B4E
:106F300000F06CFD737BEE6023F004037373184B59
:106F4000C5E90633FEF714FC0D48AC6002F081F889
:106F50000D4B144A184682F3098863B64FF00001BE
:106F600081F31188BFF36F8F00210022002301F00D
:106F700038FA00BFB883002000ED00E01C28002094
:106F8000B0270020B9C700004D6E000078520020E5
:106F9000BEC7000044270020787A002079BA00009C
:106FA00034280020787A002038B5074C074DAC42D1
:106FB00001D3002038BD04F114032046C4E9053391
:106FC00001F058F81C34F2E7F0890020288A0020EC
:106FD0002DE9F04F1D1E85B006460C46174659DDBB
:106FE00000F0C2FE80462C484FF4004C00214FF4C4
:106FF0007A320023CCFB0501F9F782F818EB000286
:10700000264B9046F31A264A9B1002FB03FA5FFABE
:107010008AFA06F1140B009403AB02AA39463046F3
:1070200001F073F810F10B0F0BD1009403AB02AA1F
:107030003946304601F069F810F10B0F08BF6FF0C8
:107040000B006379029A84F804A062F3030363716E
:107050006368039A62F31F336360C0B1BDB110F17E
:107060000C0F14D14FF02003EFF3118083F311883C
:10707000BFF36F8F2A46594600F0FAFA6B1CCAD04C
:1070800000F072FEB8EB0005C5D56FF00A0005B040
:10709000BDE8F08F0022B3E7FFE70300F08900208E
:1070A000B76DDBB670B5047802684178114EC4EB59
:1070B000C404A400120B01F00F01301901F0ECF828
:1070C0004FF02003EFF3118583F31188BFF36F8F27
:1070D00004F11400304404F03DFC28B12946064870
:1070E000BDE8704004F08DBB85F31188BFF36F8F4E
:1070F00070BD00BFF089002073520020034B9B68D5
:107100000146186E08B104F0BBBA70471C28002075
:1071100070B50D4634498B68DA7B013A0446DA7360
:10712000C26808464AB1A36889688B4212D09DB9EB
:1071300000F06CF96FF00F050AE08B6893F90E30E0
:10714000236101328368E260A36000F05FF90025EB
:10715000284670BD2369F3E791F90E1093F90E30BC
:107160009942A8BF194621EAE1714FF02003EFF3DD
:10717000118683F31188BFF36F8FA06890F90E30EA
:10718000994201DA00F0DAFA2B46224631461748D6
:1071900000F092FA054610B900F038F9D8E72368F4
:1071A00021699C4207D033B193F90E309942A8BFB0
:1071B000194621EAE1714FF02003EFF3118583F3C3
:1071C0001188BFF36F8FA06890F90E30994201D0FB
:1071D00000F0B4FA85F31188BFF36F8F00F016F951
:1071E0006FF00A05B4E700BF1C280020735200208E
:1071F0001E4B9A68D37B013B70B50446D373C368BA
:10720000012B05D0013BC360BDE8704000F0FEB823
:107210004FF02003EFF3118683F31188BFF36F8FD4
:107220000169806890F90E30994201D000F086FA29
:10723000204604F062FB0546A06080B1437BDB067C
:1072400003D183690BB900F0FDF886F31188BFF311
:107250006F8F0023AB6695F90E302361D4E7E060B1
:1072600086F31188BFF36F8FCEE700BF1C28002084
:1072700038B54FF02003EFF3118583F31188BFF386
:107280006F8F046884B12368426823F0030394423B
:10729000036008BF43600121204604F077FA85F3BC
:1072A0001188BFF36F8F38BD29B985F31188BFF3FB
:1072B0006F8F0846F7E700F108020B461046294693
:1072C00000F0FAF918B9034B9B685869EBE72046C0
:1072D000E9E700BF1C280020EFF305800D2809D83E
:1072E00028B1054B586880F40060C0F3C02080F0DE
:1072F000010070470120FAE700ED00E008B5FDF756
:10730000A7FA054B054A1B6818441061002118466E
:10731000BDE8084004F092BB502800201C28002043
:10732000F8B50D464FF02003EFF3118483F3118875
:10733000BFF36F8F0D4E0E4B4FF400410027C1FB82
:10734000006700221A6130464FF47A320023394632
:10735000F8F7D6FE074B1860074B1D60FFF7CEFF0E
:1073600084F31188BFF36F8FF8BD00BFFFE7030000
:107370001C280020502800204C2800204FF020031B
:10738000EFF3118183F31188BFF36F8F044B9A6879
:10739000D37B013BD37381F31188BFF36F8F7047A9
:1073A0001C280020094B03F12402824205D19B686E
:1073B0008B4202D14B7BDB0607D1D1E900231A6057
:1073C0000A6853600023C1E9003370471C2800207D
:1073D00038B50D4C024604F1240004F057FA054676
:1073E00000B9E568A3684AB95A7BD20606D1AA69F2
:1073F00022B9DA897F2A01D9236238BD9D4201D0A2
:10740000FFF77CFF2562F8E71C28002010B54FF03D
:107410002003EFF3118483F31188BFF36F8F084BC0
:107420009A68D37B0133D3730120FFF7D1FF84F334
:107430001188BFF36F8FBDE8104004F0FFB900BFA3
:107440001C280020F8B54FF02003EFF3118483F3DC
:107450001188BFF36F8F164A114651F8243F8B42B3
:107460000CD05BB1966A90F90E5093F90E70AF4252
:107470000BDCB34202D01B68002BF6D1936A436049
:10748000936A01601860906205E05A68C0E90032B2
:107490005A6810605860437B43F0400343730020F8
:1074A000FFF796FF84F31188BFF36F8FF8BD00BF1D
:1074B0001C280020F8B504464FF02003EFF3118696
:1074C00083F31188BFF36F8F194F07F1240501462D
:1074D0002846FFF767FF7B6AAB423A460CD05BB1A8
:1074E000B86A94F90E1093F90E708F420BDC834248
:1074F00002D01B68002BF6D1936A6360936A256003
:107500001C60946205E05968C4E9003159680C6058
:107510005C60637B906843F040036373031B5842D5
:107520005841FFF755FF86F31188BFF36F8FF8BD01
:107530001C2800201449154A8B6810B51468A34212
:1075400003D1BDE81040FFF7D9BE00241460104AF3
:107550001268BAB1DA897F2A14D80E4A93F90E401C
:10756000126894420EDB0C4A126893420AD09A6960
:1075700042B90A69824203DC1846FFF79BFFE0E745
:10758000121A0A6110BD00BF1C28002048280020E4
:10759000502800204C28002084C0000038B5044644
:1075A0004FF02003EFF3118583F31188BFF36F8F42
:1075B000437B5A0607D501460948FFF7F3FE637B74
:1075C00023F040036373074B9868031B58425841EC
:1075D000FFF7FEFE85F31188BFF36F8F38BD00BF44
:1075E000402800201C28002070B504460D46164691
:1075F000FFF7D4FF637B43F002036373EDB12B68A5
:10760000A5609D420CD05BB194F90E2093F90E1049
:1076100091420CDC69688B4202D01B68002BF5D1CB
:107620006B6863606B6825601C606C6005E05A687D
:10763000C4E900325A6814605C60731C12D00A48B6
:107640004FF4004500214FF47A32C5FB06010023B8
:10765000F8F756FD0549421C04F11800BDE87040DA
:1076600000F0E8BA70BD00BFFFE7030099B8000062
:1076700070B50F4D0F4C0646A868FFF7B5FFAB6815
:1076800023603046FDF774FD4FF02002EFF31183C5
:1076900082F31188BFF36F8F2268A968914204BFFB
:1076A0000022226083F31188BFF36F8F70BD00BF8B
:1076B0001C2800204828002010B50C461146064A18
:1076C0009068064A10601A46FFF78EFF2046BDE814
:1076D0001040FDF74DBD00BF1C28002048280020A9
:1076E000F8B5461C04F0C4F934184FF02003EFF34A
:1076F000118783F31188BFF36F8F0D4D0D4BA86871
:107700001860FFF74BFFA8680B493246183000F0AD
:1077100091FAAA68537B43F0100353733846FDF780
:1077200027FD04F0A5F9201A20EAE070F8BD00BF9B
:107730001C2800204828002099B800002DE9F843B3
:1077400004464FF02003EFF3118983F31188BFF350
:107750006F8F04F034F84EB28046002835D01D4DAE
:1077600005F1240721463846FFF71CFE6B6AA67315
:10777000BB422A460AD04BB1A96A93F90E00B04227
:107780000BDC994202D01B68002BF6D1936A636030
:10779000936A27601C60946205E05A68C4E900326D
:1077A0005A6814605C600120FFF712FE89F31188AB
:1077B000BFF36F8FB8F1000F09D0064B9B68DB7BDE
:1077C0002BB9BDE8F84304F039B8A673EEE7BDE87D
:1077D000F88300BF1C280020044B002103F1240281
:1077E000C3E909220846FFF79BBD00BF1C28002003
:1077F000F8B5224C224BA2681B689A4232D04FF057
:107800002003EFF3118683F31188BFF36F8F04F128
:107810002405A1682846FFF7C5FD636AA268AB424C
:107820000CD05BB1A16A92F90E0093F90E708742F9
:107830000BDC994202D01B68002BF6D1A36A53607F
:10784000A36A15601A60A26205E05968C2E90031B6
:1078500059680A605A600120FFF7BAFD86F3118863
:10786000BFF36F8F4FF02003EFF3118083F3118884
:10787000BFF36F8FBDE8F840FDF77ABC1C280020ED
:1078800084C0000038B50E4C4FF400410025C1FB08
:10789000004520464FF47A3200232946F8F730FCA1
:1078A000044648B9FFF7A4FF4FF47A7284FB022321
:1078B000D00940EA436038BDFFF712FF0446F3E702
:1078C000FFE70300014B9868704700BF1C280020A9
:1078D00070B504464FF02003EFF3118683F311884F
:1078E000BFF36F8F04F009F8054670B1437BDB06E8
:1078F00003D183690BB9FFF7A5FD0023AB663146C1
:107900000548BDE8704003F07CBFD4E902329A42DA
:1079100018BF0133A360F2E77352002010B402468F
:107920000B464FF02000EFF3118180F31188BFF375
:107930006F8F946844B1013C946081F31188BFF368
:107940006F8F002010BC704733B981F31188BFF3EB
:107950006F8F6FF00F00F5E7014810BCFFF7ACBE6A
:107960007352002010B5084C08494FF0FF334FF414
:107970008062204600F0F2F804F11000044904F09F
:107980000FF8002010BD00BF54280020B88300204D
:10799000C3C70000EFF305800D2807D838B1044BAA
:1079A000586880F40060C0F3C02070470120704721
:1079B00000ED00E0024B9B68187B00F0010070476F
:1079C0001C28002010B502464FF02003EFF311846D
:1079D00083F31188BFF36F8F437B590704D484F37B
:1079E0001188BFF36F8F10BD23F00403437303F0BE
:1079F000CCFF10B11046FFF725FD21460248BDE837
:107A0000104003F0FEBE00BF7352002030B587B0B7
:107A100004460E9D04950D9D03950C9D02950B9DAE
:107A200001950A9D0095FDF78FFD044B9B6813B9E6
:107A3000236607B030BD1B6EFAE700BF1C2800208C
:107A400070B586B0002605960E9E04960D9E039690
:107A50000C9E02960B9E0F9D01960A9E0096044670
:107A6000FFF7D4FF6B1C03D02DB92046FFF7AAFF08
:107A7000204606B070BD09484FF4004600214FF47F
:107A80007A320023C6FB0501F8F73AFB0449421C91
:107A900004F1180000F0CEF8EAE700BFFFE70300AA
:107AA00099B800002DE9F04F284E294D87B0B04617
:107AB000B54205F130040FD3FFF760FC244C254E8E
:107AC000DFF894A04FF400490027444521D307B0C4
:107AD000BDE8F04FFFF79ABC54F8043C059354F806
:107AE000103C049354F8143C039354F8183C02934C
:107AF00054F81C3C019354F8203C009354E90A23A9
:107B000054E90C01FFF782FF54F8303CDD64254650
:107B1000CEE7616A4B1C04D0256821B92846FFF7DF
:107B200051FF3034D1E7B346BC46C9FB01BC4FF42A
:107B30007A32002358466146F8F7E2FA5146421C71
:107B400005F1180000F076F8EBE700BFF08900209F
:107B5000F0890020FFE7030099B800002DE9F0410B
:107B6000054686B098460E46174605F1100403F008
:107B700019FE0020CDE90400CDE90208CDE900504E
:107B80003146064B3A462046FFF75AFF0449204645
:107B900006B0BDE8F04103F003BF00BFF78300006B
:107BA000CCC70000034B1B680BB9FCF751BE00208B
:107BB000704700BFD0280020036840B1084A5268CF
:107BC000904204D01BB19A6881680A449A60426866
:107BD000136003685A600023C0E90033704700BF98
:107BE0003489002038B5104B1B78002B0F4B1C68D4
:107BF00014BF4FF0FF306FF000409C420AD04CB1F0
:107C0000A568FFF7CFFF281A00280ADBA468FFF752
:107C1000C9FF201A064B1B6913B19842A8BF18462A
:107C200038BD0020F6E700BF7352002034890020E1
:107C30001C28002070B504461646C1604FF0200392
:107C4000EFF3118583F31188BFF36F8FFFF7AAFF5E
:107C5000194B1A68012EACBF801901309A42A060FE
:107C600001D05E6832B95A6862605A682360146055
:107C70005C600BE09068A168884216DD411A916053
:107C80005168C4E9002151680C6054601A689A4236
:107C900006D0944204D1FFF7A5FF0021FCF7A0FD18
:107CA00085F31188BFF36F8F70BD091A9642A160EA
:107CB000D9D01268D6E700BF348900202DE9F04BF7
:107CC0000446FFF737FC4FF02003EFF3118583F3F1
:107CD0001188BFF36F8F214E214FDFF888903460F9
:107CE000B846D9F8004032684C45D7E900BC05D009
:107CF00024B1A368934214DD9B1AA3601BEB02001E
:107D00004CEBE2710024C8E900013460FFF76AFF20
:107D10002146FCF765FD85F31188BFF36F8FBDE841
:107D2000F08B1BEB03004CEBE371D31A33600023A1
:107D3000C7E90001A3602046FFF73EFF85F31188E5
:107D4000BFF36F8FE36898474FF02003EFF311857F
:107D500083F31188BFF36F8FC3E700BFD0280020E3
:107D600000000020348900202DE918484FF020033E
:107D7000EFF3118483F31188BFF36F8FFCF768FD75
:107D8000074BD3E9002312EB000B43F1000C5846DC
:107D9000614684F31188BFF36F8FBDE8188800BF78
:107DA0000000002008B9086070476FF015007047A8
:107DB000FF20704738B515461C4601F030F858B919
:107DC0000346DAB2944201D8012004E0AA5CFF2AFB
:107DD00003F10103F5D038BD4FF0FF30FBE773B579
:107DE0000D461646F8F7B2FB6946C0B2FBF7C0FC79
:107DF00030B10124009801F011F8204602B070BDA6
:107E00002889E968042301440DEB0302009801F07E
:107E100006F804460028ECD1BDF8042046F6071306
:107E20009A4201BFEA68BDF806309B182A8906BF4E
:107E30009B1833600324DDE737B504460D46052063
:107E400001A900F06DF89DF80630012B02D1204603
:107E500000F075F82968204600F075F82046F9F71B
:107E600067F8002003B030BD73B58C680128084660
:107E70000CBF203C183C0D4601F03DF80646284654
:107E8000FFF796FF08220146684601F03CF90123FE
:107E90008DF800306A4633462146284600F0DCFF64
:107EA000003018BF012002B070BD4FF4C0735843BA
:107EB000283070470378052B03D0062B04D0022B03
:107EC00004D14FF4C07070470320704707207047FB
:107ED00010B5044601F00FF82378062B0BBF0323DF
:107EE0004FF4C0732022584308BF13FB0020A3683F
:107EF00018BF2830181A10BD13B50C46C0B201A91E
:107F0000FBF736FC50B921460198F8F783FF044689
:107F1000019800F083FF204602B010BD0124FAE76B
:107F2000062806D80123834013F0640F01D0FFF721
:107F3000E3BF0720704701460120FFF795BF0146C8
:107F40000020FFF791BF7FB5037885680191062B6C
:107F50000CBF203D283D044600F0CDFF06462046DC
:107F6000FFF726FF082201460DEB020001F0CBF8D7
:107F700004220DEB020102A801F098F8042E38BF8C
:107F80000426F3B202AA2946204600F065FF00301D
:107F900018BF012004B070BD2DE9F0419DF81840D4
:107FA000002C14BF02240024002567184FF0800C19
:107FB000AF421BD81846BDE8F08123465C008D42D5
:107FC000A4B208D290F800802CFA06FE18EA0E0F30
:107FD00018BF44F001041B0406F1010648BF5440D9
:107FE000082EEAD1013501302346E1E70026E5E716
:107FF00070B5C66890F90B000C254D43884206EB1E
:108000000504B4BF71592146202492FBF4F401EB1E
:108010008401196002F01F0070BD07B501ABFFF7C6
:10802000E7FF019A012303FA00F01368034313608A
:1080300003B05DF804FB07B501ABFFF7D9FF019A68
:10804000012303FA00F0136823EA0003136003B06E
:108050005DF804FB4FF02003EFF3118083F31188E8
:10806000BFF36F8F7047C30703D581F31188BFF348
:108070006F8F70472DE9F84304464368058900680F
:1080800094F80AC05D43FF222844E27200214FF0B9
:108090000C0E8C4505DC00252389AB4222DCBDE8B3
:1080A000F883D4F80C80B5FBF3F20EFB01F71F2A1E
:1080B00008EB0706C8BF1F324FEA930306F1040915
:1080C000C8BF520903F10303C6E9019923F0030372
:1080D000D4BFE17248F8070001F10101C8BF00EB0D
:1080E0008200D6E76268E36820686A4381181E1D33
:1080F00086509A684A609A682046116099602A46BC
:108100000021FFF78AFF0135C6E72DE9F04F8BB05C
:10811000857A00AFC7E90232AB000A3303F4FF638C
:10812000ADEB030D4368E94603334A4623F00303EE
:1081300042F8043904460020854200F1FF3A0ADD86
:1081400028B113689B08033323F00303536052F8EC
:10815000043F8B4208D2BAF1FF3F07D13A6D0023AA
:1081600013606FF00B0043E00130E5E7207C10F076
:10817000010001D0FFF76EFF0C2303FB0AF31A1D69
:10818000E3683862134456461D68AB427CD0D5E99B
:1081900000131960296859F826204B600023C5E9AF
:1081A000003323683146EB1A204693FBF2F2FFF7C7
:1081B00042FF731C7B62A9EB890309EB86067B6196
:1081C0007B6A013B9A4517DC396A207CFFF74BFF3D
:1081D0003B6D1D60002DC4D0FB68C3F800A0236870
:1081E000ED1A59F82A3095FBF3F5BB6800201D60A5
:1081F0002C37BD46BDE8F08F236856F8042BEB1AE8
:1082000093FBF2F37A699B003B6106EB4603134450
:10821000BB614FF0010BD6F80080796A0BFB08F3C5
:10822000FB61EB187B603B6920460BEB0302FFF719
:10823000F4FE7B682268218908F1FF389844A8EB96
:10824000020862684A4390450AD2E268B969F8694F
:108250000A44111D29509168596091680B60936020
:108260000BF1010BBBF1040FD5D1207C396AFFF76C
:10827000FAFE207C10F0010001D0FFF7EBFE7B6AD4
:10828000386201337B629BE7013E721CA5F10C034F
:108290007FF47AAF002597E72DE9F04F87B0837A16
:1082A0009B000A3303F4FF6300AFADEB030D43689B
:1082B000E946033323F003030546C9F800304C4672
:1082C0000120814214D2287C10F001000E46904615
:1082D00001D0FFF7BFFE0446002E12DA4FF0FF3444
:1082E0002146287CFFF7BFFE1C37BD46BDE8F08F56
:1082F00023689B08033323F0030344F8043F013051
:10830000DFE759F82630FB6003FB08FB2B68BB60F6
:1083100042463146284603EB0B0AFFF77EFEEA6829
:108320000C2303FB0622BB68111D43F80B10936856
:10833000CAF804309368C3F800A0C2F808A0287CEB
:108340002146FFF790FE287C10F0010001D0FFF7D6
:1083500081FE0446002EC3D007F114034246314685
:108360002846FFF745FE7A69042390FBF3F3106873
:108370009B00D84000F00F000F28B1D128F0030374
:10838000BB60FB68013B4FF0000A7B60BB68B5F83F
:1083900008C0696803EB0A02FB6803FB02FB7B6809
:1083A00001FB0CF103EB0B00884211D23146284649
:1083B000FFF741FE2A6802EB0B0152F80B004B68F5
:1083C000186052F80B004360002342F80B304B60FA
:1083D0000AF1010ABAF1040FD8D198FBFAF8013E6C
:1083E0007AE708B50446084611461A46A047FFF743
:1083F00069FAFDF751F910B504464FF0FF312046F8
:10840000FEF736FF03460028F7D008334268BFF373
:108410005B8F53E8001F21F0010C43E800CEBEF152
:10842000000FF6D1BFF35B8FCB0700D59047FFF766
:10843000DFF9E2E70020704770B504460D4645209D
:10844000A04729465220A047294623465220BDE88E
:10845000704018472DE9F04F89B01C464FF0000AD4
:10846000531E06460F4603934FF0FF39D0460025B2
:1084700005E06DB9252800F03D813946B047039BE2
:1084800013F8010F03930028F3D109B0BDE8F08F72
:10849000642862D019D839280AD8312851D22D2819
:1084A0003DD030283ED0252808D13946B047DEE7F8
:1084B000582800F0A880632800F01681394625204E
:1084C000B047039B39461878F0E7702800F0918098
:1084D00006D8692841D06C283CD06828CFD0EDE779
:1084E00075286DD017D87328E8D1256804F1040BDE
:1084F0002B461C4614F8010B002840F0EC80B8F124
:10850000030F40F000815C1BA9EB0404002C00F376
:10851000E6805C46ABE7782875D07A28DEE74FF036
:108520000308ACE7B9F1000F0EDAB8F1000F00F064
:10853000E780A0F13009B8F1000F08BF4FF0020842
:108540009DE7B9F1000FF4DB0A2303FB0909A9F148
:108550003009F0E70AF1010A91E7BAF1000F12D1F0
:1085600025680434002D05DA39462D20B0476D42C8
:1085700009F1FF39CDF8009043462A463946304686
:10858000F9F736F873E7BAF1010FE9D0073424F0B0
:10859000070303F10804D3E9002312F1004043F17B
:1085A00000014FF0000C4FF0FF3B8C4508BF8345A6
:1085B00004D239463046FFF73FFF58E71546D1E76A
:1085C000BAF1000F05D122680434CDF8009043467B
:1085D000D4E7BAF1010FF6D0073424F0070303F112
:1085E0000804D3E90023002B08BFB2F1004FECD3FD
:1085F000DFE739463020B04739467820B0474FF0A2
:1086000008094FF00108BAF1010F27DC236807932E
:10861000002304930434002310220293069393460C
:10862000079B0BF1FF3B4FEA8B00C0F1200CA0F140
:10863000200123FA00F0049B03FA0CFC40EA0C0032
:1086400023FA01F1084310F00F0013D1069B13B970
:10865000BBF1000F2ED14FF0300C11E0073424F0A5
:10866000070303F108041A685B6807920493D2E7D2
:10867000059AD5E709288CBF4FF0570C4FF0300C06
:10868000394660440592B047029B06950133029338
:10869000BBF1000FECD1B8F1030F7FF4E8AE029B01
:1086A000C3EB4905002D7FF7E2AE39462020B047E5
:1086B000013DF7E7531E91450593E9DBB8F1010F42
:1086C00003D139463020B047E2E7B8F1020FDFD1DD
:1086D00039462020F7E73946B047234609E73946AF
:1086E0002020B047013C11E72068251D3946B047DE
:1086F0002C46BCE6AA46A8464FF0FF390125BEE647
:108700004FF00108BBE65C460546B8E60FB407B576
:1087100004A951F8040B0191F8F7BAFF03B05DF812
:1087200004EB04B070470369D0E90020824296BF91
:108730009B1802F1FF3303F1FF33181A70470368E7
:1087400070B584680669A342A6EB040598BF9B191F
:10875000013BAA42A3EB040328BF2A46934228BF49
:108760001346426922441C44A64298BFA41B0A60D7
:108770008460184670BD10B50446FFF7D4FF8842E8
:1087800009D3636819442369994228BFC91AC4E907
:108790000111002010BD6FF01500FBE72DE9F3413A
:1087A00080460F4616460025324601A94046FFF78F
:1087B000C6FF394604460246019800F077FC361B96
:1087C0002544274401D0002CEED129464046FFF72E
:1087D000D2FF284602B0BDE8F08170B5D0E903367B
:1087E0004468A34296BFF51803F1FF3505F1FF3544
:1087F0002D1B741E641BF51AAA4228BF2A46A242EA
:1088000028BF224644691C4413449E4298BF9B1BC8
:108810000C60C360104670BD38B505690446FFF7AB
:1088200082FF6B1E181A884208D3236819448D42B0
:1088300098BF491B2160E160002038BD6FF0150032
:10884000FBE72DE9F34180460F46164600253246E8
:1088500001A94046FFF7C1FF019904460246384688
:1088600000F024FC361B2544274401D0002CEED117
:1088700029464046FFF7D0FF284602B0BDE8F08108
:108880007047F8F75DBF004713B502AC4FF0FF33F8
:1088900044F8043D00F0030000230444934202D155
:1088A000019802B010BDC85CE0540133F6E74FF008
:1088B00080531A695869504370474FF080531869C4
:1088C00070474FF080535869704700F1804000F5C1
:1088D0001C3001230360BFF36F8FBFF34F8F7047CE
:1088E00030B54C680D689C4229BFC0E90053002197
:1088F000E41AED1832BFC0E900514C600D6093429C
:1089000003D1201C18BF012030BD0020FCE74B68BC
:1089100010B59A420C6828BF1A46C0E90042981A5E
:108920000B684860134400300B6018BF012010BD75
:1089300030B54C680B68A24228BF2246002A14BFFB
:108940001D460025A4EB02041344C0E900524C600C
:108950000B6014BF0120002030BD10F0800F14BF49
:108960000023102300F00F0018447047704708B52B
:108970000146F9F739F8F9F729F8837B032B0AD177
:108980000846FFF7EAFF012303FA00F0C043BDE801
:108990000840F9F7A7B80368002BF1D008BD87207D
:1089A000FFF7E5BF8620FFF7E2BF8520FFF7DFBFB7
:1089B0008420FFF7DCBF8320FFF7D9BF8220FFF7B9
:1089C000D6BF8120FFF7D3BFF9F7C0B80720F9F76A
:1089D000CBBA0620F9F7C8BA0520F9F7C5BA0420C2
:1089E000F9F7C2BA0320F9F7BFBA0220F9F7BCBA07
:1089F0000120F9F7B9BA08B5F8F7E8FF818108BD99
:108A000008B5F8F7E3FF4FF02002EFF3118382F38C
:108A10001188BFF36F8F82680A6002682AB9807B71
:108A200083F31188BFF36F8F08BD0420F8E708B502
:108A3000F8F7BCFF58B9EFF3108272B64C20FFF77D
:108A400044FF4C20FFF741FF82F3108808BD4C2003
:108A5000BDE80840FFF739BF5020FFF736BF54206C
:108A6000FFF733BFF8B504460D4616461F463B4692
:108A7000324629462046FBF737FD10F10B0F02D195
:108A8000FEF7B6FEF3E7F8BD2DE9F34150F8283CB8
:108A900010F82C5C1033044610D1C36850F8202C19
:108AA00099073BD5FAB913F0040304D11A461946C5
:108AB0002846FFF7D7FF002344F8283C54F8283C09
:108AC00010330DD054F8186C56B154F81C7C54F87F
:108AD000148CFEF75FFF00284BD02046FAF7B2F85F
:108AE00002B0BDE8F08150F8241C01AB2846FFF726
:108AF000B9FF10B16FF01503DEE7019A54F8243C7A
:108B0000134444F8243C54F8203C9B1A44F8203C7D
:108B100054F81C3C134444F81C3CCFE750F8241C88
:108B200001AB2846FBF748FD0028E3D1019E54F82D
:108B3000243C334444F8243C54F8203C9B1B44F828
:108B4000203C54F81C3C334444F81C3C002EB2D06A
:108B50002846FBF7C7FDB6FBF0F303FB10600028C7
:108B6000A9D154F8203C002BA5D02846FBF768FD7E
:108B7000A4E744F8180CA4F11000FEF7A9FE54F87D
:108B8000283C4833ACD0424639462846B047A7E790
:108B900000207047006808B1043800B970470368C6
:108BA0001B689B688B42F9D04068F4E7006808B105
:108BB000043800B9704703681B689B685B689B7842
:108BC0008B42F7D04068F2E7006830B5A0B10438B6
:108BD000082488B103681B689A68136A127F14FB23
:108BE0000232934203D1406830B10438F1E70833D0
:108BF00013F8045C8D42F4D130BD8170817601316F
:108C0000C9B280F82510C176704750E90230184784
:108C10008368002283F826207047836893F8240035
:108C200070478368002283F827207047836893F891
:108C300025007047836893F8242012B193F826200A
:108C40002AB993F8250018B193F82700704701203E
:108C50007047012070478368C3E9011270470229F9
:108C6000836808D004290BD001290ED1D3F8B03085
:108C700013600020704793F8B730C3F34003F7E761
:108C800093F8B73003F00103F2E76FF0220070476A
:108C90006FF02200704710B58468D4F8A800FFF781
:108CA000D0FDD4F8A830D3E900329A4204BF0023A3
:108CB00084F8253010BD202908B583683BD009D839
:108CC00008291DD0102929D0012908D1C3F8B020C6
:108CD000002008BD802940D004D8402934D06FF04E
:108CE0001200F6E7B1F5807F40D0B1F5007FF6D1F4
:108CF00093F8B81001F0BF01AAB141F0400112E0B1
:108D000093F8B81001F0FE012AB983F8B8100121D8
:108D1000FAF72AFCDCE741F00101F6E793F8B81016
:108D200001F0FD0122B983F8B81093F8B810EFE70D
:108D300041F00201F7E793F8B81001F0FB01002AB7
:108D4000F1D041F00401EEE793F8B81001F0F7011B
:108D5000002AE8D041F00801E5E793F8B81001F0E7
:108D6000EF01002ADFD041F01001DCE793F8B810E2
:108D700001F0DF01002AD6D041F02001D3E780685E
:108D8000012380F8263043682BB190F8243013B1CA
:108D90000C30FAF73BBC70478068012380F827301D
:108DA00043682BB190F8253013B10C30FAF72EBC84
:108DB000704738B585682B78032B4FF000000BD136
:108DC00085F82400D5F8AC00FFF7E8FC044605F16F
:108DD0001800FAF71BFC204638BD4368DB681847CB
:108DE00070B502684C68A24216D38B6823449A423D
:108DF00006D2D1E90435AB4204D36FF00B038B618B
:108E000000200AE0CD68121B05EBC30645F83320AD
:108E10004268726001330B61012070BD70472DE91B
:108E2000F0411E4683688B4205460C4617460FD319
:108E3000721893420CD3C068FDF7BEFF436869689F
:108E40001D683A4633462144AC46BDE8F0416047D0
:108E50006FF01500BDE8F0812DE9F843984683686E
:108E60008B4207460E4691461CD308EB0102934203
:108E700018D3C068FDF7A0FF00210546FFF7ADFF3E
:108E8000044660B96B6879685C68314443464A4679
:108E90002846A047012104462846FFF79EFF2046AA
:108EA000BDE8F8836FF01504F9E783688B422DE97C
:108EB000F04107460E4690461AD30A44934217D310
:108EC000C068FDF779FF00210546FFF786FF0446DD
:108ED00058B979686B6831449B6842462846984780
:108EE000012104462846FFF778FF2046BDE8F081BF
:108EF0006FF01504F9E708B5C068FDF75DFF43683A
:108F0000187D08BD08B5002210460121FCF704FBBE
:108F10000020FCF7CFFA002008BD4FF080434FF44B
:108F2000607220B1C3F804230020FCF7C3BAC3F871
:108F3000082370470378027903F00F0322B9181C45
:108F400018BF012040427047082B07D8012A08D1DA
:108F5000B3F1080018BF4FF0FF3070474FF0FF30FB
:108F600070470020704770B504460E461546FBF763
:108F700023FB30B906B925B12046BDE87040FBF7A8
:108F80005FBB70BD7047704770B505460E4604461E
:108F9000631B9E4205DD14F8010BFBF7C7FC013093
:108FA000F6D170BD70B501230A24B1FBF3F2092A92
:108FB00006D8024600250A2623B91370101A70BD80
:108FC0006343F2E7B1FBF3F403FB1411B3FBF6F3D5
:108FD00015B90CB9002BEFD13034147001350132C2
:108FE000EAE738B5054608460C4600F03AF821464F
:108FF00002462846BDE8384002F0AFB82DE93048B7
:10900000C37CDA0704460D4611D502F089FA83467F
:109010008C46C5E900BCE37C9B0705D56FEA0B00D5
:109020006FEA0C01C5E900010020BDE83088B0F806
:1090300010B04FF0000CECE7FCF7BCBA014600683A
:10904000FCF7CCBA08B5FCF779FBBDE80840FCF7A3
:1090500075B807B5002101A8FCF734FC03B05DF832
:1090600004FB02460346981A13F8011B0029FAD1A3
:1090700070470138013910F8013F11F8012F934270
:1090800002D1002BF7D11A46981A704710B55AB181
:109090000139841810F8012B11F8013FA04201D0CA
:1090A0009A42F7D0D01A10BD1046FCE7F0B581EA1D
:1090B0000004A50703460BD0013B0A4491421DD191
:1090C000F0BD002AFCD011F8014B03F8014B013A26
:1090D0009C07F6D11D1F0C468F183E1B032E08D887
:1090E00094086FF0030505FB0422A40023442144E7
:1090F000E2E754F8046B45F8046FEEE711F8014B12
:1091000003F8014FDAE7F0B5C9B203469C070FD167
:1091100041EA012444EA04441D469F187E1B032EA5
:109120000CD8940803EB840413449C4209D1F0BD8D
:10913000002AFCD003F8011B013AE7E745F8044B8D
:10914000ECE704F8011BF0E700207047036830B536
:10915000CD1A002D02DC6FF05F0030BD1C7814F0DA
:10916000800F0AD15C1C04601B7813600368C91A65
:1091700013688B42EFD80020EFE704F07F04013C36
:10918000032C27D8DFE804F00209121E012DE2D0DB
:109190005C78146002330360E8E7022DDBDDB3F88E
:1091A000014064BAA4B214600333F4E7032DD2DDA6
:1091B0009C785D78240244EA0544DD782C431460F1
:1091C0000433E8E7042DC6DDD3F8014024BA146067
:1091D0000533E0E76FF06300BFE770B404680E1B6F
:1091E000002E07DD26789E4208D10134046070BC51
:1091F000FFF7ACBF6FF05F0070BC70476FF06100AD
:10920000FAE737B50223154601AA0446FFF7E5FF42
:1092100040B9019A2168284600F05DFB2368019A55
:109220001344236003B030BD0023F0B5161F1C4665
:10923000844203D102EB8402BBB9F0BDD6F804C06E
:10924000ACEB030546F8045F51F82470BD422CBF17
:109250004FF0000E4FF0010EED1B9C452CBF7346E6
:109260000EF1010335600134E2E71168C81A994232
:1092700042F8040B2CBF00230123DDE72DE9F04366
:1092800084460D4602F140044FF0000EBCF10F0F72
:1092900054F8408C05F1400504F1400400F2BB8015
:1092A0004FEA101C6FF00F0404FB0C0007284FEA74
:1092B0008C1C01EB0C0502EB0C0440F2938051F87E
:1092C0000C60A3FB06671EEB060E2CBF4FF00109D6
:1092D0004FF0000918EB0E0142F80C106E68B9440B
:1092E0002CBF01220022A3FB06674A44921966683C
:1092F0002CBF0121002192196260AE6801EB070CBE
:109300004FF0000128BF0121A3FB066761448919C2
:10931000A6682CBF012200228919A160EE6802EB29
:10932000070C4FF0000228BF0122A3FB066762442E
:109330009219E6682CBF012100219219E2602E6982
:1093400001EB070C4FF0000128BF0121A3FB0667CA
:109350006144891926692CBF0122002289192161E3
:109360006E6902EB070C4FF0000228BF0122A3FB3D
:1093700006676244921966692CBF01210021921987
:109380006261AE6901EB070C4FF0000128BF0121BB
:10939000A3FB066761448919A6692CBF012200223C
:1093A0008919A161EE6902EB070E4FF0000228BF98
:1093B0000122724405F1200CA3FB0667E5699219AE
:1093C0002CBF4FF0010E4FF0000E52190EEB0701AB
:1093D0004FF0000E28BF4FF0010EE2618E440838B6
:1093E00020346546800005EB000C2146654551F8A8
:1093F000042B40F09F810444236813EB0E034FF0CD
:10940000000228BF012244F8043B4FF0010E002A5D
:10941000F2D1BDE8F08355F8406CA3FB06671EEB64
:10942000060E2CBF4FF001094FF000091EEB080695
:1094300044F8806C55F83C6CB9442CBF4FF00108DF
:109440004FF00008A3FB0667C84418EB060854F861
:109450007C6C2CBF4FF0010E4FF0000E16EB08068F
:1094600044F87C6C55F8386C0EEB07094FF0000E91
:1094700028BF4FF0010EA3FB0667CE441EEB060E7D
:109480002CBF4FF001084FF0000808EB070954F813
:10949000787C17EB0E0744F8787C55F8346C4FF065
:1094A000000828BF4FF00108A3FB0667C84418EB6B
:1094B000060854F8746C2CBF4FF0010E4FF0000EEC
:1094C00016EB080644F8746C55F8306C0EEB07097F
:1094D0004FF0000E28BF4FF0010EA3FB0667CE44ED
:1094E0001EEB060E2CBF4FF001084FF0000808EBF2
:1094F000070954F8707C17EB0E0744F8707C55F898
:109500002C6C4FF0000828BF4FF00108A3FB066742
:10951000C84418EB060854F86C6C2CBF4FF0010ED1
:109520004FF0000E16EB080644F86C6C55F8286CEA
:109530000EEB07094FF0000E28BF4FF0010EA3FB02
:109540000667CE441EEB060E2CBF4FF001084FF00D
:10955000000808EB070954F8687C17EB0E0744F87D
:10956000687C55F8246C4FF0000828BF4FF00108C4
:10957000A3FB0667C84418EB060854F8646C2CBFBC
:109580004FF0010E4FF0000E16EB080644F8646C25
:1095900055F8206C0EEB07094FF0000E28BF4FF076
:1095A000010EA3FB0667CE441EEB060E2CBF4FF048
:1095B00001084FF0000808EB070954F8607C17EB2E
:1095C0000E0744F8607C55F81C6C4FF0000828BF6B
:1095D0004FF00108A3FB0667C84418EB060854F8CF
:1095E0005C6C2CBF4FF0010E4FF0000E16EB08061E
:1095F00044F85C6C55F8186C0EEB07094FF0000E40
:1096000028BF4FF0010EA3FB0667CE441EEB060EEB
:109610002CBF4FF001084FF0000808EB070954F881
:10962000587C17EB0E0744F8587C55F8146C4FF033
:10963000000828BF4FF00108A3FB0667C84418EBD9
:10964000060854F8546C2CBF4FF0010E4FF0000E7A
:1096500016EB080644F8546C55F8106C0EEB07092D
:109660004FF0000E28BF4FF0010EA3FB0667CE445B
:109670001EEB060E2CBF4FF001084FF0000808EB60
:10968000070954F8507C17EB0E0744F8507C55F846
:109690000C6C4FF0000828BF4FF00108A3FB0667D1
:1096A000C84418EB060854F84C6C2CBF4FF0010E60
:1096B0004FF0000E16EB080644F84C6C55F8086C99
:1096C0000EEB07094FF0000E28BF4FF0010EA3FB71
:1096D0000667CE441EEB060E2CBF4FF001084FF07C
:1096E000000808EB070954F8487C17EB0E0744F80C
:1096F000487C55F8046C4FF0000828BF4FF0010873
:10970000A3FB0667C84418EB060854F8446C2CBF4A
:109710004FF0010E4FF0000E16EB080677444FF0A5
:10972000000E28BF4FF0010E44F8446CACF1100C51
:10973000BE44ABE555F8046BA3FB06781EEB070EA1
:109740002CBF012600261EEB020246442CBF4FF020
:10975000010E4FF0000E41F8042CB64446E60023FB
:109760000122C0E900238360704710B5044668B148
:10977000806830B161688900FCF766FAA068FCF780
:1097800053FA00230122C4E90023A36010BD42F272
:109790001073994270B504460D4602D96FF00F0060
:1097A00070BD43688B4216D204212846FCF736FA76
:1097B00006460028F2D0A16859B162689200FFF70E
:1097C00075FC6168A0688900FCF73EFAA068FCF7A8
:1097D0002BFAC4E901560020E2E78842F8B50646B4
:1097E0000F4603D08D681DB9FFF7BFFF002011E0C1
:1097F0004C68013C1CB155F82430002BF9D072683C
:109800003B6833600134A24205D221463046FFF75F
:10981000BEFF40B1F8BDB068121B9200002100EB02
:109820008400FFF770FCA200B968B068FFF73EFC47
:10983000DCE770B50E4601210446FFF7A8FF054698
:1098400088B9626801469200A068FFF75CFCA368D3
:1098500086EAE672002EA2EBE6721A60B4BF4FF001
:10986000FF3301232360284670BD4368B1EB431FDB
:109870003FBF83684A0901F01F0153F822003ABF35
:10988000C84000F00100002070474368DBB18168E8
:109890005A1E9B007AB951F8221000204FF0004365
:1098A000194204D1013020284FEA5303F8D1C0EB0C
:1098B000421020307047C818043B50F8040C0028B0
:1098C000E9D1013AE6E71846704708B5FFF7DDFF32
:1098D0000730C00808BDF8B50F4612F0030118BFE5
:1098E0000121436801EB9205AB42044616461AD1AA
:1098F00000212046FFF79DFF10BBB91903469E4289
:109900001ED023F0030711F8012DD4F808C0DD00A4
:1099100005F0180502FA05F55CF807202A434CF813
:1099200007200133EBE7FFF720FF00230122C4E902
:109930000023A36029462046FFF729FF0028D7D03F
:10994000F8BDF8B5054608466C68A40094421CD2E0
:10995000121B8E180021FFF7D6FB3046224610441A
:1099600000239A4213D10020F8BD23F0030CAF6806
:1099700003F00301CE0057F80C10F14011F0FF0F77
:1099800011D10133A342F0D1E9E71346FAE723F0FE
:109990000306AF6803F00301CC00B959E14000F8B9
:1099A000011D0133DDE76FF00700DDE7F8B506467E
:1099B0000D464C0901F01F07FFF767FF7368284445
:1099C000B0EB431F0AD8ACB937B1A3000021C7F1EF
:1099D000200C7268A24225D800200AE010F01F0176
:1099E00018BF012101EB50113046FFF7D0FE0028CF
:1099F000E9D0F8BD736803F18042013A121B92006E
:109A0000A000A34207D89B000022043B191DDBD015
:109A1000B168CA50F9E7B1688D581144013B0D5047
:109A2000043AEEE7B568E85800FA07F20A43EA504C
:109A30000134043320FA0CF1CBE743684A0993421E
:109A4000F0B403D301F01F0104D191B30021F0BCA5
:109A5000FFF7EFBE8AB9D1B90020F0BC7047846827
:109A60009D1854F8255044F8235001334468A41A33
:109A70009C42F4D89A00002505E00023F6E78468AC
:109A80000133A550043244689C42F8D8E3E74368A8
:109A900000259A00C1F1200C043A002BDCD0876825
:109AA000BE5826FA01F42C43BC50013B06FA0CF5D3
:109AB000F2E7002BD0D00B46DCE770B543689A0084
:109AC00033B94A68940062B9181C18BF012016E027
:109AD00084681444043A54F8044C002CF1D1013B3E
:109AE000EEE78D682E19043C56F8046C0EB9013A65
:109AF000E9E793420DD80ED39A000BB9184670BD12
:109B0000043A81688C58A9588C4202D803D3013B8F
:109B1000F3E70120F3E74FF0FF30F0E72DE9F04FD6
:109B200085B0164603930E9B5A68736801339A42B8
:109B300081468B4653D30E9B986800284FD09200E5
:109B40000021FFF7E0FA0E9BD6F804A09B68009373
:109B5000DBF80430009D534528BF53460AF1010746
:109B60000193BF0000245445D9F808001BD1009B85
:109B7000391F0B443A461946FFF798FA31464846D2
:109B8000FFF79BFF0028B3BF0E9BD9F80820B168F0
:109B90009A68B8BFD9F808102046FFF745FB0020A7
:109BA00005B0BDE8F08FDBF8081050F824802A6873
:109BB0000B68019803FB0823039A534302932A4638
:109BC0004346FFF75BFB029BB1682A465046FFF70E
:109BD00055FB45F8048B0023EB510134C3E76FF0CC
:109BE0000300DDE770B543689A0023B94A68940022
:109BF00052B99BB924E084681444043A54F8044CE4
:109C0000002CF3D1013BF0E78D682E19043C56F887
:109C1000046C0EB9013AEBE7934202D90268104690
:109C200070BD096801D24A42F9E70268002A01DDE5
:109C3000002912DB002901DD002A10DB99000BB995
:109C40001A46ECE70439846866586C58A642E6D890
:109C500001D25242E3E7013BF1E70122DFE74FF097
:109C6000FF32DCE71FB581EAE173A3EBE173002962
:109C70000093B4BF4FF0FF330123019301A90123E7
:109C80000293CDF80CD0FFF7ADFF05B05DF804FBF3
:109C900090422DE9F04106460C46154602D0884216
:109CA00033D12C46D4F80480012333604FEA880373
:109CB000B8F1000F31D141463046FFF768FD074645
:109CC00040BBB368D4F808E0194604460546A845E9
:109CD0002DD103EB8503ECB17268AA4205F10108AE
:109CE00008D841463046FFF752FD002831D1B3680D
:109CF00003EB85031A6814194FF0000128BF0121F6
:109D000043F8044B45460C46E5E7FFF766FD07467A
:109D10000028C6D03846BDE8F081A2681A44043B4A
:109D200052F8042C002AC6D108F1FF38C0E70A68AF
:109D30005EF8250014194FF0000C28BF4FF0010CFD
:109D4000241841F8044B2CBF01240024644401353D
:109D5000BDE70746DEE7F0B50F4685B0064611467B
:109D600038461546FFF7A9FE00282FDB0023012205
:109D7000B542CDE90123039306D1294601A8FFF797
:109D80002CFD0446A0B901ADB7420AD16868A968A4
:109D900001233360830088B9B268FFF745FA0024D5
:109DA00006E039463046FFF718FD04460028EDD09E
:109DB00001A8FFF7DAFC204605B0F0BDCA18043B45
:109DC00052F8042C002AE7D10138E4E76FF00904C7
:109DD000F1E7F8B50C681368634305460F4616466D
:109DE00016D511463846FFF768FE002806DB3246D6
:109DF00039462846FFF7AFFF40B1F8BD3A46314635
:109E00002846FFF7A8FF0028F7D164422C60F4E74A
:109E1000FFF73EFFF0E7F8B50C6813686343002BCB
:109E200005460F46164616DD11463846FFF745FE35
:109E3000002806DB324639462846FFF78CFF40B142
:109E4000F8BD3A4631462846FFF785FF0028F7D18E
:109E500064422C60F4E7FFF71BFFF0E72DE9F047C1
:109E6000002386B0154688424FF0010280460E4618
:109E7000CDE90023CDE90232CDE9043305D16846AE
:109E8000FFF7ABFC044650BB6E46A84506D14146E1
:109E900003A8FFF7A2FC044608BB03ADD6F8049064
:109EA0004FEA8903B9F1000F23D16F68BB0057BB9C
:109EB00009EB07014046FFF76AFC044678B9014602
:109EC0004046FFF7B6FC044648B94FEA870AAAF1B4
:109ED000040A0FBB32682B685343C8F8003003A84C
:109EE000FFF743FC6846FFF740FC204606B0BDE89C
:109EF000F087B2681A44043B52F8042C002AD4D1EB
:109F000009F1FF39CEE7AA681A44043B52F8042C41
:109F1000002ACDD1013FCAE7AB68D8F8082053F832
:109F20000A30B16852444846FFF7A8F9013FCEE72E
:109F30001FB50123009201AACDE90133CDF80CD061
:109F4000FFF78CFF05B05DF804FB2DE9F04F99B0E9
:109F50000F4601900021184690460393FFF782FEBA
:109F6000002800F0A581002401250399179440469C
:109F7000CDE90954CDE90B45CDE90D44CDE90F54A8
:109F8000CDE91145CDE91344CDE91554FFF795FD11
:109F9000A04226DA019B2BB9DFB90024204619B074
:109FA000BDE8F08F21460198FFF743FC04460028E6
:109FB000F2D009A8FFF7D9FB0CA8FFF7D6FB0FA832
:109FC000FFF7D3FB12A8FFF7D0FB15A8FFF7CDFBD7
:109FD000E4E741463846FFF700FC04460028E8D194
:109FE000DBE7414609A8FFF7F8FB04460028E0D16B
:109FF0000CAE03993046FFF7F0FB04460028D8D199
:10A00000D8F804100C9502310FA80995FFF7BFFB93
:10A0100004460028CDD101460FA8FFF70AFC0446EC
:10A020000028C6D1022112A8FFF7B1FB0446002880
:10A03000BFD1032115A8FFF7AAFB04460028B8D119
:10A040003046FFF722FC00F01F001F2876D0C0F139
:10A050001F03194609A80293FFF7A8FC044600282D
:10A06000A7D102993046FFF7A1FC04460028A0D1F1
:10A070000A9DDDF834A005F1FF390AF1FF33A9EBA1
:10A08000030B00934FEA4B13194630460493FFF736
:10A090008DFC044600288CD14FEA8B0B314609A871
:10A0A000FFF7A0FD00284BDA04993046FFF7C5FC06
:10A0B000044600287FF47DAF009B9B0004930AF1C7
:10A0C0008043023B9B0007936FF0030303FB0AF3FB
:10A0D00005F18045013D0693CAEBCA63AD000593C7
:10A0E000009B99453BD8019B5BB10FA91846FFF730
:10A0F00074FB08BB039BD8F800201B685343019AEC
:10A100001360002F3FF455AF029909A8FFF795FCA3
:10A1100090B9D8F80030099309A93846FFF75DFBDC
:10A120000146002840F0C2803846FFF79BFD00281A
:10A130007FF43FAF01233B6004463AE7029497E780
:10A14000119951F80B20013241F80B2009A9324630
:10A150000846FFF760FE044600289FD029E70498D0
:10A160000B990E9A4B5912580698DDF844A0934269
:10A1700000EB0506A5F1040B7ED34FF0FF334AF840
:10A1800006305AF8063001334AF80630A5F1080ABD
:10A19000119A9359013B9351002112A8FFF749FBF3
:10A1A0000028C9D1009B0E9A002B7DD0079BD15867
:10A1B000149B1960049952585A60119B12A90846C1
:10A1C0009A59FFF7B5FE014600286FD115A8FFF791
:10A1D00030FB0028B0D10B9A179BB9F1010F18BFC3
:10A1E00052F80A00186052F80B10596052599A60E0
:10A1F00015A912A8FFF7F6FC0028C9DC119B0CA9D1
:10A200009A5912A8FFF794FE002895D1059B03EBFD
:10A21000090A4FEA4A1A514612A8FFF7C7FB00285D
:10A220008AD109A9084612AAFFF7F5FD01460028C0
:10A230003CD109A8FFF716FD002819DA0CA912A8CD
:10A24000FFF7CBFA00287FF477AF514612A8FFF74B
:10A25000ADFB00287FF470AF09A912AA0846FFF7EA
:10A26000B8FD00287FF468AF119A9359013B9351D0
:10A2700009F1FF39043D33E751F80BC08AB11946A3
:10A280000023184640EA0C00F5F78AFF00234FF040
:10A29000FF328B4208BF824200D210464AF80600C5
:10A2A0006FE74FF0FF30F9E7009981E70C4680E651
:10A2B0006FF00B0472E670B504460D46104600219F
:10A2C0001646FFF7CFFC002824DB2A4633462146FA
:10A2D0000020FFF73AFE054638B1284670BD3246E9
:10A2E00021462046FFF775FD90B900212046FFF773
:10A2F000B9FC0028F3DB31462046FFF773FC002849
:10A30000EBDB324621462046FFF785FD0028F2D0E0
:10A310000546E2E76FF00905DFE72DE9F04FADF202
:10A32000546D06460F461846002103921D46FFF75E
:10A3300099FC002840F31E82AB68D3F8008018F027
:10A34000010F00F0178200210398FFF78BFC002813
:10A35000C0F2108208F10204640004F008044444CE
:10A36000032104FB08F3C3F10203013903FB04F4E6
:10A37000F7D101234FF4C06214A8CDE90831CDE92B
:10A380000A13CDE90C11CDE90E311091FEF7BBFE99
:10A390000398FFF77AFAB0F5287F80F0DF80EF2886
:10A3A00000F2DF804F2800F2DF80182834BF4FF022
:10A3B000010B4FF0030B6B6803F101084146304677
:10A3C000FFF7E5F90346002840F05C81414617A8F5
:10A3D000FFF7DDF90346002840F054814FEA4801B9
:10A3E0000BA8FFF7D4F90346002840F04B813B68E7
:10A3F000049301330AD139460EA8FFF7EEF903465C
:10A40000002840F03F8101230E930EAFDDF878362F
:10A410001BB19B68002B40F0AA80012108A8FFF720
:10A4200008FA0346002840F02D81696808A88901D0
:10A43000FFF7BCFA0346002840F0248108A92A4609
:10A440000846FFF738FF0346002840F01B81DDF87F
:10A45000783623B10C2208A91846FEF727FE2946B4
:10A460003846FFF7BFFB0028C0F286802A463946EF
:10A4700017A8FFF720FF0346002840F0038164423D
:10A480000DF12C092346CDF800902A4608A917A8FB
:10A49000FFF744FB0346002840F0F48008A930464B
:10A4A000FFF79BF90346002840F0EC8007AB01273B
:10A4B0001393CDF8009023462A4611A930460797FA
:10A4C000CDE91177FFF72AFB0346002840F0DA8038
:10A4D000BB4556D1039B4FF000095B680293C84609
:10A4E000CA464F46BAF1000F40F0AD80029B002BE8
:10A4F00040F0A4804FF0010A0AFA0BFA0DF12C0982
:10A50000029B434540F00F81012307AA0793CDE941
:10A51000113313922346CDF800902A4611A93046F4
:10A52000FFF7FCFA0346002840F0AC80049A0132A1
:10A5300040F0A880039A5268002A00F0A380039A92
:10A5400092681268D20740F19D80049B33603246C6
:10A5500029463046FFF73DFC034693E04FF0060BDB
:10A5600029E74FF0050B26E74FF0040B23E70C22F9
:10A57000DDF8781608A870E7394617A8FFF72DF917
:10A5800079E70BF1FF33029307FA03F30593029B7C
:10A5900069680C279F4014AB03EB07080131404664
:10A5A000FFF7F5F8034600286CD117A94046FFF7DE
:10A5B00014F90346002865D182462346CDF8009061
:10A5C0002A4641464046FFF7A9FA0346002859D1DA
:10A5D000029B0AF1010A5345EFD8059B03F10108DC
:10A5E0000DF5CA634FF001091F4409FA0BF9A7F2F0
:10A5F000F4570DF12C0AC1457FF66CAF69683846F7
:10A600000131FFF7C4F8034600283BD1A7F10C0144
:10A610003846FFF7E2F80346A0BB23463846CDF89C
:10A6200000A02A4617A9FFF779FA0C37034648BB62
:10A6300008F10108DFE74FF0020953E7029B013BF5
:10A6400002934FF0200A039B029A9B6853F8223032
:10A650000AF1FF3A23FA0AF313F0010336D1B9F1F4
:10A66000000F3FF43FAFB9F1010F2FD10BAB0093B7
:10A670002A46234631463046FFF750FA0346002863
:10A680003FF430AF01220BF1FF3402FA04F402FA76
:10A690000BF50C26A542029364D817A8FFF765F8BE
:10A6A0000BA8FFF762F80EA8FFF75FF8DDF8782631
:10A6B000029B0AB1926822B908A80293FFF755F8E5
:10A6C000029B18460DF2546DBDE8F08F08F10108A9
:10A6D000ABEB08029340C34547EA0307ABD14FF009
:10A6E00000080BAB00932A46234631463046FFF75D
:10A6F00015FA03460028C5D108F10108C345F0D872
:10A700000BAB14A80C21009301FB070123462A463A
:10A710003046FFF703FA03460028B3D14FF0010992
:10A7200007468046DEE62346CDF800902A463146AD
:10A730003046FFF7F3F903460028A3D17F001AEA59
:10A74000070F03D1029B01330293D9E62346CDF8CC
:10A7500000902A4617A93046FFF7E0F90346002883
:10A76000F0D08FE714AB06FB0430FEF7FEFF013498
:10A77000029B8FE76FF00303A3E700207047704749
:10A7800070472DE9F843044691469846DDE908767E
:10A790000D4679B9B9F1000F15D1B8F1000F1AD1F2
:10A7A0000FBB46BB7DB304F10800FFF78EF8606075
:10A7B000002006E00830FFF710F80028EAD0A0F5E6
:10A7C0008140BDE8F883494604F12C00FFF705F805
:10A7D0000028E2D0F3E7414604F13800FEF7FDFF20
:10A7E0000028DDD0EBE7394604F12000FEF7F5FF45
:10A7F0000028D6D0E3E7314604F11400FEF7EDFF60
:10A800000028CFD0DBE72846DBE770B504460E46CC
:10A8100015460021AC22FEF776FCC4E9296570BD1F
:10A8200010B50446A0B38C30FEF79FFF04F19800EA
:10A83000FEF79BFF04F16800FEF797FF04F120008C
:10A84000FEF793FF04F13800FEF78FFF04F12C00B0
:10A85000FEF78BFF04F11400FEF787FF04F10800F8
:10A86000FEF783FF04F18000FEF77FFF04F1740020
:10A87000FEF77BFF04F15C00FEF777FF04F1500068
:10A88000FEF773FF04F14400BDE81040FEF76DBF12
:10A8900010BD6C220021FEF736BCFBF79BBA2DE9F8
:10A8A000F84305460E46144612B90020BDE8F88369
:10A8B000036803F03F07D318036022BF43680133E6
:10A8C0004360A7B1C7F14008424510D300F1280901
:10A8D000424609EB0700FEF7E9FB49462846FBF72D
:10A8E000CBFA0028E2D14644A4EB080407462644EC
:10A8F00005E02846FBF7C0FA0028D7D1403C3F2CA2
:10A90000A6EB0401F5D8002CCFD005F12800224693
:10A910003844FEF7CBFBC8E7FFF7C1BF036803F07D
:10A920003F035A1C034470B5382A0D4600F128062F
:10A930004FF08001044683F8281006EB020073D81C
:10A94000C2F138020021FEF7DEFBD4E900315A0FD4
:10A9500042EAC102110EDB0084F86010110C84F889
:10A96000611084F86320110A1A0E84F864201A0C0E
:10A9700084F865201A0A84F8621084F8662084F846
:10A98000673031462046FBF777FA00284BD1E37A4F
:10A990002B7063896B70A3681B0AAB70A368EB70A4
:10A9A000E37B2B71E3896B71E3681B0AAB71E3688E
:10A9B000EB71E37C2B72638A6B7223691B0AAB72A7
:10A9C0002369EB72E37D2B73E38A6B7363691B0A64
:10A9D000AB736369EB73E37E2B74638B6B74A36956
:10A9E0001B0AAB74A369EB74E37F2B75E38B6B7568
:10A9F000E3691B0AAB75E369EB7594F823302B769A
:10AA0000638C6B76236A1B0AAB76236AEB76A36EA4
:10AA10004BB994F827302B77E38C6B77636A1B0A6A
:10AA2000AB77636AEB7770BD0021C2F14002FEF79D
:10AA30006AFB31462046FBF71FFA0028F3D1014696
:10AA4000382230467FE7FFF769BF70B50E460168D0
:10AA5000154659B10C688B681D4203D04B682A46D5
:10AA60003046984714B121462468F4E770BD10B50C
:10AA700004688068A468C0692468012904D158402A
:10AA8000C4F80405002010BD003320FA02F04FF096
:10AA9000010118BF012300F001009140834214BF5F
:10AAA000C4F80815C4F80C15ECE770B504688068A4
:10AAB000A468C0692568D5F81465D5F81045D5F89F
:10AAC000045560406C403440604001291CBFD040B8
:10AAD00000F001001860002070BD8368186830B570
:10AAE00058B10024814213D108685CB95C681860D1
:10AAF000A14200D158600020086072B9002030BD2A
:10AB00002846EFE720605868814208BF5C60F2E7A2
:10AB100005680446002DF3D13AB11A680A605868F6
:10AB200019600028EAD15960E9E76FF01500E6E7FF
:10AB3000F8B5026883689768DC69D3E902120A40B5
:10AB4000D3E90510014322EA010239681B69D1F8F3
:10AB500010155C404C4022EA0404012500260AB985
:10AB60002046F8BD2A4209D03B7906F01F0000219B
:10AB700040EA4310FBF7FCFC22EA050201366D00B7
:10AB8000EDE7F8B5846803689D68D4E902321A409D
:10AB9000D4E905310B4322EA03020127002602B95A
:10ABA000F8BD174212D0E169236995F804C04B4003
:10ABB000F34013F0010F06F01F0014BF0221032120
:10ABC00040EA4C10FBF7D4FC22EA070201367F0072
:10ABD000E5E701292DE9F04118BFD4B287680646A0
:10ABE00012BF25461F2500244FF00108AC4202D9B0
:10ABF0000020BDE8F081FB6808FA04F223EA0203B2
:10AC0000FB6021463046FBF7CBFC0028F1D1013434
:10AC1000E4B2EBE701292DE9F04118BFD4B287680F
:10AC2000064612BF25461F2500244FF00108AC42FE
:10AC300002D90020BDE8F081FB6808FA04F2134352
:10AC4000FB6021463046FBF7ABFC0028F2D1013413
:10AC5000E4B2ECE738B504460D46FDF728FE844221
:10AC600009D2002C07DBA84205D32C4484428CBFB8
:10AC70000020012038BD0020FCE770B50D462846B5
:10AC8000194616461C46FFF7E5FF38B14CB122467F
:10AC900029463046FEF70AFA002070BD6FF0150015
:10ACA000FBE72046F9E72DE9F3411D4643680C46D2
:10ACB0001B696946164601AA9847DDE90021002371
:10ACC00001F1FF3818469E469C46B8F1FF3F02D17D
:10ACD0006FF0150018E01768CEB1516801FB07004E
:10ACE000A04208F1FF3817DD03B10092009B5B68BA
:10ACF0006B6076B1A4EB0E04B4FBF3F404FB03E346
:10AD000064442B60AC60002002B0BDE8F0813844A0
:10AD1000E6E7A4EB0C04F1E75368BC4403FB07EE41
:10AD200008320123D1E713460122FFF7BCBF2DE90A
:10AD3000F047436886B0894692461B6902AA01A97A
:10AD400098470024A0462646029BB34202D806B08C
:10AD5000BDE8F087019F07EBC60745467B68049373
:10AD60003A68A5EB08039A4202D80136A846EBE7F9
:10AD7000514603A803940595C8470028E7D0049BD3
:10AD800001351C44ECE70023435082B04358019343
:10AD9000019B02B0704783689B689A7B72B102681E
:10ADA00092681268D2F8201141B14FF48071C2F854
:10ADB00008130121D16000229A7370471A680AB102
:10ADC00058681047704782680B4692E8030083E892
:10ADD00003000020704703689B681B68D3F82401B8
:10ADE00018B1D3F88004C3F88004704702689268F1
:10ADF000126808B58368D2F8100150B11B7B0B7044
:10AE000010464FF48871FFF7BEFF01231360002046
:10AE100008BD4FF0FF30FBE713B5036802AC9B6839
:10AE200004F8011D1A684FF490711046FFF7ABFF4C
:10AE30000123C2F84445C2F848359360D2F8201186
:10AE40000029FBD0D36002B010BD03689B6870B5C9
:10AE50001C68D4F820310E46DBB18568AB689B894D
:10AE60004FF490719A422046A8BF1A46FFF78BFF15
:10AE70000023A9689342896807DB0123C4F84415BD
:10AE8000C4F84825A360104670BDF05CC854013377
:10AE9000EFE71A46F7E738B503689B681A68D2F8F7
:10AEA00010310C4653B185684FF488711046FFF796
:10AEB0006AFF2B7B23700120106038BD1846FCE729
:10AEC000036882689B6892681B68002191734FF445
:10AED0008072C3F80423704783689B6801229A73C9
:10AEE000704703689B681B68D3F8200118B1D3F83A
:10AEF0000403C0F30020704703689B681B68D3F805
:10AF00001001003018BF0120704703689B681B6860
:10AF10001022C3F80423704703689B681B68102243
:10AF2000C3F80823704703689B681B684FF40072DE
:10AF3000C3F80423704703689B681B684FF40072D2
:10AF4000C3F8082370470120704783689B68C3E9F2
:10AF50000012704708B503689B681968D1F804337C
:10AF6000DB05024605D4D1F8040310F0100006D129
:10AF700008BDFFF7B6FF0028F5D00120F8E710461E
:10AF8000FFF7BAFF003018BF0120F1E7036A585CF1
:10AF90007047006A0844704710B40C46016A2046A6
:10AFA000114410BC1A46FEF781B810B50C46016A70
:10AFB000204611441A46FEF769F8B0FA80F04009BD
:10AFC00010BD07B5036A082219446846FEF76EF8FB
:10AFD0000198009900BA09BA03B05DF804FB07B5FF
:10AFE000036A042219440DEB0200FEF75FF8019892
:10AFF00000BA03B05DF804FB07B5036A02221944E6
:10B000000DF10600FEF752F8BDF8060040BA80B216
:10B0100003B05DF804FBF0B51D4687B013BA1446C3
:10B020002ABACDE9002369460646082204A89DF8FD
:10B030003070FEF73BF8002D08BF182C0DF11701FA
:10B040000BD29DF817301F448DF81770306806AA90
:10B050000368521A984707B0F0BD002D08BFB4F539
:10B06000807F2CBF01230023002D08BFB4F5803F53
:10B0700006D3012D08BF002C2ABF02330133DBB2F7
:10B0800001229A40891A18373B440B70DEE77FB5DE
:10B09000446906684C61C4690E600CB1013CC4612E
:10B0A000551C03F02004501CCD610C620CD144F0FF
:10B0B00004040C6204A91F3301F8013D0122336826
:10B0C0003046984704B070BD0CB11544CD61009373
:10B0D00008460023FFF79FFFF4E773B51E46C369D8
:10B0E00004460D460BB1013BC361009200232A4682
:10B0F0002046FFF790FF206803682A46314602B0D9
:10B10000BDE87040184702230160C0E9073270476C
:10B1100037B51D46C36914460BB1013BC36100231B
:10B12000009322462B46FFF776FF03B030BDF7B5FC
:10B1300011461A46DB171E4682EA0605C26903F06D
:10B14000200381EA06040AB1013AC2610093224653
:10B150002B46FFF760FF03B0F0BD10B414460B465A
:10B160006022214610BCFFF7B8BF8023FFF78FBFD6
:10B170000A6A0B68520713B5036009D502A9FF22BA
:10B1800001F8012D18461C680122A04702B010BD2D
:10B19000CB69012B06D0002B40F2013008BF4FF4E1
:10B1A0004070F3E74369002B0CBF4FF000400020D4
:10B1B000ECE701207047F8B5FF2305688374416808
:10B1C000AB6A9942044602D140F20110F8BD686AA8
:10B1D0000368984700F01F03002200F0E007172BD8
:10B1E000A774E274E260238205D91B2B19D8A3F15E
:10B1F000180101228A406168AE6A0132761AB242B1
:10B20000E2D87809012826D14FF400726282172B08
:10B2100037D9182B44D1686A0368013198472082D6
:10B220002FE01F2B07D040F2051040F20313E02F50
:10B2300008BF1846CAE700F0C003402B08D0802B97
:10B2400006D0E02F40F2051008BF4FF48170BDE733
:10B250000423E37415E00728D9D1143B072B10D839
:10B26000DFE803F0040B0B0B110B09090020F52399
:10B270002082A374AAE70123E374686A03689847ED
:10B28000A0740020A2E7686A01310368984780B281
:10B290001F282082F5D8FF23A3744FF4837095E70D
:10B2A000192B02D1686A4368B7E7E37C43F00103D6
:10B2B000CFE738B585686B1C044609D0837CC02B6A
:10B2C00017D0013D8560A5B9FF238374002038BDE8
:10B2D000D0E900319A6A91420BD0586A03689847C6
:10B2E000FF2806D16368A574013363600023A3605F
:10B2F000ECE72046BDE83840FFF75DBFF8B50746EC
:10B30000406A0E460368096815469847316800F0A0
:10B310001F0001311728316005D8C0B20021C5E9EE
:10B3200000010020F8BD1B2824D8BB6A183801246E
:10B3300084405B1AA34220D3012C786A06D10368AB
:10B340009847C0B20021C5E900010CE0022C03D1EE
:10B350004368984780B2F5E7042C08D18368984782
:10B36000002328606B60306820443060D9E7C368F0
:10B370009847E8E740F20510D4E740F20110D1E722
:10B3800013B504466A46011D0068FFF7B7FFA37CAA
:10B3900003F0DF03402B01BF6368009A9B186360D2
:10B3A0002046FFF786FF02B010BDC368F7B504461C
:10B3B0000F46154693B1136003686168586A836944
:10B3C00098472A686368134463602A68E3689B1A95
:10B3D000E36000263860304603B0F0BDC37C9907B7
:10B3E00003F0040209D57AB900233B6020462B60A4
:10B3F000E360FFF75EFF0646EDE72AB1426843F0DF
:10B40000020301324260C37423686168586A0368AA
:10B4100098470346D4E90002816A8A4202D140F289
:10B420000116D8E7FF2B02D101326260DCE7A27C73
:10B4300023F01F0393422ED16A46211DFFF75EFFC2
:10B44000064610B100232B60C5E7DDE9002300218B
:10B450008B4208BF92422A6002D04FF48066BAE75E
:10B46000D4E900C1DCF82800401A9042D7D3DCF8B8
:10B470002400E26083692A4698472A686368134477
:10B4800063602A68E3689B1AE3603860E37C43F0FA
:10B490000203E3749FE74FF482769CE72DE9F04FB7
:10B4A00089B08146129D8B4617461E4605B903ADED
:10B4B000CC46BCE80F002C460FC4DCF800302360FB
:10B4C000012300243370A24602AA01A92846CDF820
:10B4D00008A0FFF76AFFD8B9019BFBB1029B14EBF0
:10B4E000030813D23278B2B13A68424513D36A687E
:10B4F000D9F800000BEB0401D21A406A139CA04754
:10B50000003018BF012030704446DDE74FF4806002
:10B5100009B0BDE8F08F86F800A0F5E73C60F7E7DA
:10B52000036870B50446586A616803689847D4E9AF
:10B53000003110F00105586A04D0C3680131BDE83C
:10B5400070401847836801319847294670BD5062A2
:10B55000C069C2E90A011A6000210122C3E901128F
:10B560001846FFF728BEF7B5064607460D460C46B7
:10B570000FCE0FC533682B60FB7C5B0713D54FF0F4
:10B58000FF33A3606368013363602046FFF713FE57
:10B59000B0F5817F1DD1636801336360FF23002014
:10B5A000A374A06015E06A46211D2068FFF7A6FE7F
:10B5B000DDE9002300218B4208BF9242A26004D142
:10B5C000002B08BFB2F1FF3F05D17B6863604FF4E9
:10B5D000806003B0F0BDA17CA02903D1002AF4DB78
:10B5E0005100A1601343D9D02046FFF7E4FDF0E7F6
:10B5F00030B5837C03F0DF02402A87B004460D4655
:10B6000007D0802B0FD0A02B0DD0FFF7B9FE07B0CD
:10B6100030BD06AA4FF0FF3342F8143D0021034627
:10B62000FBF794FBF3E7ADB101A92046FFF79BFFC1
:10B630000028ECD1013D039B2BB9029B636020469F
:10B64000FFF737FEE3E7294601A8FFF7D1FF0028FF
:10B65000F1D0DCE740F20140D9E783681BB14FF439
:10B660008061FFF7C5BF032070474FF0FF330B60C9
:10B6700000230A461946FBF769BB0430FBF712BDED
:10B6800013B504240A1904D200236946FBF7A0FC71
:10B6900010B1002002B010BD224601A90098FDF7AC
:10B6A00005FD00980430F5E710B10438FBF7FABC4B
:10B6B00070470023C0E90233C0E90000704738B585
:10B6C000437BDB0604460D4603D183690BB9FBF7C8
:10B6D000B9FE0023A366656138BD2DE9F843044631
:10B6E0000F469046994600F108054FF02003EFF30E
:10B6F000118683F31188BFF36F8F284600F0FDF8A1
:10B7000040B14146FFF7DBFF2846314600F079F8AB
:10B7100000200CE0B9F1000F1CD00820FBF7EEFC74
:10B7200038B986F31188BFF36F8F6FF00B00BDE857
:10B73000F8830123C0F804800360036803F0030268
:10B7400067B923681343036063682060002BDBD173
:10B750006060D9E7C8F800904046EEE73B6833F0F8
:10B7600003030BD10260626812B9C4E90000CBE7A1
:10B77000136803F0030303431360E9E71343036013
:10B780003B6803F0030318433860BDE710B5044677
:10B7900030B10268930703D0446809B1FFF784FF12
:10B7A000204610BD0023C0E9003300F10803C0E9C2
:10B7B000023370470A4600234168FFF78EBF437B80
:10B7C000DB0603BF8069B0FA80F0400900207047B3
:10B7D00038B504464FF02003EFF3118583F3118849
:10B7E000BFF36F8F01468068FBF7DCFD637B23F0BE
:10B7F0000203637385F31188BFF36F8F0023A36087
:10B8000038BD08B5FBF768FD20B10846BDE8084023
:10B81000F9F7AEBC81F31188BFF36F8F08BD08B58F
:10B820000246FBF759FD20B11046BDE80840F9F784
:10B830009FBC82F31188BFF36F8F08BD4FF02003C8
:10B84000EFF3118083F31188BFF36F8FFFF7E7BF2A
:10B8500038B504464FF02003EFF3118583F31188C8
:10B86000BFF36F8F01468068FBF79CFD637B23F07D
:10B870000203637385F31188BFF36F8F0023A36006
:10B8800004F11800BDE8384000F0B2B803689842EF
:10B8900014BF18460020704750F8103C70B504469D
:10B8A000A0F11805CBB14FF02003EFF3118683F31D
:10B8B0001188BFF36F8F294650F8100CFBF772FD0B
:10B8C00014F80B3C23F0020304F80B3C86F31188B8
:10B8D000BFF36F8F002344F8103C14F80B3C23F0A7
:10B8E000140304F80B3C2846FFF769FF20B12846F3
:10B8F000BDE87040FBF7A6BD70BD38B54FF0200322
:10B90000EFF3118283F31188BFF36F8FFFF7BEFF50
:10B91000044682F31188BFF36F8FC8B14FF0200344
:10B92000EFF3118583F31188BFF36F8F01468068B1
:10B93000FBF738FD637B23F00203637385F3118803
:10B94000BFF36F8F0023A36004F1180000F050F8DC
:10B95000204638BD70B5064600253468A64200D0A2
:10B960000CB9284670BD2046FFF772FF2046FFF74E
:10B9700026FF01250028F0D02046FBF763FDECE709
:10B98000C0E90212C0E900007047437BDB0603BF39
:10B990008069B0FA80F0400900207047F5F7B6BE24
:10B9A0007047036D10B5044603B198472046FFF772
:10B9B000ECFF38B12046FBF7F1FD637B43F0080351
:10B9C000637310BD637B9B0702D52046FFF700FF22
:10B9D000A369002BF1D004F1180000F009F8ECE79E
:10B9E0000373002342738173C373C0E90633704746
:10B9F00010B54FF02002EFF3118482F31188BFF3EA
:10BA00006F8F03683BB1FCF7D7F8002084F31188EF
:10BA1000BFF36F8F10BD6FF01500F7E710B54FF053
:10BA20002003EFF3118483F31188BFF36F8FFCF7CA
:10BA3000D9F884F31188BFF36F8F10BD70B5044639
:10BA40000E464FF02003EFF3118583F31188BFF307
:10BA50006F8FFCF7C7F8A04205DD012803DD3146F2
:10BA60002046F8F7BDFE85F31188BFF36F8F70BDD8
:10BA700008B5FCF779F908BD08B54FF02002EFF3DF
:10BA8000118382F31188BFF36F8FFFF7C7FF012186
:10BA90000228D8BF0846FFF7D1FFF9F785FDECE78C
:10BAA0007047FFFF2C47FF7F0100000000000000EF
:10BAB000F93900000000000039900000848900205E
:10BAC00097AD000000000000399000000000000069
:10BAD00039900000000000003990000000000000D4
:10BAE0000D68000000000000399000000000000018
:10BAF00039900000000000003990000000000000B4
:10BB000039900000000000003990000000000000A3
:10BB10003990000000000000399000000000000093
:10BB20003990000000000000399000000000000083
:10BB300039900000000000000947000000000000EC
:10BB40003990000000000000399000000000000063
:10BB50003990000000000000399000000000000053
:10BB60003990000000000000399000000000000043
:10BB70003990000000000000399000000000000033
:10BB80003990000000000000399000000000000023
:10BB90003990000000000000399000000000000013
:10BBA0003990000000000000399000000000000003
:10BBB00039900000000000003990000000000000F3
:10BBC00039900000000000003990000000000000E3
:10BBD00039900000000000003990000000000000D3
:10BBE00039900000FD25000087880000788900203A
:10BBF00097AD000000000000399000000000000038
:10BC000039900000000000003990000000000000A2
:10BC10003990000000000000399000000000000092
:10BC200039900000000000003990000034C400008A
:10BC3000B11600000000000034C4000061320000B2
:10BC400000000000E4C20000B9350000EC8A0020CA
:10BC500017C30000058F00000000000021C3000092
:10BC6000058F0000000000002BC3000055470000B6
:10BC70000000000034C40000215800000000000053
:10BC800034C400004991000000000000BFC0000063
:10BC900041650000E8BF0000A4C700004165000046
:10BCA000E0BF0000ACC00000F16800000000000030
:10BCB000ABC700008D6C000064C00000B2C700007C
:10BCC000BD6C00005CC0000034C40000A96F00001F
:10BCD0000000000034C4000065790000000000008E
:10BCE00019000000200000001300000016000000F2
:10BCF0000F0000000B000000140000001500000001
:10BD000000C2010000000806090000000000000059
:10BD10000338FDD87047000045490000898F0000B6
:10BD20000200000005000000060000000100000005
:10BD3000F0C000004CBD00000800000077C295F381
:10BD400060D2EF7F3552500F2CB679800E01000083
:10BD50000200000058BD000000000000BEC200004C
:10BD60002600020200000020C6C2000022000B11C3
:10BD7000FD1900006D890000C9890000C389000019
:10BD8000BD890000B7890000B1890000AB890000BF
:10BD9000A58900009F8900000D1C0000291C0000DF
:10BDA000B9230000F1890000EB890000E58900005B
:10BDB000DF890000D9890000D3890000CD89000007
:10BDC000091B0000A11A0000791C00008D2500004D
:10BDD000011F0000918C0000E1360000000000000F
:10BDE0000000000000000000B38D0000978C0000F0
:10BDF0007F8D0000118C00001B8C0000998D0000CD
:10BE0000238C0000000000002D8C000000000000CA
:10BE100000000000358C0000538C0000578C00009F
:10BE2000B78C00005F8C00000000000000000000E4
:10BE300000200100ACC00000010000000020010053
:10BE400000020000ACC00000020000000020010061
:10BE500000600600ACC000000300000000220100EA
:10BE6000005E0600ACC000000400000000220100DB
:10BE7000005E0600ACC00000050000000080070066
:10BE800000600600ACC000000600000000E00D00ED
:10BE900000E00100ACC000000700000000C00F007F
:10BEA00000400000ACC0000008000000493900005C
:10BEB000000000000000000085380000113800007C
:10BEC00000000000982F8A4291443771CFFBC0B523
:10BED000A5DBB5E95BC25639F111F159A4823F9255
:10BEE000D55E1CAB98AA07D8015B8312BE853124AE
:10BEF000C37D0C55745DBE72FEB1DE80A706DC9B6F
:10BF000074F19BC1C1699BE48647BEEFC69DC10F1A
:10BF1000CCA10C246F2CE92DAA84744ADCA9B05C56
:10BF2000DA88F97652513E986DC631A8C82703B019
:10BF3000C77F59BFF30BE0C64791A7D55163CA0627
:10BF400067292914850AB72738211B2EFC6D2C4D33
:10BF5000130D385354730A65BB0A6A762EC9C28121
:10BF6000852C7292A1E8BFA24B661AA8708B4BC2B7
:10BF7000A3516CC719E892D1240699D685350EF4E1
:10BF800070A06A1016C1A419086C371E4C77482798
:10BF9000B5BCB034B30C1C394AAAD84E4FCA9C5B0E
:10BFA000F36F2E68EE828F746F63A5781478C8845F
:10BFB0000802C78CFAFFBE90EB6C50A4F7A3F9BE41
:10BFC000F27871C6E56600006FAA0000ABAA000017
:10BFD000DBAA000015AC0000D3AB0000000000009D
:10BFE00000000050000000000003005001000000AD
:10BFF0007BAC00009169000021690000D568000059
:10C00000E168000001000000EDAD000019AE000085
:10C01000D7AD0000456A0000C7AD00004BAE000080
:10C0200097AE0000C1AE0000D9AE0000E3AE000044
:10C030000BAF000019AF0000E3AE0000F9AE000046
:10C0400027AF000037AF000055AF000047AF00003A
:10C050004BAF000000000000000000000020004086
:10C060000100000000800240010000003C89002027
:10C07000908900209C890020D8890020F089002028
:10C08000F5FFFFFF4427002008010C0110011401F7
:10C0900018011C01200124012C0130013401380158
:10C0A0003C014001440148014C0150014E52465FA1
:10C0B000464C4153485F4452565F4E414D45004700
:10C0C00050494F5F310001040100010403020401E3
:10C0D0000401030403020401040304020401040133
:10C0E0000403010303040104000000000000000039
:10C0F0003082010A0282010100D106081A18442C7C
:10C1000018E8FBFDF70DA34F1FBBEE5EF9AAD24B5B
:10C1100018D35AE96D188019F9F09C341BCBF3BC85
:10C1200074DB42E78C7F10537E435E0D572C44D165
:10C1300067080F0DBB5CEEECB399DFE04D840BAAF2
:10C14000774160ED152849A701B43C10E6698C2FB2
:10C150005FAC414D9E5C14DFF2F8CF3D1E6FE75B94
:10C16000BAB4A9C8887E473C94C37767544BAA8D5C
:10C170003835CA62617EB7E115DB7773D4BE7B7256
:10C1800021896924FBF8656E643EC80ED785D55CAD
:10C190004AE4530D2FFFB7FDF31339833FA3AED20B
:10C1A0000FA76A9DF9FEB8CEFA2ABEAFB8E0FA82B0
:10C1B0003754F43EE12BD0D3085818F65E4CC888AB
:10C1C0008131AD5FB08217F28A692723F3AB873ED6
:10C1D000931A1DFEE8F81A246659F81CABDCCE68E9
:10C1E0001B666435ECFA0D119DAF5C3AA7D167C6AA
:10C1F00047EFB14B2C62E1D1C902030100017F7FFF
:10C200007F7F7F7F7F7F7F7F7F7F7F7F7F7F7F7F3E
:10C210007F7F7F7F7F7F7F7F7F7F7F7F7F7F7F7F2E
:10C220007F7F7F7F7F7F7F7F7F3E7F7F7F3F343534
:10C23000363738393A3B3C3D7F7F7F407F7F7F00F8
:10C240000102030405060708090A0B0C0D0E0F1066
:10C250001112131415161718197F7F7F7F7F7F1A0D
:10C260001B1C1D1E1F202122232425262728292AA6
:10C270002B2C2D2E2F303132337F7F7F7F7F414219
:10C28000434445464748494A4B4C4D4E4F50515206
:10C29000535455565758595A6162636465666768C6
:10C2A000696A6B6C6D6E6F70717273747576777886
:10C2B000797A303132333435363738392B2F464C92
:10C2C0004153485F30005352414D5F300002030438
:10C2D00005060708090B0C0D0E0F10111213143070
:10C2E0002E3031004344435F41434D5F300046618F
:10C2F000696C656420746F207265626F6F743A2098
:10C300007370696E6E696E6720656E646C657373B9
:10C310006C792E2E2E0A00434C4F434B5F33324B29
:10C3200000434C4F434B5F31364D007379735F636D
:10C330006C6F636B00696D6167657300736C6F741C
:10C340000076657273696F6E000A0D006461746136
:10C35000006F6666006C656E007263002A2A2A2AE6
:10C360002A20425553204641554C54202A2A2A2A35
:10C370002A0A002020537461636B696E672065721E
:10C38000726F720A002020507265636973652064C1
:10C3900061746120627573206572726F720A002089
:10C3A000204246415220416464726573733A2030E2
:10C3B0007825780A002020496D707265636973657D
:10C3C000206461746120627573206572726F720AF5
:10C3D000002020496E737472756374696F6E2062F9
:10C3E0007573206572726F720A002A2A2A2A2A201F
:10C3F0004D5055204641554C54202A2A2A2A2A0AB3
:10C40000002020537461636B696E67206572726FE0
:10C41000722028636F6E7465787420617265612084
:10C420006D69676874206265206E6F742076616C38
:10C430006964290A002020556E737461636B696E0C
:10C4400067206572726F720A002020446174612057
:10C450004163636573732056696F6C6174696F6EB5
:10C460000A0020204D4D464152204164647265739C
:10C47000733A20307825780A002020496E73747250
:10C48000756374696F6E20416363657373205669C9
:10C490006F6C6174696F6E0A002020466C6F617466
:10C4A000696E672D706F696E74206C617A79207384
:10C4B0007461746520707265736572766174696FFA
:10C4C0006E206572726F720A002A2A2A2A2A205563
:10C4D00053414745204641554C54202A2A2A2A2AAE
:10C4E0000A0020204469766973696F6E20627920A2
:10C4F0007A65726F0A002020556E616C69676E65FF
:10C5000064206D656D6F7279206163636573730A72
:10C510000020204E6F20636F70726F636573736FBE
:10C520007220696E737472756374696F6E730A003A
:10C530002020496C6C6567616C206C6F6164206FB2
:10C5400066204558435F52455455524E20696E74DB
:10C550006F2050430A002020496C6C6567616C2095
:10C56000757365206F662074686520455053520AC4
:10C57000002020417474656D707420746F2065789C
:10C58000656375746520756E646566696E656420A3
:10C59000696E737472756374696F6E0A00526573A5
:10C5A000657276656420457863657074696F6E2086
:10C5B000280053707572696F757320696E746572A7
:10C5C00072757074202849525120002A2A2A2A2A7A
:10C5D0002048415244204641554C54202A2A2A2AB8
:10C5E0002A0A002020427573206661756C74206FE2
:10C5F0006E20766563746F72207461626C65207260
:10C600006561640A0020204661756C74206573635F
:10C61000616C6174696F6E20287365652062656C5A
:10C620006F77290A002A2A2A2A2A20446562756718
:10C63000206D6F6E69746F722065786365707469C0
:10C640006F6E20286E6F7420696D706C656D656EFD
:10C6500074656429202A2A2A2A2A0A002A2A2A2AD0
:10C660002A20257320256429202A2A2A2A2A0A001A
:10C670002A2A2A2A2A204861726477617265206515
:10C680007863657074696F6E202A2A2A2A2A0A0044
:10C690002A2A2A2A204B65726E656C20416C6C6FC9
:10C6A000636174696F6E204661696C7572652120E3
:10C6B0002A2A2A2A0A002A2A2A2A2A204B65726E46
:10C6C000656C204F4F505321202A2A2A2A2A0A001B
:10C6D0002A2A2A2A2A204B65726E656C2050616EC8
:10C6E000696321202A2A2A2A2A0A002A2A2A2A2099
:10C6F000556E6B6E6F776E20466174616C2045726B
:10C70000726F7220256421202A2A2A2A0A00437582
:10C710007272656E74207468726561642049442089
:10C720003D2025700A4661756C74696E6720696EDC
:10C73000737472756374696F6E206164647265737B
:10C7400073203D20307825780A00495352006573E4
:10C7500073656E7469616C2074687265616400460B
:10C760006174616C206661756C7420696E2025733C
:10C7700021205370696E6E696E672E2E2E0A004658
:10C780006174616C206661756C7420696E207468D8
:10C7900072656164202570212041626F7274696E38
:10C7A000672E0A004750494F5F3000554152545F91
:10C7B0003100554152545F30006D61696E0069640B
:10C7C0006C6500737973776F726B7100776F726B42
:10C7D0007175657565000000358400000090D00318
:10C7E0000B0000000000000000000000000000003E
:10C7F0000000000000000000000000000000000039
:10C800000000000000000000000000000000000028
:10C810000000000000000000000000000000000018
:10C820000000000000000000000000000000000008
:10C8300000000000000000000000000000000000F8
:10C8400000000000000000000000000000000000E8
:10C8500000000000000000000000000000000000D8
:10C8600000000000000000000000000000000000C8
:10C8700000000000000000000000000000000000B8
:10C8800000000000000000009C880020B888002004
:10C8900000C20100000008000000000000000000CD
:10C8A00000000000B934000080000000092F0000E3
:10C8B00000000000092F00008000000000000000C0
:10C8C0000000000000000000000000000004000064
:10C8D000DA45002000000000000000000000000019
:10C8E000000000000000000000040000DA49002001
:10C8F0000000000028BE0000654A000000000000A3
:10C90000FFFFFFFF7BA700007FA7000081A70000BB
:10C9100007910000000000000000000033520020DA
:10C920002000000000000000000000005352002022
:10C930002000000000C2010000010300F488002074
:10C940000000000040420F000001030004890020A5
:10C950000000000034890020348900202CBC000035
:10C960000000000000000000C8BC00000000000043
:10C970000000000074BC0000000000000000000087
:10C9800050BC0000ACBE0000000000005CBC000019
:10C99000B8BE000000000000B0BC000008C00000ED
:10C9A00024890020BCBC000008C0000014890020BD
:10C9B00068BC0000000000000000000080BC000017
:10C9C000000000000000000098BC0000C4BF000090
:10C9D000EC2600208CBC0000C4BF00000C27002007
:10C9E000D4BC00000000000000000000A4BC000057
:10C9F000F0BF00000000000044BC0000D4BD0000F7
:10CA0000C087002038BC00000000000000000000CB
:10CA10003C10002000040000030003006C1F0020F5
:10CA20000100000000000000000000005C1C00206D
:10CA30001800000020000100901F002001000000ED
:10CA40000000000000000000288A0020288A002042
:10CA500000000000000000000F00000000000000C7
:10CA600000000000448A0020448A002012010002D5
:10CA70000000004015190F521100010203010902C4
:10CA80000000000100E03209040000010202000081
:10CA900005240010010524010201042402020524DA
:10CAA0000600010705800310000A09040100020ABC
:10CAB000000000070580024000000705000240005A
:10CAC00000040309042A034E6F72646963205365EE
:10CAD0006D69636F6E647563746F720000000000AF
:10CAE0000000000000000000000000000000001036
:10CAF000034D4355424F4F54000000000000000A10
:10CB000003302E3031000000000000FF0000000064
:10CB1000678A0020FB8B0000893600006934000022
:10CB200000000000000000000300000084880020D6
:020000040001F9
:102000003DB8F396000000000002000028AC00007C
:1020100000000000000000000000000000000000C0
:1020200000000000000000000000000000000000B0
:1020300000000000000000000000000000000000A0
:102040000000000000000000000000000000000090
:102050000000000000000000000000000000000080
:102060000000000000000000000000000000000070
:102070000000000000000000000000000000000060
:102080000000000000000000000000000000000050
:102090000000000000000000000000000000000040
:1020A0000000000000000000000000000000000030
:1020B0000000000000000000000000000000000020
:1020C0000000000000000000000000000000000010
:1020D0000000000000000000000000000000000000
:1020E00000000000000000000000000000000000F0
:1020F00000000000000000000000000000000000E0
:1021000000000000000000000000000000000000CF
:1021100000000000000000000000000000000000BF
:1021200000000000000000000000000000000000AF
:10213000000000000000000000000000000000009F
:10214000000000000000000000000000000000008F
:10215000000000000000000000000000000000007F
:10216000000000000000000000000000000000006F
:10217000000000000000000000000000000000005F
:10218000000000000000000000000000000000004F
:10219000000000000000000000000000000000003F
:1021A000000000000000000000000000000000002F
:1021B000000000000000000000000000000000001F
:1021C000000000000000000000000000000000000F
:1021D00000000000000000000000000000000000FF
:1021E00000000000000000000000000000000000EF
:1021F00000000000000000000000000000000000DF
:1022000058E700207174010085AA0100FD720100E9
:10221000FD720100FD720100FD720100FD720100FE
:10222000FD720100FD720100FD720100416F0100AD
:10223000FD720100FD720100E96E010067AA010054
:1022400031740100317401003174010031740100F6
:1022500031740100317401003174010031740100E6
:1022600031740100317401003174010031740100D6
:1022700031740100317401003174010031740100C6
:1022800031740100317401003174010031740100B6
:1022900031740100317401003174010031740100A6
:1022A0003174010031740100317401003174010096
:1022B0003174010031740100317401003174010086
:1022C0003174010031740100317401003174010076
:1022D0003174010031740100317401003174010066
:1022E0003174010031740100317401003174010056
:1022F0003174010031740100317401003174010046
:102300007BB972B90029BEBF00204FF0004106E042
:1023100008BF00281CBF6FF000414FF0FF3000F0F5
:10232000A5B9ADF1080C6DE904CE002909DB002B3D
:102330001ADB00F035F8DDF804E0DDE9022304B033
:102340007047404261EB4101002B1BDB00F028F895
:10235000DDF804E0DDE9022304B0404261EB410115
:10236000524263EB43037047524263EB430300F076
:1023700017F8DDF804E0DDE9022304B0404261EB28
:1023800041017047524263EB430300F009F8DDF866
:1023900004E0DDE9022304B0524263EB43037047DB
:1023A0002DE9F047089E04468846002B4BD18A420F
:1023B000154667D9B2FA82F24AB1C2F1200701FA92
:1023C00002F320FA07F7954047EA030894404FEAE2
:1023D000154E230CB8FBFEF71FFA85FC0EFB178881
:1023E00043EA084307FB0CF1994209D9EB1807F1BE
:1023F000FF3080F01B81994240F21881023F2B444C
:102400005B1AA4B2B3FBFEF00EFB103344EA0344A4
:1024100000FB0CFCA44509D92C1900F1FF3380F016
:102420000781A44540F2048102382C4440EA074069
:10243000A4EB0C0400271EB1D4400023C6E90043DE
:102440003946BDE8F0878B4209D9002E00F0EB80B9
:102450000027C6E9000138463946BDE8F087B3FADF
:1024600083F7002F47D18B4202D3824200F2FA80D9
:10247000841A61EB030301209846002EE0D0C6E9E0
:102480000048DDE702B9FFDEB2FA82F2002A40F02E
:102490008F80491B4FEA154E1FFA85F80127B1FBC3
:1024A000FEFC230C0EFB1C1143EA014308FB0CF15C
:1024B000994207D9EB180CF1FF3002D2994200F291
:1024C000CD808446591AA3B2B1FBFEF00EFB101466
:1024D00043EA044408FB00F8A04507D92C1900F191
:1024E000FF3302D2A04500F2B6801846A4EB0804E0
:1024F00040EA0C409FE7C7F1200CBB4022FA0CFEDB
:102500004EEA030E01FA07F420FA0CF521FA0CF357
:102510004FEA1E482543B3FBF8F92C0C08FB19338E
:102520001FFA8EFA44EA034309FB0AF49C4202FABA
:1025300007F200FA07F10BD91EEB030309F1FF3094
:1025400080F087809C4240F28480A9F102097344A4
:102550001B1BADB2B3FBF8F008FB103345EA034494
:1025600000FB0AFAA24508D91EEB040400F1FF3370
:102570006BD2A24569D90238744440EA0940A0FBF5
:102580000289A4EB0A044C45C2464B4654D351D0B1
:10259000002E69D0B1EB0A0564EB030404FA0CFCCD
:1025A000FD40FC404CEA0505C6E90054002747E71A
:1025B000C2F1200320FA03F7954001FA02F021FA54
:1025C00003F34FEA154E3843010CB3FBFEF71FFA35
:1025D00085F80EFB173341EA034107FB08F38B42F2
:1025E00004FA02F407D9691807F1FF3C2FD28B4295
:1025F0002DD9023F2944CB1A81B2B3FBFEF00EFB6A
:10260000103341EA034100FB08F38B4207D96918F4
:1026100000F1FF3C17D28B4215D902382944C91A60
:1026200040EA07473BE73746304609E70746E7E613
:102630001846FBE64145ABD2B8EB020A69EB0E0245
:1026400001381346A4E76046E9E7184695E7674670
:10265000D1E781467CE702382C4447E7ACF1020C15
:102660002B442FE7384608E73746E9E6704700BFB6
:1026700043680A461BB19B6C0BB101491847704770
:10268000852601002DE9F347D0E9004663685B6CBD
:1026900005460BB120469847002706F10C086368F1
:1026A0005B6B3BBB63685B6AFBB120469847E0B15C
:1026B0000021A86808F0C4FD0746002872D1204612
:1026C00007F061F811E0384807F014FC374807F0CC
:1026D00011FC4946A86808F0B3FD63689B6923B103
:1026E00001220DF107012046984702B0BDE8F087AE
:1026F00018461DE0204698470028D3D0D5F824A0DE
:10270000BAF1000F08D1402006F04CF9814668620A
:102710000028D8D0A0F83EA0696ACA8F131D1944BA
:1027200063689B69C2F13A02002BE1D020469847CA
:10273000696ACB8F184480B2C8870028AFD03A2886
:1027400008D00844C2780D2AA9D842F20143D340E8
:10275000DB07A4D5B06808F06EFD404606F004FD26
:102760006F629CE75B69311D3944921BC3B12046FF
:102770009847304486B2FA8F6368B242F2D86368F1
:102780001B6B1BB1204698470028F8D0AB681B682C
:1027900013B9204606F0F7FF384608F0DCFCA4E742
:1027A0001846E6E70026E6E7F5BC010018BD010083
:1027B00013B54FF08052094CD2F8A830D2F8A420BB
:1027C00000929BB243F44043054A0D2104F10900F5
:1027D00000F052F9204602B010BD00BF4C17012096
:1027E0002FBD01002DE9F04F6C4897B005F0A4FE15
:1027F000074628B96A4807F07DFB17B0BDE8F08F9F
:10280000684805F099FE80460028F3D0664805F038
:1028100093FE814610B9654807F06CFB644805F0EB
:102820008BFE054610B9634807F064FB624C634BAE
:10283000A36004F150036360614B236304F17803E8
:10284000E362604B2760C4E915435F4BC4F88030F6
:10285000012204F12803002104F10C0004F1340BDF
:10286000E367019304F15C0AC4F82880C4F850902F
:10287000A56708F037FE01220021584608F032FE15
:1028800004F1840601220021504608F02BFE0122AB
:102890000021304608F026FEC82006F019FC4B48FF
:1028A00008F032FE21463846FFF7E2FE019B404623
:1028B0001946FFF7DDFE04F150014846FFF7D8FE48
:1028C00004F178012846FFF7D3FE384606F060FF92
:1028D000404606F05DFF484606F05AFF284606F0DF
:1028E00057FF3B4807F006FB4C22002102A808F0E6
:1028F00049F9022304F10C028DF8153006928DF887
:102900002930CDF82CB08DF83D30CDF840A08DF8B1
:102910005130159604214FF0FF3202A806F094FEC4
:1029200001460028F6D1059B03F4F832B2F5005FAA
:1029300009D160F310332748059306F041FC38466F
:1029400006F01CFFE6E70A9B03F4F832B2F5005FDD
:1029500007D160F3103358460A9306F031FC404625
:10296000EEE70F9B03F4F832B2F5005F07D160F396
:10297000103350460F9306F023FC4846E0E7149BC3
:1029800003F4F832B2F5005FC4D160F3103330467F
:10299000149306F015FC2846D2E700BF58BC01008E
:1029A00062BC01007CBC010086BC01008DBC010042
:1029B000A1BC0100A8BC010074000020FC1801208B
:1029C0000C190120DC180120EC18012040420F00F6
:1029D000BCBC0100800000202DE9F04F85B09B4673
:1029E0000E9CDFF890A0012CB8BF0124012B0CBF76
:1029F0003023202315468046894601940293012600
:102A00000A2700220AF101040AB9AA451FD2B5FB20
:102A1000F4F049463030C04701360122013F012F12
:102A2000B5FBF4F14FF00A0304FB1155BAFBF3FABE
:102A3000E8D1494605F13000C047BBF1030F03D18F
:102A4000019B9C1B002C0FDC05B0BDE8F08F019BA7
:102A5000BB42E3DBBBF1020FE0D849460298039288
:102A60000136C047039AD9E749462020C047013CB8
:102A7000E8E700BFFFC99A3B0CB430B585B008AB9E
:102A8000CDE9010153F8042B00930446002501A968
:102A90000648039507F0D2F8DDE902309842B8BF46
:102AA000255405B0BDE8304002B07047179C0100C6
:102AB00030B585B0CDE901010446002501A90548DE
:102AC000039507F0BBF8DDE902309842B8BF255402
:102AD00005B030BD179C01004FF02003EFF31182C9
:102AE00083F31188BFF36F8F06490123C1F8403586
:102AF0004FF08041C1F8783582F31188BFF36F8FB2
:102B00000020704700E0014020B1034B800143F0FA
:102B100001031847704700BF40BA0100054B1B680E
:102B2000082B01BF044B1868B0FA80F0400918BFA9
:102B300000207047300100103401001008B54FF03C
:102B400080430022C3F80C21C3F81021C3F83825B4
:102B50004FF0805203F54043D2F80414C3F8201517
:102B6000D2F80814C3F82415D2F80C14C3F82815A9
:102B7000D2F81014C3F82C15D2F81414C3F8301579
:102B8000D2F81814C3F83415D2F81C14C3F8401541
:102B9000D2F82014C3F84415D2F82414C3F8481509
:102BA000D2F82814C3F84C15D2F82C14C3F85015D9
:102BB000D2F83014C3F85415D2F83414C3F86015A1
:102BC000D2F83814C3F86415D2F83C14C3F8681569
:102BD000D2F84014C3F86C15D2F84424C3F8702519
:102BE000FFF79CFF10B1164B164A1A60FFF796FFCD
:102BF00018B1154BFB22C3F81825FFF78FFF48B11A
:102C00001249134B0A681B6822F00F0203F00F03EE
:102C100013430B60FFF782FF18B10E4B4FF40072A5
:102C20001A604FF08043D3F80024D20744BF6FF0FE
:102C30000102C3F80024084B084A1A6008BD00BF0F
:102C40008C5600404881030000F00040E40E004034
:102C50005802001040960240D41401200090D00386
:102C6000044A91689368CB1A23F07F438342F9D3D7
:102C7000704700BF10E000E0034B044A1B68B3FB41
:102C8000F2F35843FFF7ECBFD414012040420F0089
:102C9000064A10F0800F00F00F0314BFD2F81005A1
:102CA000D2F81405D84000F00100704700700240CF
:102CB000054B1B68082B05D1044B1868003018BF62
:102CC00001207047002070473001001034010010CF
:102CD000054B10F0800FA3F1900208BF134600F0DF
:102CE0000F0003EB0010704784020020024A00230B
:102CF0001360024A137070471C7C02405D5B002029
:102D000007B5084A00231370074A019302A81370FD
:102D1000012300F8043D054B1B68984703B05DF89C
:102D200004FB00BF5C5B00205F5B002014030020FD
:102D3000F8B54D680B4F954228BF15460C46064620
:102D40002A460968384607F0F0FE60682368401B91
:102D5000C6E9007560601D440030256018BF012081
:102D6000F8BD00BF1C030020F8B54C68944228BF92
:102D7000144606460D468CB1094F0968224638466E
:102D800007F0D3FE37606B6874601B1B6B602B68A9
:102D9000201C23442B6018BF0120F8BD0460F2E71B
:102DA0001C03002007B500238DF804300B4BD3F82B
:102DB0002025ADF80620D3F8C034094A002B13684B
:102DC0000CBF4FF480714FF001210B431360054B92
:102DD00001A81B68984703B05DF804FB007002402F
:102DE000F001002014030020074BBFF35B8F024665
:102DF00053E8000F00EA020143E8001CBCF1000F99
:102E0000F6D1BFF35B8F70478001002013B5FFF749
:102E10006DFF0D4B93F88E20032A12D0D3F880401B
:102E20007CB96FF08070FFF7DFFF06238DF8043068
:102E300008238DF80630054B8DF807401B6801A864
:102E4000984702B010BD00BFF40100201403002019
:102E500008B5FFF74BFF084B93F89E20032A05D1D6
:102E60006FF00100BDE80840FFF7BEBFD3F8903017
:102E7000002BF5D008BD00BFF4010020012273B57E
:102E800002FA01F51E491F4E0B6810F0800F43EA4D
:102E9000050304460B6027D000F00F021A4B33F8ED
:102EA000123003F1804303F51C331A684AB1002243
:102EB0001A60BFF36F8FBFF34F8F802811D007F0D8
:102EC00029F9316829400AD106238DF804308DF89C
:102ED00006408DF807100D4B01A81B68984702B0FB
:102EE00070BDFFF7B5FFECE733681D42F7D106234D
:102EF0008DF804308DF806008DF80720EBE700BF51
:102F0000F00100208001002034BC010014030020E7
:102F100008B5054B1A78104607F0F2F8BDE80840EE
:102F200001461046FFF7AABF5F5B002013B5FFF70D
:102F3000DDFE104B93F81E21032A05D16FF480703B
:102F4000FFF752FF02B010BDD3F81041002CF9D1A9
:102F50006FF48070FFF748FF06238DF80430882354
:102F60008DF80630044B8DF807401B6801A8984780
:102F7000E8E700BFF401002014030020204B13B544
:102F8000D3F80044C3F80044BFF36F8FBFF34F8FF3
:102F9000BFF36F8FBFF34F8FE1050BD5194B0122A4
:102FA0001A7002A800230193022300F8043D164B77
:102FB0001B689847A2050AD5124A002302A801936C
:102FC0001370032300F8043D0F4B1B6898476305FB
:102FD00013D50C4B1A7882B100221A70084B0121CC
:102FE000C3F80815582007F043F802A804230192FB
:102FF00000F8043D044B1B68984702B010BD00BFA9
:10300000007002405C5B0020140300202DE9F04FAB
:10301000724B87B01A780193002A40F08280DFF863
:10302000C4B16F4B18686F4B1C68204079D010F00A
:10303000012479D094FAA4F4B4FA84F40F2C86BF56
:10304000A4F110085FFA88F844F080084046FFF7C2
:103050003FFE4FFA88FABAF1000F064608F00F0556
:10306000828966DAD0E9003104A8984700B9306057
:103070005D4B82221A60019B059A01201870A040C6
:10308000B368DBF80040134424EA0000BAF1000FF3
:10309000CBF80000B3600498544B77DA072D9BBF40
:1030A000142101FB0533C3F8A006C3F800068CBF4A
:1030B000C3F8A426C3F80426FFF7FAFDAB002DB22F
:1030C0006E004B4A4B49002871D1BAF1000FB5BFD1
:1030D00092468A4604242824B244474F474E1C4453
:1030E00005463560BFF36F8FBFF34F8F204606F064
:1030F000BFFF0220FFF7C0FD3368002BF1D01E2078
:10310000FFF7BAFD3B689B064FD50120FFF7B4FDE2
:10311000BAF8003003F1804303F51C331B68002B21
:10312000DFD007B0BDE8F08F90FAA0F0B0FA80F4DD
:1031300084E7072D2D4B24D9D3F8C09419F4803F90
:1031400018BF4FF000094B467168376804A8B847AC
:10315000049B002B8AD0059B4B4587D2012002257A
:10316000A040B573C043FFF73FFE06238DF80C3037
:10317000234B8DF80E808DF80F501B6803A89847DD
:103180004FE705F5947153F82190DCE7072D9BBFBD
:10319000142101FB0533C3F8A007C3F800078CBF57
:1031A000C3F8A427C3F8042786E70220A8E7BAF1EA
:1031B000000FACBF28200420184406F059FF12EA83
:1031C0002A0A38BF8A463AF8153003F1804303F5DE
:1031D0001C331A68002AFCD0A3E700BF5D5B002007
:1031E00080010020F00100201C7C024000700240A1
:1031F00034BC010046BC01007474024004710240FA
:103200001403002038B5174BD3F86C44C3F86C4452
:10321000BFF36F8FBFF34F8FFFF74AFD38B9124AE4
:10322000136823F0011103F001130C43136001250F
:103230001CB9BDE83840FFF7E9BE94FAA4F3B3FA2D
:1032400083F30F2BD9B2C8BFA1F1100005FA03F325
:10325000CCBFC0B241F0800024EA0304FFF70EFEA9
:10326000E6E700BF007002401803002037B50446AF
:10327000FFF73CFDFFF72CFD837B032B0CD1204691
:1032800006F03EFF012303FA00F0C043FFF7ACFD58
:10329000FFF7BCFE03B030BD0568002DF8D1204615
:1032A00006F02EFF012303FA00F0C043FFF79CFD58
:1032B00006238DF80430044B8DF806408DF8075036
:1032C0001B6801A89847E3E714030020024A002383
:1032D0001360024A13707047140300205E5B0020E5
:1032E00038B5514B4FF40062C3F80024BFF36F8F21
:1032F000BFF34F8FFFF7DCFC4C49A8B14FF0200320
:10330000EFF3118483F31188BFF36F8F0868484B84
:10331000032200287ED149F2753008601A600860E7
:1033200084F31188BFF36F8F4FF02003EFF3118404
:1033300083F31188BFF36F8F08683E4AC0230028CB
:103340006AD149F2753008601360086084F311880F
:10335000BFF36F8F344B0120C3F80005BFF36F8FAD
:10336000BFF34F8FD3F800040005FBD54FF4006086
:10337000C3F80004BFF36F8FBFF34F8F4FF02003EC
:10338000EFF3118483F31188BFF36F8F086800286F
:1033900044D149F275330B6010600B6084F31188DF
:1033A000BFF36F8F244B40F2E3721A600433402264
:1033B0001A60BFF36F8FBFF34F8FA3F6040300248F
:1033C0008022C3F81C25C3F830451C4B40F2FF1285
:1033D0001A601B4B1C60FFF789FC1A4B1C701A4BC0
:1033E00002221A70FFF764FC98B14FF02003EFF34C
:1033F000118583F31188BFF36F8F08680C4B80B978
:1034000049F275320A6018600A6085F31188BFF3CB
:103410006F8F38BD1A6083E7136097E7002313604E
:10342000BCE71C60F1E700BF0070024000EC064002
:1034300014ED064014EC064000780240F001002034
:10344000800100205F5B00205E5B00200E4B0022AD
:1034500010B51A70A8B9FFF72BFC0C4B0C4A0028CA
:103460000CBF184610460B4CC4F80403272003F089
:10347000C5FE0123C4F80435BFF36F8FBFF34F8F30
:1034800010BD0248EFE700BF5C5B00200714E001BD
:103490000714C00100700240034B1878012894BF44
:1034A00000200120704700BF5E5B00201B4B70B501
:1034B0001C7884BB1A4A106001221A70264664F0F8
:1034C0007F05082CEDB20CBF4FF400714021284657
:1034D00006F064FE2846FFF7FBFB0134092C8673D7
:1034E00006608660EBD1002440212546204606F088
:1034F00055FE2046FFF7ECFB0134E4B2092C85733E
:103500000560856001D1074870BD082C0CBF4FF4E1
:1035100000714021EAE70448F6E700BF5E5B002047
:10352000140300200000AD0B0500AD0B2DE9F8439E
:10353000074606F0E5FD4FF02003EFF3118583F316
:103540001188BFF36F8F17F00F0903D1274B1B783A
:10355000BB4246D1264A274B12681C68D24301263B
:1035600092B286402243324298463CD13846FFF719
:10357000AFFB0C233A06844603FB09F32DD51E4A04
:103580000868134400F060408A68B0F1005F02F000
:1035900001021DD1D2B9194ACCF8002007C983E82D
:1035A0000700CCF804300023CCF808308CF80E303B
:1035B000134B144834438022C8F80040C3F8042158
:1035C00085F31188BFF36F8FBDE8F8830E4AE3E7F8
:1035D0000AB90E4AE0E70E4ADEE70E4A13440E4AE5
:1035E000DAE70E48ECE70E48EAE700BF5F5B002031
:1035F000F00100208001002084010020B5A001001E
:1036000000E100E00000AD0BD7A00100312D01006A
:10361000692D01001401002087A001000A00AD0BF4
:103620000B00AD0B044B40F48070C3F81805BFF3DA
:103630006F8FBFF34F8F70470070024000F00F0391
:10364000072B11D810F0800F084A0BBF03F58873C1
:1036500003F5847302EB830352F8230008BF586814
:10366000431E584258417047002070470070024086
:1036700010B508220021044607F084FA0E4BD3F857
:1036800080242270D3F884246270D3F88824D3F87D
:103690008C1442EA01226280D3F89024D3F8941467
:1036A00042EA0122A280D3F89824D3F89C3442EA5B
:1036B0000323E38010BD00BF0070024013B5FFF785
:1036C00015FB0F4B9A7B032A05D16FF48030FFF76F
:1036D0008BFB02B010BD1C687CB96FF48030FFF723
:1036E00083FB06238DF80430064B8DF806408DF8D9
:1036F00007401B6801A89847EBE706F06BFDE8E779
:10370000F401002014030020014B1878704700BF1B
:103710005F5B002038B50246FFF7CAFA0446104640
:1037200006F0EEFC01238340DB4302F00F001B4A4E
:10373000BCB94FF02001EFF3118581F31188BFF37D
:103740006F8F11680B4013604000154B00F2C5707D
:1037500018605C6004331B6885F31188BFF36F8FBA
:1037600038BD4FF02001EFF3118481F31188BFF3CE
:103770006F8F1168072803EA0103136009D800F569
:103780009470084B002243F82020BFF36F8FBFF3E3
:103790004F8F84F31188BFF36F8FE1E7F0010020B2
:1037A0000078024000700240F7B501464FF0200358
:1037B000EFF3118483F31188BFF36F8FFFF788FA5B
:1037C0000546084606F09CFC012311F0800F03FA21
:1037D00000F02A4E17D1336830EA03020AD00846B7
:1037E000FFF798FF0323AB7384F31188BFF36F8F48
:1037F00003B0F0BD2A60C043214A03403360136820
:1038000003401360EEE701F00F02072A0FD880296A
:103810001C4F1D4B28D002F2DA3252003A601A686F
:103820001F68D2B242F002023A431A601B68144F7A
:1038300032683B6862EA030C1CEA000FD4D022EA2B
:1038400000021843002332602B600323AB738DF812
:1038500007300E4B386006228DF804208DF80610D4
:103860001B6801A89847BFE740F2B4723A601A6833
:103870001F68D2B242F00402D6E700BF80010020E8
:10388000F001002000780240047802401403002078
:10389000F7B5164B164CD3F880542368154EDA430F
:1038A000154B37781B6892B238461A4306F028FC4D
:1038B000012303FA00F0104202D03846FFF774FFEC
:1038C00005F080056FF001103570FFF78DFA236861
:1038D00043F00103236002A800230193052300F8AD
:1038E000043D064B1B68984703B0F0BD00700240D2
:1038F000F00100205F5B0020800100201403002005
:10390000554B2DE9F041D3F80453002229461646C1
:10391000012400297CD1FFF7CBF9002869D14F4B56
:103920001B78002B65D1960263D54D494C4E40F271
:10393000A9730B604B4B1C6814F0FF041CBF186884
:10394000044040F2AA700860186810F0FF001CBF25
:103950001968084040F2AB713160196811F0FF013D
:10396000B4461CBF1E68314040F2AC76CCF8006013
:103970001E6834403C4E08D037682743376040F219
:10398000A977CCF800701C601C68354F40F2AD740C
:103990003C601C68204008D0346844EA004434602D
:1039A00040F2AA743C60186018682D4840F2AE746A
:1039B0000460186801400DD0CC0748BF42F40002F3
:1039C000C806274840F2AB74046019601B6848BF02
:1039D00042F00102336833F001111CBF05F0807022
:1039E000024313F0011F04D06B0544BF316042F461
:1039F00080621E4F02F4000622F400044FF001081A
:103A0000E4B9FFF703FB2EB3BDE8F041FFF740BF79
:103A100091FAA1F31648B3FA83F39F00384407687C
:103A20003FB10660BFF36F8FBFF34F8F04FA03F00F
:103A3000024304FA03F321EA03016AE794FAA4F5C6
:103A4000B5FA85F557F8253008FA05F5984724EAC0
:103A50000504D5E7BDE8F081007002405D5B002001
:103A600000780240047802401803002068BA010080
:103A700000710240F8B5114E114A34681268240CE6
:103A80002404144301271CB940F2FF133360F8BD2E
:103A900094FAA4F5B5FA85F5E8B20F2DC6BF103833
:103AA000C0B240F0800000F00F03072B01D8FFF7F1
:103AB0007BFE07FA05F524EA0504E4E7F00100209F
:103AC000800100200D4B802210B52720C3F88421EF
:103AD00003F0B8FB80B10A4CFFF7CCFF0023C4F819
:103AE0000435BFF36F8FBFF34F8F272003F096FB92
:103AF0004FF0FF33C4F8083310BD00BF00E100E011
:103B00000070024008B5FFF7DDFF094BD3F804232E
:103B1000C3F808230022C3F80025BFF36F8FBFF35B
:103B20004F8FFFF7E3F8034B01221A7008BD00BF67
:103B3000007002405E5B002038B54FF02003EFF3C9
:103B4000118583F31188BFF36F8F0F4B1B7803F040
:103B5000FF0433B9002485F31188BFF36F8F20462B
:103B600038BDFFF787FF094AD2F8003413F4007319
:103B7000F0D10121C2F82C15D2F80014890544BFF8
:103B8000C2F82C351C46E6E75C5B00200070024062
:103B900010B50446FFF708FE134A04F00F0064B2A4
:103BA000002C4FF00103B4BFD2F81015D2F8141551
:103BB00003FA00F36FEA0303B5BF0B400B40C2F8F2
:103BC0001035C2F81435BFF36F8FBFF34F8F074B1B
:103BD000074A33EA240428BF14460123225C934099
:103BE000014AC2F8083310BD0070024054BD010004
:103BF0004BBD0100F8B5234A234B244D47B233EAAD
:103C0000270328BF134600F00F0401211B5D01FAB2
:103C100003F3C5F804330646FFF73AF888BB002FD4
:103C2000B4BFD5F81035D5F8143501FA04F1B5BF95
:103C300019431943C5F81015C5F81415BFF36F8F54
:103C4000BFF34F8F013C062C1BD8002F19DB4FF020
:103C50002003EFF3118483F31188BFF36F8F304695
:103C6000FFF758FD304606F04BFA094A012303FAE4
:103C700000F0136823EA0003136084F31188BFF394
:103C80006F8FF8BD4BBD010054BD010000700240B4
:103C900080010020030610B504460AD400F00F038B
:103CA000072B06D89B00074AD358012B01D1FFF7F9
:103CB00031FD054BC3F81845BFF36F8FBFF34F8F2E
:103CC00010BD00BF447402400070024007B502A955
:103CD000002241F8042D084804F05EFD10B100F008
:103CE00043FA0190019818B1012343600023038136
:103CF00003B05DF804FB00BFFC03002030B50C4DA1
:103D00000C4987B000240E23CDE902434FF44072E2
:103D1000094BCDE90444CDE90044284605F0E2FA18
:103D20002846064907F0F2FB204607B030BD00BF29
:103D30008C03002058A40020E94001005DBD010073
:103D400008B500F007FA094806F05FFA04232822B4
:103D50000748084907F0D6F9074B084A1A604FF49C
:103D60000040BDE8084000F01BBC00BF6803002015
:103D70007003002034100120D814012037A2010064
:103D8000F8B50F4BBFF35B8F002553E8007F43E886
:103D90000052002AF9D1BFF35B8F0A4C0A4E361B42
:103DA0003611B54200DBF8BD63685B792BB123683F
:103DB000DB6813B139462046984701351034F0E7E7
:103DC00060030020F8B9010008BA0100064BBFF3F8
:103DD0005B8F53E8002F013243E800210029F8D11E
:103DE000BFF35B8F704700BF60030020044A054BA0
:103DF0009B1AB1EBD30F34BF52F83100002070474B
:103E0000A8B90100F8B90100064B4268C31A1B119A
:103E1000013313714268012311605371024A137018
:103E2000704700BFF8B90100605B0020F8B5114B86
:103E3000BFF35B8F53E8004F621C43E80021002969
:103E4000F8D1BFF35B8F2CB90B4D0C4E761B36119E
:103E5000B44200DBF8BD2701EB191B7B43B1EB59E2
:103E60005B6903B1984704220021E819FFF7CCFFF2
:103E70000134EDE764030020F8B9010008BA01003D
:103E800048B1054B984205D3A03398422CBF00207F
:103E90000120704700207047341001202DE9F84FB1
:103EA000524B1B78044603B960B34FF02003EFF385
:103EB000118683F31188BFF36F8F4D4806F0B5F973
:103EC000054686F31188BFF36F8F78B1BFF35B8F20
:103ED000484B53E8002F013A43E800210029F8D16C
:103EE000BFF35B8F8CB1284606F07CFA24B9424BB5
:103EF0001B680BB1FFF744FF3D4806F094F9041C22
:103F000018BF01242046BDE8F88F3C4B1B78DBB975
:103F10002B7ADB0718D406F078FA8146284606F09B
:103F200041FA26462246CC4623464FF0010E1CF8A5
:103F3000011B09B198420ED8314B324ADFF8DCB090
:103F40009B1AC3F3C90AD6B92F4E304FBF1B3F117E
:103F50004FF0000847E0252902D182F00102E6E790
:103F6000002AE4D041F02007613F192FDFD87329E0
:103F700004BF0EFA03F2164301330022D7E7B6FA64
:103F800086F7C7F11F073946284606F00EFA204B80
:103F90009842024602D31F4B984213D31046FFF7B4
:103FA0006FFF78B91C4B9A420CD0012363F30208CF
:103FB00060F3C5086AF38F1843464A4639465846A7
:103FC00006F05EF9012303FA07F726EA0706BAE7C7
:103FD00073685B7923B1336829461B68304698477C
:103FE00008F101081036B845F2DB7CE7605B002081
:103FF000680300205C03002060030020615B002058
:10400000B0B90100A8B90100F8B9010008BA01006F
:104010005CB701006CC801009BBD010065BD0100DB
:104020001A4B70B51B68418105469847184CE860EB
:10403000BFF35B8F54E8003F013344E80032002AAD
:10404000F8D1BFF35B8F4FF02003EFF3118683F3BA
:104050001188BFF36F8F0F48294606F0DAF886F310
:104060001188BFF36F8F0C4B1B7823B10020BDE884
:104070007040FFF713BF23680A2B06D1074B18685F
:1040800018B1BDE8704005F043B870BDD8140120E8
:104090005C03002068030020615B0020F80300201F
:1040A000F8B50E4F3D7875B90D4C0E4EFFF7BEFEBC
:1040B000361B3611B54207DB0020FFF7EFFE002864
:1040C000FAD101233B70F8BD63685B791BB12368AB
:1040D00020461B69984701351034EBE7615B0020EF
:1040E000F8B9010008BA010008B5FFF79FFE05F016
:1040F00035F8094A106028B1084B1B68092B01DD0F
:1041000005F006F80020FFF7C9FE0028FAD14FF4A9
:104110007A7004F0DDFFF5E7F80300205C0300206F
:1041200007B504380190BFF35B8F50E8003F5A1E7B
:1041300040E800210029F8D1BFF35B8F012B03D1A8
:1041400001A9034804F056FB03B05DF804FB00BF6F
:104150007003002020231A460149024806F0D2BF0E
:10416000D4100120FC03002073B502AC002344F8F6
:10417000043D094E0120FFF791FE0546FFF726FE9C
:1041800000222146304604F007FB08B1002DF1D192
:10419000019802B070BD00BFFC03002007B502A962
:1041A000002241F8042D054804F0F6FA10B1FFF79B
:1041B000DBFF0190019803B05DF804FBFC030020D5
:1041C0007FB5047A457A019014F001044FEA151581
:1041D00010D0019B1A7A920706D504AC5B6944F8AB
:1041E000043D104D039BB3B901A90E4804F002FB36
:1041F00004B070BD002DECD0AC420198E9D221464C
:1042000006F0D3F80646FFF73BFE10B13046FFF745
:1042100087FF0134F0E71E682146284604F0EAFAD9
:104220000396DFE7FC0300200EB403B503AB0146A1
:1042300053F8042B0448019305F000FD002002B060
:104240005DF804EB03B07047B1A701002DE9F04F12
:1042500085B011F00204064690469DF8387001F0D2
:10426000010901F0080507D011F0440F37D11A46B3
:104270003249FFF7D9FF0446B9F1000F0AD0304B9D
:10428000304953F82720304B3046002A08BF1A46E1
:10429000FFF7CAFF3DB12D4B2D4953F8272030467B
:1042A000FFF7C2FF0546B8F1000F44D0012303FA1F
:1042B00007F7284B17F0100F274F18BF1F46BDF800
:1042C00040109DF83C00FFF791FD3946024630460C
:1042D000FFF7AAFF2844204405B0BDE8F08F1F4A2D
:1042E000116831B31E4A4FF4616E1468B3FBF4F3E6
:1042F0004FF47A7CB3FBF1F4B4FBFEF20EFB124EEA
:1043000001FB14340CFB04F44FF03C0AB4FBF1FB4A
:1043100001FB1B44BEFBFAF30CFB04F4B4FBF1F10C
:10432000CDE901B10AFB13E100910E49FFF77CFFD3
:10433000A1E708469FE7084FC1E700BF00BE0100A4
:10434000CCBA010025BE0100F2BD0100E0BA0100B7
:1043500028BE0100F7BD0100FBBD010018040020CC
:104360001C04002009BE01002DE9F8439846089B73
:104370001746DA0604460E4605D49B064CBF214973
:104380002149FFF751FFDFF888900025454528DBDC
:10439000DFF88080DFF880900025BD4227D2725D73
:1043A00049462046FFF740FF0135082DF5D1174952
:1043B000DFF85C80DFF864902046FFF735FF0025CA
:1043C000AF4219D9725DA2F120035F2B28BF2E22C4
:1043D00049462046FFF728FF0135082DF0D1BDE8FA
:1043E000F88349462046FFF71FFF0135CEE74146D7
:1043F0002046FFF719FFD7E741462046FFF714FF95
:10440000EAE700BF64BE010063BE0100C3BD010056
:10441000C1BD0100BFBD0100B9BD0100C5BD0100A6
:1044200038B50C46E107054603D5084A0849FFF7A9
:10443000FBFEE20608D4A30628464CBF0549064900
:10444000BDE83840FFF7F0BE38BD00BFF2BD010047
:1044500025BE010064BE010063BE01002DE9F047E6
:104460008B7A17460A7A13F007046FEA020288B0C3
:1044700005460E46D2B21BD04989C3F3C20389094F
:104480000291CDE9004302F00102F3683946FFF7DB
:10449000DDFE8146337ADA070CD42946304606F031
:1044A0001DF84CB3224639462846FFF7B9FF23E0F2
:1044B000A146EFE734BB2746EB68069306AA3B46C6
:1044C000A968304605F0F6FF069A6B681A603AB1A3
:1044D000AB68134413F8014CA4F10A035C425C413D
:1044E000284606F058F9069B1F44002BE4D11CB166
:1044F00014492846FFF798FE284606F04CF908B004
:10450000BDE8F087304605F080FF0F490246284697
:10451000FFF78AFE4FF000084FF0080A05AA43464D
:1045200006A93046CDF814A005F0C4FF059A002A6C
:10453000B8D04B46009706A92846FFF715FF059B04
:104540009844EBE7C8BD010025BE010073B5D0E972
:1045500000435D680F4A42F20F738B4228BF0B463F
:104560006846052103F09CFC2B4606460B2220469C
:10457000094905F0A6FF2B4632466946204605F05C
:10458000A0FF2B461B220549204605F09AFF02B0EA
:1045900070BD00BF87C20100E6BD0100CABD0100B9
:1045A000084A10B50123084C13600021A04204D82A
:1045B00001B11360054B186010BD40085B0001217C
:1045C000F4E700BF1C04002040420F001804002044
:1045D000044B01221A70044B00221A70034B044A48
:1045E0001A607047635B0020FB5B002030040020F2
:1045F000645B002008B5034806F0CDF8024B0122A9
:104600001A7008BD0CBB0100FB5B00200148FFF7DE
:104610009DBF00BF0CBB010010B508460C4605F05D
:10462000B4FE214604480F22FFF718FF2046BDE8DC
:10463000104005F0D7BE00BF0CBB0100044B1B7837
:104640001BB142F2107006F05FBF0A2004F040BDBB
:10465000FB5B00202DE9F74F5B4E337881460F4618
:1046600043B95A4C824609EB07039A4540D3AAEB5B
:1046700009001DE0DFF86C81554D0A24337823B919
:104680004FF0FF31404604F09DF93A46494600207C
:1046900002F0A2FB3378824613B9404604F002FAD6
:1046A000BAF1000F18D001232B7033783BB938468C
:1046B00003B0BDE8F08F5CB92C704FF0FF340020E0
:1046C00002F0D4FB0028F2D02B78002BF3D1EEE7D8
:1046D000013CFFF7B3FFF2E72B7813B1013C04D1A3
:1046E0002C702B78002BC9D1E1E7FFF7A7FFF8E783
:1046F0001AF8012B23680A2A5FD1364D5A1B012A6A
:1047000004BF0133236023680D220A2603F8012C1D
:104710001E705A1C304B2260D3F800B0BBF1000F62
:1047200026DD2E4B196819BB2A490193BBF1630F93
:10473000A2EB050201F11700D846A8BF4FF06308AD
:1047400006F0DCF917222649224806F0EEF9226825
:10475000019B17322260BBF1090F4FF001021A6072
:104760001DDC202308F130086B7585F81480EB748C
:104770004FF0FF311B4804F025F922681549521B00
:10478000002002F029FB0546164804F08BF9124B75
:104790007DB91A6801321A600E4B236063E798FBFB
:1047A000F6F306FB1386303630332B756E753E23D9
:1047B000DDE700221A60094BEDE70B498B423EBF53
:1047C000591C21601A704EE7FB5B0020300400206A
:1047D000635B0020645B0020280400202C04002080
:1047E0004EBE0100C8180120E35B00202DE9F04116
:1047F000114B124D124C5B1B9B106343114C4FF03D
:10480000240ED4F81CC000249C4203D16FF0220077
:10481000BDE8F0810EFB0456776867450AD3366918
:1048200046B197F802808788B84503D13346BDE882
:10483000F04118470134E7E7901A0120481A012097
:10484000398EE338400400202DE9F041114B124D20
:10485000124C5B1B9B106343114C4FF0240ED4F899
:104860001CC000249C4203D16FF02200BDE8F081FF
:104870000EFB0456776867450AD3B66946B197F8C8
:1048800002808788B84503D13346BDE8F041184718
:104890000134E7E7901A0120481A0120398EE338E5
:1048A000400400202DE9F84F9046104B104A0F4667
:1048B0009B1A10499B10064601FB03FA00249146FF
:1048C0004FF0240BA24502D16FF022000BE00BFB4E
:1048D00004935D690DB90134F4E742463946304628
:1048E000A8470028F7D1BDE8F88F00BF901A012033
:1048F000481A0120398EE33807B583788DF80030E7
:104900000379427943EA0223ADF80230C378032BDE
:1049100037D868468DF8043001F050FF002811DACE
:1049200002234FF0000263F302021749174B1848A5
:104930005B1A6FF3C502DB0863F38F129DF800105A
:1049400005F08AFC9DF8000001F0DCFF002811DA78
:1049500002234FF0000263F302020B490B4B0D4898
:104960005B1A6FF3C502DB0863F38F129DF800102A
:1049700005F072FC084B012083F8710003B05DF86C
:1049800004FB0020FAE700BFA8B90100E8B9010064
:1049900076BE010096BE01004004002037B5104CE1
:1049A00002ABE26843F8042D0546A168802001F0BF
:1049B000E5FF019AA3681344A360E3689B1AE360D0
:1049C0005BB9402A09D1402D07D900231A46194660
:1049D000802001F0D3FF0B30F7D003B030BD00BF13
:1049E0004004002008B509480378C3F34113083395
:1049F00050F823303BB100F1080200F11001984754
:104A0000C043C00F08BD1846FCE700BF40040020AB
:104A100037B500220B4601920546002849D1294CA2
:104A200001BB0822214606F00FF8002803DA802097
:104A300001F0FAFE20E0E588256104F13003C4E9C5
:104A4000023515B12378DB0916D0FFF7CBFF00281C
:104A5000EDD02369AB42D4BFE360E5602846FFF7A1
:104A60009DFF09E0D4E90212002A01AB06DC0246F0
:104A700005F0EAFF0028DADB03B030BD05F0E4FF03
:104A8000002804DA802001F0CFFE2846D0E7019903
:104A9000A268E3680A445B1AA260E360002BEBD1D2
:104AA00004F13003A360FFF79DFF0028BFD0E0882A
:104AB000D5E78028E0D1034BDA68002ADCD0D8881B
:104AC000CDE700BF40040020014600F10803BFF31A
:104AD0005B8F53E8002F42F0010043E8000CBCF16B
:104AE000000FF6D1BFF35B8FD30702D4014806F065
:104AF000A2BB7047DC5A00202DE9F74FA04D6B692F
:104B000006460C46904663B9377807F01F07012F19
:104B100000F09C800BD3022F00F0D5806FF01500C1
:104B200002E098470028EFD103B0BDE8F08F72781B
:104B30007088D8F80030092AF0D801A151F822F085
:104B4000694B0100334C01001D4B0100414C010039
:104B50001D4B0100834B01008D4B01001D4B0100DB
:104B6000BB4B0100C54B010000201870587095F830
:104B70007320824214BF022202461A70022323606D
:104B8000D2E7C0B201F0C0FD0020CDE7020A131F3A
:104B9000012BC3D9072AC1D8EB690021C0B21D7807
:104BA000002DBBD05E78964203D1884200F0E080B1
:104BB00001312B44F3E71B78E0E095F872201A707E
:104BC0000123DBE0C4B28DF8074014B985F87240C8
:104BD000DAE74FF0FF08EE690027C146337843B9A2
:104BE000AB691BB10DF1070103209847002F95D049
:104BF000ECE77378042B0DD0052B0ED0022B06D1D9
:104C000096F805809DF80730434508BF01273378A3
:104C10001E44E3E796F80390F9E79DF80730434513
:104C2000F5D1B9F1000FF2D13046FFF765FE074626
:104C3000EDE701287FF472AF002085F8730073E779
:104C400001287FF46BAF85F873009DE77078D8F882
:104C500000300A2807D00B2809D000287FF45EAF67
:104C6000187058708AE70020187027605CE796F883
:104C700004A096F802B0EE69FF27B9464FF000088D
:104C800033783BB9AB6913B1414607209847002000
:104C9000206049E77378042B04D0052B0BD03378C0
:104CA0001E44EDE7B77896F80390BA45F7D1CB45A7
:104CB00008BFB046F3E7BA45F1D1CB45EFD1304656
:104CC000FFF71AFEEBE773783079D8F800808DF89B
:104CD0000700012B2AD022D3032B7FF41FAF748847
:104CE000002C7FF41BAF4FF0000263F30202254952
:104CF000254B5B1ADB0864F3C50263F38F12014690
:104D0000224805F0A9FA9DF8070001F08DFDAB6976
:104D1000002B3FF439AF0DF10701082026E0414692
:104D200001F0D6FD002088F801009EE77488002C71
:104D30007FF4F4AE03234FF0000263F30202114943
:104D4000114B5B1ADB0864F3C50263F38F12014653
:104D50000F4805F081FA9DF8070001F0A1FDAB694D
:104D6000002B3FF411AF0DF10701092098470BE725
:104D7000022AC8F800307FF41EAF5B88236003E787
:104D800040040020A8B90100E8B90100F8BE010004
:104D9000E3BE01002DE9F34150F8303C10F8345CDB
:104DA0001033044610D1C36850F8282C99074CD50D
:104DB000FAB913F0040304D11A461946284605F03F
:104DC00008FD002344F8303C54F8303C10330DD03B
:104DD00054F8206C56B154F8247C54F81C8C04F020
:104DE0002BFA00285CD02046FFF76EFE02B0BDE82B
:104DF000F08150F82C1C01AB284605F0EAFC014676
:104E000090B101234FF0000263F302022C482D4BB6
:104E10001B1A6FF3C502DB0863F38F122A4805F0F3
:104E20001BFA6FF01503CDE7019A54F82C3C13449C
:104E300044F82C3C54F8283C9B1A44F8283C54F87D
:104E4000243C134444F8243CBEE750F82C1C01AB2E
:104E5000284601F011FE0028E3D1019E54F82C3CB5
:104E6000334444F82C3C54F8283C9B1B44F8283C21
:104E700054F8243C334444F8243C002EA1D0284666
:104E800001F090FEB6FBF0F303FB1060002898D110
:104E900054F8283C002B94D0284601F031FE93E7CB
:104EA00044F8200CA4F1180004F05EF954F8303CEA
:104EB00048339BD0424639462846B04796E700BF64
:104EC000A8B90100E8B9010040BF01000A4930B5A6
:104ED0000023442404FB031292F87450854206D147
:104EE000906F10F1100F14BF0020012030BD01336E
:104EF000042BEFD10020F9E74004002073B5214CCA
:104F00000D4606460023442101FB03F2A01890F849
:104F10007400B04223D1743214446B1E012B1CD890
:104F200014BB012D19D101AB01220DF10301304653
:104F300001F0A2FD019B002BF5D101224FF00001F1
:104F400062F3020163F3C5010F4A104B10489B1A2C
:104F5000DB0863F38F1105F072F902B070BD013305
:104F6000042BD1D10024D8E704F066F9343408B119
:104F7000012D03D12046FFF70DFFEEE72046FFF796
:104F8000A3FDEAE740040020A8B90100E8B9010048
:104F900026BF01002DE9F04F85B0054601919046EE
:104FA00099464FF02003EFF3118B83F31188BFF381
:104FB0006F8F364F0026442307F1900203FB06F45F
:104FC00002EB040A002150460393029204F0F8F821
:104FD000DDE9022388B93E19B36F13F1100F22D116
:104FE0005046019304F0C0F8019B8BF31188BFF386
:104FF0006F8F184605B0BDE8F08F0136042EDDD165
:1050000001234FF0000163F30201214A214B2248A2
:105010009B1ADB086FF3C50163F38F1105F00FF9DD
:105020006FF00B03E1E7019BC6F88400C6E91F3867
:105030000E9BC6F888300F9BC6F88C306FF00F03BC
:1050400086F87450C6F8B490B367284601F0AAFDFC
:1050500068B1284601F0A6FDB8FBF0F303FB108011
:1050600028B1D6F8B43043F00403C6F8B43019F0D0
:10507000020F06D004F1A8003844FFF725FD0023F5
:10508000B3E7284601F03CFD0346AEE740040020AC
:10509000A8B90100E8B901000BBF01002DE9F041FA
:1050A000104D00246FF0470705F1A8084FF02003CA
:1050B000EFF3118683F31188BFF36F8F2B199A6F6B
:1050C000103204D19F6708EB0400FFF7FDFC86F364
:1050D0001188BFF36F8F4434B4F5887FE6D1BDE803
:1050E000F08100BF400400202DE9F74F1F4C204EF7
:1050F000204A361BB31002FB03FA031F012B804624
:10510000894624D81C4D95F8713003B3FFF7C6FFCC
:1051100027464FF0000BDA4516D0396A0022387F57
:10512000D3B2984203D80BF1010B2437F3E701EB1C
:10513000C30301921879009101F002FC019A0099D1
:10514000002802F10102EADA002385F87130002517
:10515000AE4202D103B0BDE8F08F2819C36813B185
:105160004A46414698472435F2E700BF481A0120D5
:10517000901A0120398EE33840040020054B064A7E
:105180001A62064A5A62064A9A62064AD8615A6107
:105190000020704740040020F94A0100ED4701005B
:1051A000A5480100494801002DE9F743384E96F81B
:1051B0007040002C4ED13748B06101F0EDFC01F099
:1051C00063FA002847DB02AD402305F8084D284666
:1051D000ADF802308DF8044001F0F0FA00283ADB17
:1051E000802728468DF8007001F0E8FA002832DBAD
:1051F0002949204601F0BEFC00282CDB2649384610
:1052000001F0B8FC002826DB244D254B254F5B1B05
:105210009B105F43A74221D1234CDFF8908004F517
:105220008877002501222562C4E9065820461146E8
:10523000443406F057F9A742F4D1002001F062FB94
:10524000002808DB802001F05DFB002803DB012340
:1052500086F87030002003B0BDE8F083D5F82090C8
:105260004FF000082A7F5FFA88F39A4202D801348F
:105270002435CFE709EBC30259F83310107901F058
:1052800079FC08F101080028ECD04FF0FF30E2E78C
:1052900040040020E9500100114A0100481A012091
:1052A000901A0120398EE338D0040020954D01007A
:1052B000104B10B593F87040CCB900F057F990B985
:1052C00001224FF0000162F302010B4B0B4A9B1AC3
:1052D00060F3C501DB080A4863F38F1104F0AFFFE8
:1052E0004FF0FF3010BDFFF749FFFFF75DFF0020D3
:1052F000F8E700BF40040020E8B90100A8B90100A8
:10530000BEBE01002DE9F04F8D498E4A8E4F521AD4
:105310008E49921001FB02F389B08D4A0393002657
:10532000BF1A4FF001130446C7F3C9070193B146F2
:10533000B346B04622784AB9864BA01C984200F08A
:10534000FD80FFF7DFFF09B0BDE8F08F6278052A26
:105350000FD8DFE812F0A0000E00F100A000060058
:105360009D00E2782AB9A27832B309F101095FFA07
:1053700089F922781444DDE701FB025BDBF80400C5
:10538000844207D1DBF80820002AEED049462046A7
:105390009047EAE70132039B9342EDD101234FF09E
:1053A000000263F302026FF3C50267F38F12214616
:1053B000694804F051FF68E02421614DEBE7DBF818
:1053C0002010A57801EBC201087985424CD1012556
:1053D00094F803C08DF81CC094F805E094F804C05C
:1053E0004CEA0E2CADF81AC094F802C08DF818C023
:1053F000E8B21CF0800F02902BD005F1100C019840
:1054000003FA0CFC1CEA000F2BD1029860F07F001D
:105410008DF8180006A8CDE90413029201F084F972
:10542000029ADDE90413E0B99DF81820A27012F089
:10543000800F14BF019B019B0A7118BF10354FF0FC
:10544000010215BFAA4002FA05F513432B4301934D
:105450008FE7019803FA05FC1CEA000F01D10298BE
:10546000D6E70135102DB3D101329BF81C108A42CA
:10547000A5DB4FF00001012363F302016FF3C501C7
:10548000364867F38F1104F0DAFE4FF0FF305AE729
:1054900000220123E9E7032E29D1FDF789F905460A
:1054A00098B105F016FB02902D4805F012FB029A08
:1054B000824217D0012262F3020A6FF3C50A67F332
:1054C0008F1A5146274804F0BAFE2046002510F8EE
:1054D000022BD11E5208013A0244002917DA013684
:1054E000F6B246E72946A01C05F01FFBEDE7002EAB
:1054F000EBD1B8F1000F14D14FF00001012363F399
:10550000020168F3C50167F38F111748BBE74554E3
:10551000013A00EB010C92F800E00CF801EC0239C2
:10552000DBE7A4EB080288F80220C2F3072288F820
:10553000032088F80490D2E7A0461AE7104602E755
:10554000481A0120901A0120E0B90100398EE33891
:10555000A8B90100451A0120FBBF010061BF01008D
:105560007EBF010094BF0100DEBF010008B50C48FA
:10557000FFF7C8FE88B101234FF0000163F3020179
:10558000084A094B09489B1ADB086FF3C50163F30E
:105590008F1104F054FE002008BD0148FCE700BF55
:1055A0002C190120A8B90100E0B901001BC00100BD
:1055B00010B50446104803F0D7FD104B1868C4F826
:1055C000B000002198889B79A4F8B40084F82510D5
:1055D00084F8241084F8261084F8271084F8B63054
:1055E00084F8B81084F8B71004F128004022BDE810
:1055F000104005F0C7BA00BFCC05002030BA01004A
:10560000D0F8A4301B68F7B59B681B6A1D7D044663
:105610002846FFF75BFC90B904F150064022314662
:10562000D4F8940004F001FDA4F11807054B009391
:1056300002460197022331462846FFF7ABFC03B030
:10564000F0BD00BFF558010030B5036885689A6861
:10565000104C85B042F2A1004FF40033CDE90103B4
:10566000002385F8B930106AADF80C100A2201A9A0
:10567000007905F0AEF895F8B93013B1002005B007
:1056800030BD012005F040FF013CF4D16FF0040073
:10569000F5E700BFA186010070B504460E4601790A
:1056A0001948154605F0B3F898B902234FF00002E7
:1056B00063F302021549164B5B1A60F3C502DB085F
:1056C0001448A18863F38F1204F0C6FD6FF0120036
:1056D00070BD6378212B0ED0222B08D0202B0FD148
:1056E000072229680C3805F020FA0020F0E76388CB
:1056F00000F8053CF9E70C38072328603360F4E72D
:105700006FF01500E4E700BFC4050020A8B9010050
:10571000D8B901003AC0010010B5014604460D4851
:1057200005F083F890B902234FF0000263F3020200
:1057300009490A4B5B1A60F3C502DB08214663F393
:105740008F120748BDE8104004F086BD012300F821
:10575000033C10BDC4050020A8B90100D8B9010060
:1057600082C0010010B584680023C4F8C0300E4B1D
:10577000C4F8BC00596804F1C00289B9C3E9002229
:105780004FF0FF320021094805F0ACFE084B002025
:10579000C4E90430074BE060A061C4E9073010BDE4
:1057A0000A605A60ECE700BFC4050020CC05002069
:1057B00071A8010001560100014600F10803BFF382
:1057C0005B8F53E8002F42F0010043E8000CBCF16E
:1057D000000FF6D1BFF35B8FD30702D4014805F069
:1057E0002ABD7047DC5A0020F7B50D1E0746144647
:1057F00002F1280618DD2A463146D4F8A80004F044
:10580000C1FB854210D901234FF0000263F302026D
:105810001149124B5B1A6FF3C502DB08291A63F3B7
:105820008F120F4804F018FD012384F825306368B7
:1058300033B194F827301BB104F10C00FFF7BCFF23
:10584000084B009301940123402231463846FFF76C
:10585000A1FB03B0F0BD00BFA8B90100D8B9010099
:10586000A8C00100E957010070B506460D46014683
:105870001C4804F0C0FF044690B902234FF0000218
:1058800063F302021849194B5B1A60F3C502DB0887
:10589000314663F38F121648BDE8704004F0DCBC5B
:1058A0000A2D1DD023681B68032D9B6804F8BC5C7F
:1058B000A0F1BC0007D0042D01D0012D10D1BDE80E
:1058C0007040FFF775BE1B6A02460021187BFFF788
:1058D0008BFF012304F8983C04F8963C04F8953CAF
:1058E00070BD00BFC4050020A8B90100D8B90100EF
:1058F00061C0010010B50123144682F824300C4821
:1059000003F032FC636833B194F826301BB104F124
:105910000C00FFF751FFD4F8AC30D3E900239A42D2
:1059200005D004F11800BDE81040FFF745BF10BDD9
:10593000CC050020F8B585682B78032B17464FF06F
:1059400000041FD185F82440D5F8AC0004F01AFB00
:10595000B842064610D202234FF0000263F302025F
:1059600009490A4B5B1A64F3C502DB08391A63F371
:105970008F12074804F070FC05F11800FFF71CFFB8
:105980003046F8BD2046FCE7A8B90100D8B90100AF
:10599000A8C0010007B502AB012203F8011D19469A
:1059A000FFF7C8FF6421034803F00AFC03B05DF869
:1059B00004FB00BFCC05002010B54FF02003EFF32F
:1059C000118283F31188BFF36F8F154C237833B99D
:1059D00082F31188BFF36F8F6FF0440010BD013B5D
:1059E000DBB2237033B182F31188BFF36F8F6FF096
:1059F0000F00F3E70B4B1878012138B1217082F3C7
:105A00001188BFF36F8F6FF00A00E7E7197082F318
:105A10001188BFF36F8F044A11601870DEE700BF72
:105A2000FE9B0020FD9B002004000040F8B54FF0D5
:105A30002002EFF3118382F31188BFF36F8F294A9D
:105A40001078441C147080B183F31188BFF36F8FFA
:105A50004FF08043D3F80C3403F00113B3F1011F6E
:105A60000CBF00206FF0430009E01F4D2F783FB1BD
:105A7000107083F31188BFF36F8F6FF00A00F8BDC9
:105A800001262E7083F31188BFF36F8F4FF080448F
:105A900019B3384601F0C2FBC4F80071D4F80433DE
:105AA000C4F804632660D4F8002192B10022C4F83F
:105AB00000210E4A13F0010F4FF0010308BFC4F894
:105AC00008330020C2F8803101F098FB00232B70CE
:105AD000BEE720BF40BF20BFE5E7C4F80011266045
:105AE000F4E700BFFE9B0020FD9B002000E100E0EA
:105AF00070B54FF02002EFF3118382F31188BFF3EA
:105B00006F8F244D2A789AB183F31188BFF36F8F7A
:105B10004FF08042D2F81C34D2F8182403F003036B
:105B200043F48033934314BF6FF04300002070BDF3
:105B300001242C7083F31188BFF36F8F4FF08043E3
:105B4000154EC3F804210225C3F81815C3F80453F1
:105B500011F0030134604FF01806C3F80863C3F86E
:105B60000C21C3F81021D3D11022C3F83825C3F873
:105B70000463D3F81824D20302D4C3F80453C7E74C
:105B8000C3F80443FFF752FF0028C1D1034BC3F809
:105B90000041BDE7FC9B00200800004000E100E060
:105BA0002DE9F0434FF080434E4DD3F80891D3F8E0
:105BB0000423D3F800E18046D3F80403D3F804C1EA
:105BC000D3F80C11D3F810412F68AE6804350034B7
:105BD00085B002F0010218BF01242D68B9F1000F51
:105BE00003D04FF00009C3F80891BEF1000F69D04F
:105BF0004FF080434FF0000EC3F800E15AB14FF070
:105C00008043DFF8E4E001224FF00209C3F80823E3
:105C1000CEF800901A61BCF1000F41D161B1324B56
:105C20004FF08049002119604046C9F80C11FFF778
:105C3000C3FE0123C9F8143074B14FF08043002132
:105C40000124C3F810114046C3F80443FFF7EEFEE9
:105C500010B9264BC3F800414FB1224B00221A6005
:105C60001B6801934FF48E70019B00F0D3FC4EB182
:105C70001F4B00221A601B6802934FF49270029B24
:105C800000F0C8FC55B31B4B00221A601B6803933D
:105C9000039B4FF4907005B0BDE8F04300F0BABC30
:105CA0004FF080430022C3F804218207B6D50222B8
:105CB000C3F80823D3F81C349B07AFD10029BCD00C
:105CC0000124ACE7002AA6D04FF08043D3F80C346F
:105CD00003F00113B3F1011F9DD190E705B0BDE8BA
:105CE000F08300BF1C010040340C004000E100E0E4
:105CF00024010040200100400146014805F09BBA04
:105D00001C190120020600F00F0303D5072B05D94B
:105D100009487047072B07D90848704708482422CC
:105D200002FB03002830704703F10900044B2422D2
:105D300002FB0030F6E700BF8C160020D0170020D1
:105D40004415002070B50546244802F0F5FB98B9CB
:105D500001224FF0000162F30201214B214A9B1AFC
:105D600060F3C501DB0863F38F111F4804F067FA85
:105D70006FF01204204670BD1C4E3178FDB141BB5E
:105D800043681B689847044614B314F1440F1FD0AE
:105D900001224FF0000362F302031249104A144833
:105DA000521A1449D2086FF3C50362F38F13002D02
:105DB00008BF01462246104804F062FADAE751B102
:105DC000436829465B68984710F1100F0446DBD101
:105DD00035700024CEE70C46CCE700BFE4C00100DC
:105DE000F0B90100A8B9010053C10100FF9B0020D8
:105DF00078C1010072C101007DC101000949BFF3F2
:105E00005B8F51E8003F43F0010241E80020002889
:105E1000F7D1BFF35B8FDB0703D40839024805F0E5
:105E20000ABA704754150020DC5A002010B5054C02
:105E30000021204605F004FA18B1043005F074F989
:105E4000F6E710BD1C19012073B56C46002318221B
:105E50002146224802F010FD002837DA204B214D60
:105E6000214801264FF00001ED1A66F302016FF39D
:105E7000C501C5F3C90565F38F1104F0E0F9FFF71B
:105E8000D5FF002318222146144802F0F5FC002813
:105E90000EDA4FF0000166F302016FF3C50165F3FE
:105EA0008F11124804F0CBF90023184602B070BDE0
:105EB000009B94E803001A1D82E8030004221A756F
:105EC0001846FFF719FFFFF799FFEDE7009B94E8ED
:105ED00003001A1D82E80300E7E700BF7C180120D9
:105EE000A8B90100F0B90100B6C20100D4C2010096
:105EF0002DE9F041867807463046FFF703FF330669
:105F00000546FC7813D5002C43D1FFF79DFF0346CF
:105F1000002852D0012285F8224002750322027423
:105F2000DD60FFF7E9FEBDE8F041FFF767BF5CB158
:105F3000012C2ED1FFF788FF034600283DD085F8BD
:105F4000214004750474EBE7FFF77EFF002834D08E
:105F5000BA7812F0800F02F00F03194A0FD0072B06
:105F60009BBF142101FB0323D2F8A836D3F80836CF
:105F7000EB600123037502230374C560D1E7072B8F
:105F80009BBF142101FB0323D2F8A837D3F80837AD
:105F9000EEE701224FF0000362F3020309490A4AC7
:105FA0000A48891AC9086FF3C50361F38F13324693
:105FB0002146BDE8F04104F063B9BDE8F08100BFBF
:105FC00000700240F0B90100A8B901008AC20100C6
:105FD0002DE9F041064688B01822002102A804F0FD
:105FE000D1FD3378013B052B20D8DFE803F09F0378
:105FF000141F8F1603238DF814300024FFF724FF9D
:10600000034698B105A9047500F10C0203C982E8A2
:10601000030018461EE00423EDE7B7783846FFF783
:1060200071FE827A054622B1032A6BD908B0BDE819
:10603000F0813B06F47812D5002C50D1FFF704FF15
:1060400003460028F2D0012285F82240027503227F
:106050000274DD60FFF750FEFFF7D0FEE6E75CB1AB
:10606000012C3CD1FFF7F0FE03460028DED085F876
:10607000214004750474ECE7FFF7E6FE07460028AC
:10608000D4D002234FF0010880F814800374C56057
:1060900005F10C01B07804F086F8014670B124488F
:1060A000244B4FF000021B1A68F3020264F3C5028E
:1060B000DB0863F38F12204804F0CEF81F4AE9682A
:1060C000B2F8B0328B4206D95B1AA2F8B03204F0B3
:1060D00081F83846BEE70023A2F8B032F9E7012183
:1060E0004FF0000361F3020362F3C5031149104A44
:1060F0001348891AC90861F38F133A46214604F000
:10610000BFF893E73046FFF7F3FE8FE76846FDF7E9
:10611000AFFA9DF80130052B04D19DF8003013F043
:10612000600F83D0074B0593012467E7022465E7DE
:10613000A8B90100F0B901006AC2010044150020AD
:106140008AC20100B01600202DE9F0410025DFF8D9
:1061500080812E4665F07F00C0B2FFF7D3FD07694E
:106160000446EFB900F110013B464022404602F0E0
:1061700083FB002814DA01234FF0000263F30202CC
:106180004F49504B50485B1A67F3C502DB0863F375
:106190008F12294604F060F86FF00B00BDE8F08123
:1061A0002369E660C4E9063301231D44082D84F801
:1061B0002030267284F8216084F82260CAD100253C
:1061C000DFF80C812E46E8B2FFF79CFD0769044614
:1061D00047B900F110013B464022404602F04CFB1B
:1061E0000028C8DB0127236984F820703D44082D6E
:1061F00084F82160C4E90633E660267284F82260E0
:10620000E1D13249D1F858510C46CDB92B464FF463
:10621000806201F5AC712E4802F02EFB00280FDAE7
:10622000284B274A2B484FF0000167F302019B1AC5
:1062300065F3C501DB0863F38F1104F000F8ABE7E9
:10624000D4F85831D4F89C52C4F86031C4F86431A1
:106250000126002384F86861C4F8543184F8693158
:1062600084F8503184F86A31B5B92B464FF4806216
:106270001949174802F000FB00280DDA114B104AAB
:1062800016484FF0000166F302019B1A65F3C50141
:10629000DB0863F38F11D0E7D4F89C32C4F8A43242
:1062A0000020C4F8A832012384F8AC32C4F8980264
:1062B00084F8AD0284F8940284F8AE026EE700BF61
:1062C000A8B90100F0B90100EEC00100441500209A
:1062D0006018012010C10100E017002031C1010049
:1062E0002DE9F04FA94BAA4AAA4D87B09B1AC3F3D8
:1062F000C903074600930021A74804F0A1FF064602
:1063000010B907B0BDE8F08F6B79317D5BB900291A
:10631000F1D1327B042A68D8DFE812F0F700B80028
:10632000C20005011101042900F2608101A252F8A6
:1063300021F000BF136301004963010055650100AE
:106340007D650100B165010017F8043C6BB90122BD
:1063500062F3020963F3C509009BF1688F48497A2B
:1063600063F38F194A4603F077FF337CF468032BFD
:106370003BD8DFE803F002427479A3690193082255
:106380000021184604F0FEFB854A019BD2F88014D8
:106390001970D2F884145970D2F88814D2F88C0489
:1063A00041EA00215980D2F89014D2F8940441EACD
:1063B00000219980D2F89814D2F89C2441EA022254
:1063C000DA800822E26000212268607A9047019B0F
:1063D00093F90020002A0CDBDA8852B1B5F8B0320C
:1063E0009B1AA5F8B03203F0F5FE301D04F09CFEB8
:1063F00081E70023A5F8B032F7E794F82130002BAD
:10640000F3D094F82030002BEFD0002384F8213013
:106410004FF0FF3184F820306248019302F0D2FA45
:10642000A269019B03926268059303A9607A0492B2
:10643000FDF77CF85C4A904201460CD00122019B9A
:106440005A4862F3020863F3C508009B63F38F1890
:10645000424603F001FF534802F024FBC5E72368DE
:106460000121607A9847C0E7A37A63B994F8233092
:106470004BB94FF0FF314B4802F0A4FA03F0BFFED6
:10648000484802F00FFB23680221EAE7FDF704F811
:106490000028AAD1FCF724FF0120FFF753FCA4E752
:1064A000002464F07F00C0B2FFF72CFC037A13B124
:1064B000407AFDF79FFB0134082CF2D195F850315A
:1064C0001BB195F85101FDF795FB0024E0B2FFF7F1
:1064D00019FC037A13B1407AFDF78CFB0134082CC8
:1064E000F4D195F894321BB195F89502FDF782FB33
:1064F0000120FCF7ABFF01236B712B68002B3FF4ED
:1065000074AF0021022098476FE700246C71FDF7FB
:10651000F9FA2046FFF716FC2B68002B3FF465AF15
:1065200021460420EFE7002B3FF45FAFFDF704FBAB
:106530002B68002B3FF459AF00210520E3E72A68C0
:10654000002A3FF452AF002B3FF44FAF002106204A
:1065500090474AE707F10C044FF0FF31204602F064
:1065600031FAFFF7F1FD204602F09CFA57F8083C9B
:10657000002B3FF43AAF00210120C4E757F8083C54
:10658000002B3FF432AF00210A20BCE7F0B9010034
:10659000A8B90100441500201C190120F0C2010017
:1065A00000700240581500200000AD0B16C301001A
:1065B0000124009B144864F3020A6FF3C50A63F3D5
:1065C0008F1A514603F03BFE002004F030FAFDF72D
:1065D00099FAFCF77BFEFFF729FCFFF7B5FD204693
:1065E00004F025FA0948FCF761FFFEE6012363F396
:1065F000020B009B06486FF3C50B63F38F1B5A46D3
:1066000003F02AFEF1E600BF3CC30100D15F0100A8
:1066100053C30100B0F5907F10B529D0B0F5927F3B
:1066200013D0B0F58E7F4FF0010410D1FFF70CFCB2
:1066300000B3002202750473FFF75EFB0E4B1B795B
:10664000C3B1BDE81040FFF7D9BB0224EEE70B4B06
:106650000B4A0C484FF0000164F302019B1A6FF3E0
:10666000C501DB0863F38F11BDE8104003F0E7BDFF
:106670000024DBE710BD00BF44150020F0B9010085
:10668000A8B9010052C2010038B51A4C257965BB82
:10669000194BA56004F11400C4E9033504F060FD52
:1066A0002A460121272000F0DBFD1448FCF7FEFEFE
:1066B000134B98421BD1012004F0B9F9FFF744FDB8
:1066C000054608B9012323710E4B1B680BB1FFF778
:1066D00095FB4FF08043D3F83834DB0703D54FF4F4
:1066E0008E70FFF797FF284638BD0025FBE76FF057
:1066F0000405F8E744150020E1620100D15F0100C4
:106700000000AD0B1C190120064B1A7932B15B79E0
:10671000002B0CBF6FF01200002070476FF01200CA
:10672000704700BF4415002008B50279037803F0D4
:106730000F039AB9B3B301234FF0000163F30201D1
:1067400062F3C501184B194A19489B1ADB0863F319
:106750008F1103F074FD4FF0FF3008BD082B0ED9E8
:1067600001234FF0000163F30201104A0E4B114860
:106770009B1A6FF3C501DB0863F38F11E9E7012A68
:1067800010D1082B0ED002234FF0000163F3020159
:10679000064A054B08489B1A6FF3C501DB0863F3F3
:1067A0008F11D6E70020D8E7F0B90100A8B90100A1
:1067B0009BC10100BAC10100D9C1010038B5164B17
:1067C0001B79014623B305782846FFF79BFAB8B139
:1067D00045720B79498883724C1E0C40416012D07F
:1067E00001234FF0000163F302010C4A0C4B0D48EA
:1067F0009B1A6FF3C501DB0863F38F1103F01FFDD4
:106800006FF0150402E0284603F0C8FC204638BDAE
:106810006FF01204FAE700BF44150020A8B9010088
:10682000F0B90100EFC10100194B1A7910B501460A
:1068300052B35B7943B3FFF765FA044608B3837A32
:10684000032B05D8DFE803F0020D090903F0DAFC99
:106850000020A369E060E36110BD0846FCF7E2FE9A
:10686000F6E701234FF0000163F30201094A0A4BE6
:106870000A489B1A6FF3C501DB0863F38F1103F01D
:10688000DEFC6FF01500E7E76FF01200E4E700BFF1
:1068900044150020A8B90100F0B9010017C2010099
:1068A00008B50A4B1A7901464AB15B793BB1FFF74B
:1068B00029FA38B10846FDF7EDF9002008BD6FF060
:1068C0001200FBE76FF01500F8E700BF4415002049
:1068D00038B50B4B1A7905460C4652B15B7943B17A
:1068E000FFF710FA40B12846FCF7A8FE2070002000
:1068F00038BD6FF01200FBE76FF01500F8E700BF3E
:10690000441500200D4938B50B7905466BB1FFF7EA
:10691000F9F968B1047A74B901230372487918B19E
:106920002846FDF767F9204638BD6FF01200FBE7F7
:106930006FF01500F8E76FF04400F5E7441500200C
:106940000D4B1A7910B501466AB15B795BB1FFF75F
:10695000D9F9044650B1037A5BB10846FDF718F93E
:106960000020207210BD6FF01200FBE76FF01500E1
:10697000F8E76FF04400F5E7441500202DE9F043F7
:10698000374C1F46237985B0064689469046002B32
:1069900060D06379002B5DD003065ED5FFF7B2F9B6
:1069A0000546002859D04FF0FF3104F1140002F0E1
:1069B00009F895F8223003F0FF024BB104F11400FE
:1069C00002F070F86FF00A04204605B0BDE8F083CD
:1069D0006C68A86944452BBF4446012385F82320F1
:1069E00085F823302246494604F09FF8EC6007B151
:1069F0003C60AC7A4CB9FCF787FEB04205D003F09E
:106A0000FEFB184802F04EF8DEE7AB690193012760
:106A1000EB6885F8227001A90024304602930394A4
:106A2000FCF784FD104B98420146EAD00F48104B0A
:106A300085F822404FF000021B1A67F3020264F34C
:106A4000C502DB0863F38F120A4803F005FC6FF000
:106A50000404D6E76FF01204B6E76FF01504B3E74D
:106A600044150020581500200000AD0BA8B9010006
:106A7000F0B9010039C201002DE9F0411D461E4B5D
:106A800090461A790F46002A30D05B7973B303061B
:106A90002FD411B9B8F1000F2BD1FFF733F9044609
:106AA00038B34FF0FF31154801F08CFFE3684345E0
:106AB0001E4628BF464657B9B8F1000F07D105B1A9
:106AC0002B600E4801F0EEFF0020BDE8F081324659
:106AD000E169384604F029F8E3693344E361E36887
:106AE0009B1BE360002DECD02E60EAE76FF01200F4
:106AF000EBE76FF01500E8E744150020581500207B
:106B000038B51A4D2A79034632B36A7922B31B0687
:106B100025D4FFF7F7F8044608B34FF0FF3105F12D
:106B2000140001F04FFFE3688BB90125A36984F8D5
:106B30002050E36194F821304BB1FFF785F988B11B
:106B40000575C4600574FFF7D7F8FFF757F90848D3
:106B500001F0A8FF002038BD6FF01200FBE76FF0D6
:106B60001500F8E76FF00B00F5E700BF44150020B3
:106B70005815002008B5074B1B792BB1FFF7C2F859
:106B800028B10160002008BD6FF01200FBE76FF034
:106B90001500F8E744150020014B1860704700BF4E
:106BA0004415002008B5074B1B7923B1FFF7AAF85D
:106BB00020B1406808BD6FF01200FBE76FF01500D0
:106BC000F8E700BF44150020104B002210B4C3F8B2
:106BD00040214FF02002EFF3118482F31188BFF3BC
:106BE0006F8F0B4AD3F804051168401A20F07F43D9
:106BF00023F0FF030B44136084F31188BFF36F8FFE
:106C0000C0F30F2010BC02F0ABBC00BF001001406D
:106C1000F817002037B51E4801F08EFC002833D04D
:106C200043681C4D1B680121984700244FF4807372
:106C3000C5F80845C5F840354FF48033C5F804332E
:106C400003F1804303F58A534FF400321C601B6844
:106C50000193019B104B0121C3F880211120224692
:106C600000F0FEFA112000F0C9FA0C4A012313606B
:106C70002B60D5F8043503F5807323F07F43C5F806
:106C80004035204603B030BD4FF0FF30FAE700BF7B
:106C9000DAC001000010014000E100E008100140EE
:106CA00070B54FF6FE76B0F1FF3F08BF30464FF0AB
:106CB0002003EFF3118483F31188BFF36F8F124D1C
:106CC000124BD5F804151B68421EB242A1EB03001B
:106CD000A8BF324620F07F4022EAE272FF3000EB8C
:106CE000022020F0FF000344591A21F07F411F29A0
:106CF00098BF03F5807323F07F43C5F8403584F3D4
:106D00001188BFF36F8F70BD00100140F81700208D
:106D10004FF02002EFF3118382F31188BFF36F8FDE
:106D2000064AD2F80405064A1268801AC0F30F20FA
:106D300083F31188BFF36F8F704700BF00100140CD
:106D4000F81700204FF02003EFF3118283F311882E
:106D5000BFF36F8F0649074B0868D3F8043582F3F9
:106D60001188BFF36F8F1B1A23F07F4318447047BD
:106D7000F81700200010014010B5114C114AA26113
:106D80000323C4E90433104BE36122664FF48063AC
:106D90000E4A23626266002310220D49A362E01DA1
:106DA0006362E3622367E3666367A26603F079FECA
:106DB0000849204603F075FE2023A37110BD00BFD3
:106DC000FC17002074C30100109C0020009C0020D0
:106DD0007DC3010081C301002DE9F047224D074624
:106DE0001820144600FB07528846936A566AB3423D
:106DF00033D8126AA2EB060909F1FF32944211D886
:106E00004FF0180907FB09932B4422465868414666
:106E1000304403F08AFE09FB075534446C620120BC
:106E2000BDE8F08713449C421BD807FB000005EB2C
:106E3000000A4A46DAF80400304403F076FEB4EB68
:106E4000090406D0224608EB0901DAF8040003F031
:106E50006CFE182303FB0755E0E7013B9B1BA34295
:106E6000CED20020DCE700BFFC170020034A182325
:106E700003FB00239A6A586A801A7047FC170020A7
:106E800004488168406A884203D003494FF0805229
:106E90000A607047A05A002004ED00E00448002377
:106EA0002021C2180133302B82F80013F9D170472A
:106EB00000E100E0094A0A499368096899660949AE
:106EC00058664B6843F080534B60002383F311886E
:106ED000BFF36F8F9368986E704700BFA05A002071
:106EE0002CBC010000ED00E013498A684FF0280037
:106EF0001044EFF3098C80E8F01F202080F3118804
:106F0000BFF36F8F0D4F4FF000664A6A8A603E6094
:106F1000506E0023536680F3118804B506488068DC
:106F200003F0B7FDBDE8044002F1280090E8F01F2F
:106F30008CF3098870470000A05A002004ED00E09F
:106F40001EF0040F0CBFEFF30880EFF30980816996
:106F500031F8021C11F0FF010229FFD001B503F046
:106F60008DFD01BD38B51B4C05461B4802F0C2FF24
:106F7000A36AD90602D5194802F0BCFFA36A1A0712
:106F800002D5174802F0B6FFA36A9B070ED5154835
:106F900002F0B0FF616BA36A180607D5124802F031
:106FA000A9FF1DB1A36A23F08003A362094CA36A61
:106FB000DA0702D50D4802F09DFFA36A9B0602D5B1
:106FC0000B4802F097FFA36AA36A43F0FF03A36292
:106FD000002038BD00ED00E016C401002DC4010002
:106FE00061C4010075C401008EC40100A5C4010084
:106FF000C5C4010038B51E4C05461E4802F07AFF94
:10700000A36AD90402D51C4802F074FFA36A1A05CA
:1070100002D51A4802F06EFFA36A9B050ED51848E8
:1070200002F068FFA16BA36A180407D5154802F0A7
:1070300061FF1DB1A36A23F40043A3620C4CA36A51
:10704000590502D5104802F055FFA36ADA0509D5A3
:107050000E4802F04FFF064A936A43F47F4393625F
:10706000002038BDA36A9B04F5D50948F1E700BFAD
:1070700000ED00E088C301009FC3010061C401006E
:10708000B1C30100CBC30100E1C30100FDC3010096
:10709000C5C4010010B5194C194802F02BFFA36AB2
:1070A0009A0102D5174802F025FFA36ADB0102D539
:1070B000154802F01FFFA36A180302D5134802F017
:1070C00019FF0E4CA36A590302D5114802F012FFB2
